:020000040800F2
:1000000000A0002091260108E9A90008C5160108F2
:10001000E7A90008E5A90008E3A90008000000001E
:10002000000000000000000000000000E1A900083E
:10003000DFA9000800000000DDA900089198000871
:10004000F9260108F9260108F9260108F926010810
:10005000F9260108F9260108F9260108F926010800
:10006000F9260108F9260108F9260108F9260108F0
:10007000F926010861DC0008FDE60008F926010800
:10008000F9260108F9260108F9260108F9260108D0
:1000900019A20008F9260108F9260108F926010825
:1000A000F926010811E50008B7E4000835E5000865
:1000B00005E50008F5E40008E5E40008F926010874
:1000C000F9260108F9260108F9260108F926010890
:1000D000F9260108F5E60008EDE60008F926010812
:1000E000A1980008F9260108790F0108F9260108EE
:1000F000C5E40008F9260108D5E40008F92601083E
:10010000000000000000000000000000F9260108C7
:10011000F9260108F9260108F9260108F92601083F
:10012000F9260108F9260108F9260108F92601082F
:10013000F9260108F926010800000000000000006F
:10014000F9260108F9260108F92601080000000037
:10015000000000000000000000000000000000009F
:100160000000000000000000F9260108F92601083F
:10017000F926010800000000000000000000000057
:0801800000000000F92601084F
:100188002DE9F04F2DED068B754E764B3360AFB0F1
:10019800002373600FF0F2FA18B90FF011FB0BF09F
:1001A80023F80BF0DFF8704B704C1A7842F001021C
:1001B8001A706F4A4FF47001C2F888100022099231
:1001C8000A92226842F4803222600493236803F47E
:1001D80000330A93099B013309930A9B1BB9099BB6
:1001E800B3F5A04FF2D1236813F4003318BF0123ED
:1001F8000A930A9B012B00F089805D4F5D4BFB60E1
:10020800636AB360636ADFF8A4B1DFF8A481DFF83A
:10021800A49143F080736362636943F4FC032EADD9
:10022800636103238DF86A3041F6FF7325F8503D6A
:100238004FF0904029460DF005FE4FF6FF734E48EB
:10024800ADF8683029460DF0FDFD4C4829460DF003
:10025800F9FD4B4829460DF0F5FD584629460DF0A5
:10026800F1FD294647480DF0EDFD284606F02CFA29
:100278001A9B454AB3FBF2F3444A1360444B454A80
:100288004FF0000AC3F800A0434B5A60F02287F8E9
:1002980023200722C3F808A0404F1A60D8F8083076
:1002A8003B6099E80F0085E80F0063691A9843F4EA
:1002B80000136361636943F4001363614FF4885367
:1002C800ABF828304FF48843ABF828301BA90DF061
:1002D800B9FD1DA91C980DF0B5FD642009F08DF934
:1002E8004FF48C722E48514614F043FBE3692D4AB3
:1002F80043F00703E361A36943F4C523A36163697A
:1003080043F4F013636102F1E00E55E0264B12222C
:100318001A606368636063686360636843F480635A
:100328006360636823F47C136360636843F4E813D1
:100338006360236843F08073236022680B4B92014B
:10034800FBD55A6822F003025A605A6842F002024A
:100358005A60636803F00C03082BFAD14DE700BF1D
:10036800800100200FAB0008D02B002000100240B5
:1003780000ED00E00005FA05000400480008004808
:10038800000C00480014004840420F00381C0020B0
:10039800AC1C00203F19010010E000E0C427002039
:1003A800F41C0020A8770108002002400010004833
:1003B800EC100020A4570108937B506892F80FC0F6
:1003C80003F00701DB0800EB83038900186A4FF08C
:1003D8000F0A0CFA01FC0AFA01F120EA010119627C
:1003E800196A10324CEA010172451962E4D10022FF
:1003F80095490023535401320E2AF9D1DFF87CA223
:100408000AF11A02FF2199540133072BF6D18F4ABA
:100418008F4B1360DFF868B28E4A03930321117083
:1004280058460021242214F0A4FA14228BF8002044
:100438008949039B3F6801228BF8182098F805B07A
:1004480081F800B0A3F5F171CAF824108349A3F527
:1004580091730B60824B03EBCB035B78CAF82830AF
:10046800BB0648BFCAF8282000237E4A40F2DC5168
:1004780022F813100133082BF7D113A800211C22EE
:1004880014F077FABBF10E0F03D00BF0EF03082B33
:1004980002D101238DF85C30022008F061FF18B109
:1004A8004088003018BF0120C7F340038DF8523050
:1004B800C7F380138DF85430C7F340338DF84C30B0
:1004C800C7F3C03300F001008DF84F3017F4006314
:1004D8008DF8510007D098F8843103F1FF3EDEF122
:1004E800000343EB0E038DF85030C7F300438DF83B
:1004F8005530B36AB8F84401ADF86000003318BF4E
:1005080001238DF85630C7F300538DF85730B8F8EB
:100518004631ADF85A30F804B8F8523148BF52485D
:10052800ADF85830C7F380438DF85330B8F85031E0
:1005380044BFB0F84C01ADF86000B3F5FA7FADF8F0
:100548005E3084BF0023ADF86030484898F8D43155
:1005580086F82C30002386F82D3043709DF85C30E7
:1005680007F00101002BC7F3C0028DF84D108DF87C
:100578004E200CBF0023022301B902B1013309EB5D
:1005880083094FF0000AD9F810309A1E1A330392E3
:100598000593039A32F8023F03924FF6FF72934293
:1005A80000F072819DF855004FEA132EDAB25FFA17
:1005B8008EF330B110012E4F3F582E48874200F07D
:1005C8005E819DF8520050B1294F2B4807EB021766
:1005D8007968814203D13889012800F050819DF85B
:1005E8004F0050B1224F244807EB02177968814227
:1005F80003D13889042800F042819DF8500050B199
:100608001B4F1D4807EB02177968814203D13889CF
:10061800022800F03481BEF1020F02D19DF84C107F
:1006280004E0BEF1010F04D19DF84D10002900F03F
:1006380026819DF8561051B39DF85C1039BB9DF882
:100648005410F9B1111F1FE08C010020501A00202E
:10065800DE120020CD10002044090020881E002052
:100668006C7D010840100020EC100020AD01002036
:10067800A8770108004401400008004880010020D4
:10068800541A0020A2F10801012998BF0423CA4F77
:100698009DF857104FEA02194F4431B19DF85C108C
:1006A80019B9043A032A40F2D380012B4AD1C24A2D
:1006B800DFF81083079202EB0901FF2391F80DE0A0
:1006C80088F8743088F875304868C8F8847001F183
:1006D80008030989ADF868104FF0000B02218DF866
:1006E8006B1088F878B01AA98DF86AE0069388F834
:1006F80030B0C8F834B0C8F838B0C8F83CB0C8F85A
:1007080070B088F876B088F877B00DF09BFB069B40
:10071800079A997852F809005A460CF0A9FB38460E
:100728000FF01EFCA54BC8F88830A54BC8F88C30D4
:10073800C8F890B0384608F1880108F18C020DF02D
:1007480077FF9CE0022B49D15FFA8AF21C2101FB5A
:1007580002FC9C4ACDF81CC002EB0C08964A88F8AB
:1007680079A0012188F8781002EB09014FF0000BFD
:1007780091F80DE0486888F87AB001F10802098913
:10078800ADF8681088F882B01AA9C8F884708DF896
:100798006AE006928DF86B300DF054FB864B069A92
:1007A80053F8090091785A460CF062FB38460FF06E
:1007B800D7FB844BDDF81CC0834AC8F8882003EBBC
:1007C8000C01824AC8F88C208831C8F890B03846A5
:1007D8000A1D0DF02DFF0AF1010A50E0032B35D157
:1007E8009DF85330DFF8DC81DFF818923BB198F8B8
:1007F8002EB0384608214FF6FF7200231AE0BDF8E4
:100808005E2098F82EB0BDF86030B2F5FA7F0BD9AB
:100818006F49B1FBF2F23846082192B20DF03BFB6A
:100828006C4B49F82B000AE06B49B1FBF2F23846F1
:10083800012192B20DF02FFB684B49F82B00C360E1
:1008480098F82E30013388F82E3018E0042B16D192
:1008580096F82D80BDF858205F4B93FBF2F238468E
:10086800BDF85A30012192B20DF015FB96F82D30E3
:1008780006EB88080133C8F8580186F82D30039B29
:10088800059A93427FF485AE96F82D2086F8782154
:10089800534A544B92F800E0AEF117020027022A9F
:1008A8001F709C461AD8736A3B44D3ED007AF5EE64
:1008B800407AF1EE10FA02D1B36A63BB26E04A4AE5
:1008C80007EB02080FCB88E80F009CF800301037C0
:1008D8000133C02F8CF80030E5D1EDE7434B13F816
:1008E8003E908CF8009003EBCE03D3F804A0BAF145
:1008F800000FE1D04F45DFDA3B4A3B0103EB02082A
:1009080053440FCB013788E80F00F3E7384E3368BC
:10091800DF0424D41DE0374B374A13F83E0010702B
:1009280003EBCE035E68002EF0D000238342EDDA9D
:10093800C3EBC3017218DFF8D080D2F8009041F8F9
:10094800089001EB08079188B9809279BA71013350
:10095800ECE70EF0EF03082B284B20D122E09CF89F
:100968000020012AF5D9264B03EB0212103210336E
:100978009342EED053ED047AB6EE007A67EE877AAA
:1009880043ED047A53ED057A67EE877A43ED057AED
:1009980053ED037A67EE877A43ED037AE7E7BEF112
:1009A8000E0F33D11A7842F010021A70BEF1180FE8
:1009B80033D109F0DFF930E0A8770108F5C800085D
:1009C800D5C900088001002075CF0008CDC80008EF
:1009D80000127A00F5C9000840420F00E5C9000876
:1009E80044090020F01C0020800800206C7D0108CC
:1009F800C4270020F8660108141E0020D41800201F
:100A080088080020C01C0020151E00201A7822F03B
:100A180010021A70BEF1190FCAE709F08FF933688E
:100A2800DFF834B3580358BFBC4BBD485CBF012244
:100A38001A70049B049A1B7843F0040313706269CC
:100A48004FF408534FF002094FF0010A42F4001224
:100A5800ADF8683029468DF86AA08DF86B90626110
:100A68000DF0F0F9AF4AB0491160002008F01CFF02
:100A7800A26942F48052A261E26842F48052E260C4
:100A880062694FF0904642F400326261326A22F4A1
:100A980070023262326A42F4A0023262326A22F092
:100AA80070623262326A42F0A0623262326A22F0C6
:100AB80070423262326A42F0A0423262326A22F4F2
:100AC80070223262326A42F4A022002732624FF06A
:100AD8000308E022304629461A928DF86C908DF86A
:100AE8006D808DF86E708DF86F7005F063FF1022C1
:100AF800304629461A9205928DF86CA08DF86D80C3
:100B08008DF86E708DF86F7005F054FFE168874EB0
:100B180041F48051E160E16821F48051E160844949
:100B2800888820F480500004000C8880888880B26F
:100B380040F480508880088800F4415040F44570A3
:100B480040EA08000880888820F470600004000CDF
:100B580040F4E0608880888B20F40060000407235C
:100B6800000C88830B82088880B240F0400008801F
:100B780070490E60616941F480216161E16941F465
:100B88000011E161216B21F010012163216B41F01B
:100B980010012163DBF8201021F07061CBF82010E0
:100BA800DBF8201041F08061CBF82010DBF8201032
:100BB80021F07041CBF82010DBF8201041F0804183
:100BC800CBF82010402158461A9129468DF86E70AE
:100BD8008DF86F708DF86C908DF86D8005F0EAFED9
:100BE800802158461A91294605F0E4FE3168524B97
:100BF800059A21F0010131603068504901403160A7
:100C08004F493161316841EA0A013160B760F760E4
:100C1800B760B16841F40041B16031683160716812
:100C280021F0784121F400417160316841EA0A01FC
:100C380031601D68434E0493304605F4006339461D
:100C480005F4004B039313F094FE15EA09058DF89B
:100C58003D908DF83E708DF83F708DF83C800DD03A
:100C68003948CDF838A00EA905F0A4FE06220723BE
:100C780032707770F37086F802A05546BBF1000F0A
:100C88000ED0042330480E930EA905F093FE0823D6
:100C980033710723F371012375711D44B371EDB2EC
:100CA800039B6BB1022328480E930EA905F082FE20
:100CB80007233373F373012375731D44B373EDB2C4
:100CC8000EA9082320480E9305F074FE09233372F9
:100CD80007237572F3720123B3721D44E36A1B483C
:100CE80023F4F873E362E36A43F4D873E362636955
:100CF80043F0805343F00103636105F02EFC1AA80A
:100D080005F000FC124B1A93EDB2124B1B93012D08
:100D18004FF000030CBF1A4680221FE0B00D0020E0
:100D280000100048D82B00204193000800540040D0
:100D3800003001400C100020C4270020FFE0CF0045
:100D48007A25E000A81A00200008004808000240A0
:100D580040000050B81A0020000400481F924FF4C9
:100D680080728F4C20924FF480622192202220467C
:100D780022921AA94FF400521C931E932392249393
:100D8800ADF8745005F0CBFB236843F001032360F2
:100D98004FF0A0440A20A36823F04053A360A3683F
:100DA80043F08053A36008F028FCA36823F0804335
:100DB800A360A368A360A36843F00043A3604FF057
:100DC800A0418B68002BFADB8B68764A23F04053EE
:100DD8008B608B6843F000538B609068724B0340C4
:100DE80043F468339360CA68704B134043F400536C
:100DF800CB600A6B013D22F00F0215430D630024FE
:100E080001233219917800296CD05D1C042B375DC1
:100E1800D078EDB24FF0A04E0ED803EB43035A0042
:100E2800DEF830101F23934021EA030107FA02F38A
:100E38000B43CEF8303031E0092B0ED8053B0622A3
:100E48005A43DEF834101F23934021EA030107FABE
:100E580002F30B43CEF8343020E00E2B4FF006019E
:100E68000ED8A3F10A024A43DEF838C01F23934084
:100E78002CEA030107FA02F30B43CEF838300DE0F1
:100E88000F3B01FB03F2DEF83CC01F2393402CEA22
:100E9800030107FA02F30B43CEF83C30092F4FF059
:100EA800A0420FD99369A7F10A0303EB430397699B
:100EB8000721994027EA0101916191699840084307
:100EC80090610EE053697B1E03EB43035769382199
:100ED800994027EA01015161516903339840084359
:100EE80050612B460434102C8BD14FF0A0429368EC
:100EF80043F0010393604FF0A0431A68D107FAD575
:100F0800DA682B4C22F00202DA60DA6842F0020258
:100F1800DA60DA6842F00102DA609A6842F00402A4
:100F28009A60B4F85831002B40F00C86B4F95A2175
:100F3800002A40F00786B4F95C21002A40F00286B6
:100F48001C4B1D4E1B681D48B3F8563003930021F7
:100F58000C2294F85F8194F86971194D13F009FD1A
:100F680000211422304613F004FD164B3360164B53
:100F780016497360164B174A336104230B70052317
:100F880013702B6843F001032B608A469146124B7D
:100F98000022B8F1090F1A709B461FD99046F6E750
:100FA8000800024000030050E010FCFF07C0FFFDEE
:100FB800EC10002050100020AC2B002090270020BF
:100FC800D01800207FE30008BDA10008C806002053
:100FD800295C8F3D08010020F22B0020012202FA33
:100FE80008F140F2BA330B40002B40F09D8511F018
:100FF800450F00F09985192027211AAB0DF038F814
:10100800002800F091853D4B3D4A1A603D4A5A60E0
:10101800062389F801302B6843F002032B602B6804
:101028009A0702D5354B1B689847DFF8E480002300
:1010380088F87931344B4FF47A721A6033689847DC
:10104800324A0023137017B1022F40F07585304BD8
:101058004FF0000CC3F87CC11E200A2101221AABF4
:101068008DF868C0CDF814C00DF002F898B19DF85D
:101078006830DDF814C0482B40F0D385254B264A4C
:101088001A60264A5A60022389F803302B6843F015
:1010980008032B6002E0844600F0C3BD94F8543185
:1010A8000BB18AF8003094F855310BB18BF8003049
:1010B80094F856310BB1154A13702B68144F13F07E
:1010C800080F2FD0BDF90C10DFED156A642291FBD3
:1010D800F2F302FB131212B207EE902AB8EEE77A87
:1010E80007EE903AF8EEE77AE7EE267AB2EE047A5F
:1010F80067EE877AC8ED607A17E000BF9027002076
:10110800CF9F0008799F0008601B0020F32B002068
:10111800800100208806002011A00008E19E000838
:101128008988883C0023C7F88031C44B1A7842F07C
:1011380002021A70C24A4FF4884191614FF48851F3
:1011480011854FF00A0B9946DFF8F4A2BAF814306B
:101158009BB283F48843AAF81430BAF814309BB2CF
:1011680083F48853AAF81430192008F046FA0120AD
:1011780008F09AFB192008F040FA0BF1FF3B002019
:1011880008F092FB1BF0FF0BDED14FF48853AAF84E
:1011980028302B684FF4884B1B07AAF828B009D5CC
:1011A800A84BCAF818B01B689847A74BAAF828B0EC
:1011B80001221A70A54B9FEDA68AD3F800A0DFED97
:1011C800A58A9AF80C3000EE103AB8EEC00A20EE64
:1011D800080A09F0AFFFA04B83ED000A9F4B1B885C
:1011E80007EE903AF8EEE77AB7EE007AC7EE277A7C
:1011F8009B4BB0EE680AC3ED007AD6ED047A994BA2
:10120800994E67EE887AC3ED007A9AF8003007EEB7
:10121800903AF8EEE77A954BC7EE277A4FF0000A36
:10122800C3ED007A77EE677A914BC3ED007A914B64
:1012380083ED027AC3ED008AC3ED018A8E4B83EDFC
:10124800027AC3ED008AC3ED018A09F073FFB0EE9C
:10125800408AB0EE680A09F00DFF20EE006A68EED9
:10126800086A66EE007A854BE6EE887A3046FF21FA
:1012780020EE087AC3ED007A67EE007A1B22F0EEC2
:10128800675AD7EE085AE7EE087A28EE468AC3ED81
:10129800015AA6EE808AC3ED027A83ED038A784B61
:1012A80083F800A013F065FB2A68764B86F800A047
:1012B800012112F0020F19701FBF717003211970FC
:1012C800022118BFB1703046560741BF19784D1C2E
:1012D8001D70032548BF455412F00A0F0CD01A7828
:1012E80004218154511CC9B205254554D11C023230
:1012F800D2B2197006218154049A11688D0641BF33
:101308001A78551C1D70072548BF85540A0608D54C
:101318001A7809258554951C0132D2B21D700A2508
:1013280085546579082D01D00E2D04D11A78561CE4
:101338001E700B2686541A7811F4803F4FF00C0E5D
:1013480000F802E002F101061CBFDFF838E10232C2
:10135800F6B21E701FBF8EF80020434A4FF00E0EE3
:1013680002F806E04A0741BF1A78561C1E7010267C
:1013780048BF86541A78561CF6B24FF0120E11F474
:10138800806F1E7000F802E00ED094F80CE2BEF1F7
:10139800000F09D0DFF8ECE002328EF80020324A64
:1013A8004FF0130E02F806E01A7811F4007F4FF0A0
:1013B800140E00F802E002F101061CBFDFF8C4E0D9
:1013C8000232F6B21E701FBF8EF80020264A4FF078
:1013D800150E02F806E0182D0DD11A781626865437
:1013E800561CF6B24FF0170E00F806E0D61C023273
:1013F800D2B21E7085540E0341BF1A78551C1D7059
:10140800192548BF8554CD0541BF1A78511C19705C
:101418001A2348BF8354002198221B4813F0A9FAC5
:1014280004F0DDFD194B1A4A1A601A4BB4F84E1134
:101438001980194900230B8030E000BFD02B002011
:101448000010004888060020A0060020A8070020F9
:1014580035FA8E3C00000000A4070020040000209C
:101468005C0700206007002019100020BC0700203E
:10147800AC070020C0070020B00700209407002018
:101488001E07002018100020AC190020E40E0020D0
:1014980074120020E80E0020782B00208B709549EC
:1014A8000A60B4F8962190B2934921F813000133E9
:1014B800122BF9D1914E3368D8045CBFB4F89C0163
:1014C80008801B0740F1C6808D4B93F89031062B9E
:1014D80000F2BA80DFE803F004070E3D5877770082
:1014E80045F2F05201E042F6F822864B1A8004F0E9
:1014F8002CFEA8E007EE902ADFED836A814BB8EE58
:10150800E77ADFED827AE7EE267A42F6F82119804B
:101518000023FCEEE77A7E4A17EE901A42F8231071
:101528000133122BF7D17B4A7B4911607B4A40205B
:10153800137007F055FF002800F0868001234FF054
:10154800070A90F90000764A8DE808044021754B97
:1015580074E06C4B42F6F8221A806E4B724A1A609D
:101568006E4B102240201A7007F03AFF00286BD00B
:1015780001234FF0000C90F900006C4A8DE8081028
:1015880040214FF4E13359E05E4B42F6F8221A80CD
:10159800604B674A1A60614B082240201A7007F0B6
:1015A8001FFF002850D001234FF0000E90F90000D3
:1015B800604A8DE8084040214FF4E13308F027F8ED
:1015C800C7F884013CE04F4ADFF8A4C1DFF8A4E182
:1015D800594D5A4C5A4842F6F82111804F490C226D
:1015E800062B0A700ED000238CF800308EF80030DD
:1015F8002B701B232370534B027005221A704FF473
:10160800E1340BE000218CF800108EF800102970EE
:10161800027021214B4A21704B4C13703D4B4B4AB1
:101628001A60402007F0DCFE70B101230025484A0B
:1016380090F9000040218DE82800234607F0E7FFD5
:10164800003018BF012028B9082009F09BFD314B54
:10165800404A1A603368314A13F4804F1FBF08218B
:1016680011702C493C4818BF086042F2010119402A
:1016780003F0010003F4005479B1224944F62065CF
:101688000D8024B1082111702249344C0C6020B11E
:101698000C2111701F4932480860117804395170C3
:1016A800190640F1A3802F4DC8F888510024DFF8AF
:1016B800C8802D48DFF8C4A088F8014021461522CB
:1016C800C8F80440C8F80840053D13F052F9204610
:1016D800CAF800500AF04CFF244B02201B68C8F8D7
:1016E8000C3007F07DFE00284AD1802009F04AFD21
:1016F80074E000BF6C2B0020982A0020C42700202B
:10170800EC100020FE070020CDCCCC3F0000B0C478
:10171800502A0020080000209D080108481A0020CF
:101728001D0B0108A086010089080108710A01083B
:1017380071080108250A0108DC2A0020DE2A002099
:10174800DD290020DF2A002090D003009907010836
:101758000509010801090108D1080108F108010873
:10176800E1080108DE1200200C030020E827002011
:10177800DE290020DD2A0020A4060020C40600205F
:1017880098F801304479C5490C2202FB03125278BB
:10179800A24204D00133DBB2042BF4D9002388F829
:1017A8000130DAF8003098F801201B7890F9000031
:1017B800002B4FF00C0303FB021314BF0324012476
:1017C80000225B7800940192022107F020FFB44BBD
:1017D8001860002889D001200AF0CAFEB14B1868A9
:1017E800B14B00F5C5721A600AF070FFAF4AB04BF2
:1017F8001360B04AB04D8033136033680024DA03B5
:101808002C7040F1AF800DF007F8DFF810C3DFF857
:1018180010A3CDF814C040F22A334FF001081A463D
:1018280060462146049385F8008013F0A2F8DAF8A0
:101838001420A248A24D42F48022CAF81420426A19
:1018480022F00F024262426A032142EA080242621F
:101858004FF4807B02228DF835100CA98DF83420C6
:1018680003928DF83640CDF830B08DF8378005F00A
:10187800A1F8DAF81810039A41F40031CAF81810E0
:10188800298821F440710904090C29801D21E96285
:1018980028462A850EA92C866022C5F814800E9247
:1018A800ADF83E401094ADF84440ADF84640ADF870
:1018B8004840ADF84A40ADF83C8004F0C7FEAA693C
:1018C80042F00802AA616A6C42F400426A64DAF8DB
:1018D800142042EA0802CAF81420AAF57D6A504684
:1018E80004F03BFE1AA804F00DFE049B754AADF8FF
:1018F80074308023DDF814C01A921AA910221F939D
:1019080050464FF40053CDF86CC01C9223931E949C
:10191800CDF880B021942294249404F000FEEB6862
:1019280043F40073EB60DAF8003043F00203CAF8BE
:1019380000300BA80D238DF82C308DF82D808DF8F4
:101948002E408DF82F800EF0EDFA21465E4B1A6876
:101958005E4B43F8212001312029F7D10CF094F98E
:101968000CF092F933685B0553D5594BD7F8CC5432
:101978001D60042007F034FD0421C7F8D00407F0E7
:101988000BFD544B87F8D40408201D6007F028FD90
:10199800514B524C1860082107F0FEFC002187F8D3
:1019A800D5042C22204612F0E4FF8E2363704FF0FA
:1019B8007C0AE0234FF07D08E37084F800A084F8E7
:1019C8002B80474C2C220021204612F0D2FF8A237C
:1019D80063701020A023E37084F800A084F82B80A3
:1019E800C7F8D85407F0FCFC1021C7F8DC0407F04E
:1019F800D3FC87F8E0042020C7F8E45407F0F0FC93
:101A08002021C7F8E80407F0C7FC87F8EC040FF0BA
:101A180035FB3368334A13F4002318BF01231370CE
:101A280007F0C4FD304B1860304B5A79052A194627
:101A380002BF2F4B4FF4C8721A802E4B4FF47A72A4
:101A48001A802D4A137843F0080313702B4A137831
:101A580023F002031370326840F6020313406BB19F
:101A6800274B284A1A60284B03221A70274B012259
:101A78001A70274A00231380264A13808B68336024
:101A8800254B01221A7099F8003063F07F0389F81A
:101A980000302FB0BDEC068BBDE8F08F345801083C
:101AA800B824002050100020400F00200C1C0020FB
:101AB80008130020F0240020B10D00200004004885
:101AC8000044014034440140C4570108B20D0020CD
:101AD800C41800201C19002068190020EC180020E8
:101AE8002119002004280020D0070020EC10002035
:101AF800F60E0020EC2B0020D4180020F52B002037
:101B0800BC180020661200202019002000010020C7
:101B1800E00F0020E20F0020B00D0020210300207C
:101B28000010024035FA8E3CB8F1010F7FF677AA13
:101B38004FF00008FFF72BBA012F7FF6AFAA1F4618
:101B4800FFF77EBA1BB208EE103AB4F95A315FEDCE
:101B58000B7A384A09EE103AB4F95C31B8EEC88A03
:101B680008EE903A28EE278AB8EEC99AF8EEE88A85
:101B78000021B0EE480A29EE279A68EEA78A11706C
:101B880009F0D8FAF0EE40AAB0EE480A09F072FA65
:101B9800B0EE408AB0EE490A09F0CCFAF0EE409A6D
:101BA800B0EE490A09F066FAB0EE40AAB0EE680A4B
:101BB80009F0C0FAB0EE409AB0EE680A09F05AFA95
:101BC80060EE2A6A68EE097AF0EE665AE7EE8A5AFB
:101BD800194B29EE2A6A28EE007AC3ED035AF0EE73
:101BE800465A29EEC00AE7EE4A5AE6EE8A7AA6EE87
:101BF8004A7A29EE299A83ED010A28EE698A29EEA4
:101C0800AA0A83ED009A83ED02AAC3ED045A83ED74
:101C1800058A83ED067AC3ED077A83ED080AFFF794
:101C28008FB9012F7FF63AAA044B002783F800C02A
:101C3800FFF70DBA6C000020841A0020F32B002057
:101C4800954A2DE9F04F1568944C05F59C432033CF
:101C58002DED028B2360924B196889B011F4804FE7
:101C68000592984605D10EF0E9FF10B923790133A2
:101C780023718C4B1F78C7B18B4A1268954240F28A
:101C8800DF80013F1F70DBE0D9F800308748072D5F
:101C980098BF595D864B88BF29461B689847032D16
:101CA8000BD904EB45050137E880804BDFF81C921F
:101CB8001E78FDB2AE42E7D820E0D9F8002005F141
:101CC8000E0302EB83039988DA880028E9D04FF4E1
:101CD8007A73401A5843531A90FBF3F040F6C9033D
:101CE80000F57A70984205DC40F2EE239842B8BFBE
:101CF800184601E040F6CA0080B2D2E70F232779E0
:101D080084F82A3094F82B300193032594F82C306A
:101D1800B7FBF5F505EB45057D1B0393D9F80030B6
:101D28000293DFF8B0A1EBB204930025B54254DA70
:101D38006049019B31F815B04FEA450953B90EF0D7
:101D48007DFF28B1039B002B08BF4FF0000B01E07B
:101D5800DDF804B0029B988A584502D8D88A5845BD
:101D68000ED2E8B20EF014FF032D8346DFBF94F8BD
:101D78002AE00120A8402EEA0000D8BF84F82A00F3
:101D88000EF05CFF18B14C4829F800B021E0049B24
:101D980094F876002AF813B028B9022F15D93F49CC
:101DA800012081F87600BAF80210BAF80000084459
:101DB800BAF804100844414980B229F8010000B279
:101DC800032190FBF1F080B200E058463A4929F827
:101DD800010001350AF1060AA8E794F82A203848D4
:101DE800384BA2F10F014A424A4184F890206AB167
:101DF800354A1268520109D40268D9689A60521AA1
:101E0800C82A1DD9012283F8212019E002689868A0
:101E1800DA605B68121A9A4288BF2A4B4FF00001B9
:101E280084F82B1088BF83F821100025B54207DA03
:101E3800E8B20EF0ADFE204B23F815000135F5E7AA
:101E4800D8F80030DF0405D51F4B1B68DE0701D426
:101E58000EF06AFC059B19681C4B1868837A002BE6
:101E68003AD0013B144D027B35F813301AB1C3F553
:101E78003B6308339BB21BB2A3F57A73B3F57A7F41
:101E8800A8BF4FF47A7323EAE37307EE903A9FED05
:101E9800107AF8EEE77A58E0D42B0020380E0020AC
:101EA800C4270020742B0020702B0020481A002023
:101EB800080000203E0E0020982A0020B00E0020C6
:101EC800E8270020782B0020141000206C2B00201D
:101ED80000007A44660E0020D8F80020150440D58A
:101EE800D4F89420934E8A1A002A3ADB01F59C42D2
:101EF8002032C6F89420904AC07A55798F4A32F831
:101F0800152096F89850013592B292FBF0F205F040
:101F18000F0086F89800304480F899201A468848BF
:101F2800185C01330244102B92B2F8D112B292FB22
:101F3800F3F31BB2642BA8BF642323EAE37307EE11
:101F4800903A9FED807AF8EEE77AC7EE877A7E4A74
:101F58009FED7E7A67EE877AFCEEE77A17EE903A85
:101F68001380D8F800307A4F13F4807F00F009818D
:101F7800784BDFF8E491994205D999F8022012B913
:101F8800012289F8022099F80220002A00F0F9803D
:101F9800714A3E7892F82150704A681E454211688D
:101FA8004541002DC1F38063C6F380060193924634
:101FB80014BF4FF0000B4FF0030B99F82020052AAF
:101FC80000F2D980DFE802F0034D527584A1002E9B
:101FD8003AD0D4F8AC00B4F8B01007F0A2FA01284F
:101FE80009D15F495F4A09681268C988642000FB03
:101FF8000122C9F81020019B6BB1594A1268127965
:102008004AB10FF03DFB032289F820204FF47A7281
:10201800C9F81C20D1E7002D40F0AD80514AD9F80D
:10202800101010684C4A88420AD902920FF028FB17
:10203800029A032182F8201040F6B831D161BCE73A
:10204800012182F82010B8E7019B4FF4806013B19A
:1020580009F088F801E009F075F80022C9F81020A5
:1020680089E0002D46D10FF00BFBA6E725B105222C
:1020780089F82020012000E0284666B1D4F8AC2079
:10208800D189394A11805180918035490968498838
:10209800D1804FF0020B334A1168D9F814209142CD
:1020A80001D8002E64D147F23052C9F81C2003220F
:1020B80021E03A7842F002023A700EF035FB294AE4
:1020C800D9F81C1012680A44C9F81820042212E032
:1020D800244A9DB11168D9F8182091424BD9234A56
:1020E80012781AB9DAF80020D10744D43A7822F0E5
:1020F80002023A70052289F820205EE71268D9F8B2
:102108001C100A44C9F8182035E01549154A096811
:102118001268C988642000FB0122C9F810204FF416
:102128008060002289F8202089F8032009F00AF845
:1021380043E700BF380E0020A81A0020B81A002074
:10214800D10E00200000C8426C10002000C07F445F
:10215800F52B0020404B4C00782B00201410002059
:10216800CC2B0020E8270020982A0020020000201D
:1021780000287FF422AFBBF1000F02D0584607F0C9
:10218800B1FB904D05F5C470B5F84E1107F0C9F9CB
:10219800834668B90FF066FA8B4BC3F800B0C3F8F2
:1021A80004B0C3F808B0894B00221A605A609A60DC
:1021B8003B785A0736D5D8F80030DB0632D5844B41
:1021C8001B78DE062ED4834B1B7893B195F8E0314B
:1021D800BBF1000F15D17BB17F4B1A68D4F8B4302E
:1021E8009B1A002B08DA0EF09FFA7C4B83F8B8B0E4
:1021F80018E0BBF1000F0DD1102007F073FB01238D
:102208000EE03BB1744A12684FF47A7101FB032364
:10221800C4F8B43094F8B83023B107F04BFB00236E
:1022280084F8B830002295F8DEA195F8DF11B5F8EA
:1022380098E1B5F89AC11346694E019636F912002D
:102248009B087045C4BF63F07F03DBB20132604571
:10225800B8BF43F04003042AEED194F8B9205F4890
:102268009A4205D190F8BA20F92A04D8013200E040
:10227800002280F8BA2084F8B930564B594E1A78A3
:102288009946E2B93368D80708D5BBF1000F16D1D3
:102298003B78D90713D50EF0B9F810E03B785A0708
:1022A8000DD54E4B93F82B304BB14F4BDB7833B9F0
:1022B80011B10EF039FA02E0BBF1000FF9D094F831
:1022C800BA30464ADFF830B1142B40F0A78099F8AD
:1022D80000301AF1000A18BF4FF0010A6BB392F8E8
:1022E800B9305F2B11D13B7803F0040303F0FF01F1
:1022F80013B10EF019FA08E00B200391029207F0CF
:10230800F1FA029A039982F8BA10BAF1000F14D0C0
:1023180094F8B9307D2B10D13B7803F0040303F017
:10232800FF0213B10EF000FA07E00B20029207F04B
:10233800D9FA2A4B029A83F8BA203B7803F00403AF
:1023480003F0FF01002B69D194F8B930234A572BC9
:1023580011D1264B4FF47A721A80D8F800301B0638
:1023680001D50AF015FA224B1B6813F0080355D162
:10237800204A138052E0D8F80000400717D55A2B9E
:1023880015D192F8BB302BB1012382F8BB1082F82B
:10239800BC3043E092F8BD3083F0010382F8BD30D1
:1023A8000BB10C2000E00D2007F09CFA36E05D2B05
:1023B80000F01F855B2B00F01E855E2B1ED10320CD
:1023C80000F01ABDEC100020641B0020E01B002068
:1023D800D418002002000020E8270020380E002032
:1023E800982A002014100020782B0020EC2B0020C5
:1023F800D0180020E010002050100020562B01D1EA
:1024080009F050F999F80030002B00F00A8594F88B
:10241800B9306F2B40F0FF840DF0F8FFD8F800308A
:10242800580736D594F8BD30B84A93B13B78590768
:102438000FD5019BB3F90610B5F89831994208DD1C
:10244800336813F0010302BF3221A2F8C01082F8EA
:10245800BD303368DA030DD594F8C220AB4B2AB9E6
:1024680093F8BB2012B93222A3F8C020012384F8C4
:10247800C2300EE094F8BB30A44A53B13B7803F065
:10248800040303F0FF0123B9012382F8BB1082F88B
:10249800BC30DBF800A0002333600AF17B090AF1A5
:1024A800CB0B99F8002099F8013019F8010C9A42E1
:1024B8000BD2494606F0FEFF38B119F8022C012369
:1024C80003FA02F233681343336009F10409D9456A
:1024D800E7D18F4B1B7853B18E4B8F4E1A68DFF8BC
:1024E80050A212F0020F994640F03A8331E30AF104
:1024F800CA060AF589793278737816F8010C9A4277
:1025080025D2314606F0D6FF08B3B37896F804E032
:10251800824A96F803A07D480C21013B01FB0E413D
:1025280003EB43031344D1F8C8209A420FD0C1F8F3
:10253800C830002390F8F420C1F8CC30012303FA06
:102548000EF322EA030381F8C4A080F8F4300636BB
:102558004E45D0D1724B1E68724B1B68039394F89A
:102568002B300493704B029300230193029B1B684A
:10257800002B00F0E38293F800A0BAF1000F00F0FE
:10258800DD82029A039952688A1A002A0CDB01F547
:10259800FA7202994A60019901228A4094F8F4106B
:1025A80021EA020284F8F420049A002A00F0C68284
:1025B800029A597812F8042C0432D2B2002940F059
:1025C8007C825A4931F91210B5F8962102F1C800F7
:1025D800814202DD93F802B015E0C83A914203DA6D
:1025E8009978C1F1000B0EE0019A0123934094F809
:1025F800F42022EA030384F8F430039B029A03F5DB
:10260800FA7353609AE294F8F430019A1341DB07A5
:1026180000F19482BBF1000FCCBF0220012007F02B
:1026280087F90AF1FF33DFF8E490132B00F27E827A
:10263800DFE813F01400250037004B006400860023
:10264800E9004C01B301E10111027C024B005A0080
:102658008600E9004C01BB001E01830196F800903A
:10266800D944B9F1FA0FA8BF4FF0FA0929EAE97974
:10267800304686F8009006F003FF01200FE096F838
:102688000190D944B9F1640FA8BF4FF0640929EA51
:10269800E979304686F8019006F0F2FE02204946B4
:1026A800D6E196F803A0DA44BAF1640FA8BF4FF058
:1026B800640A2AEAEA7A86F803A03046D9F8F810BC
:1026C80006F094FE03205146C2E171795944642909
:1026D800A8BF642121EAE17171710D2006F052FF53
:1026E800BAF10D0F00F02282317959446429A8BF4C
:1026F800642121EAE17131710E20A9E1B1795944CF
:1027080081F30801B1710520A2E100BF380E002055
:10271800F92B002014100020D0180020305C01088C
:1027280070100020E8270020000F0020982A0020C1
:102738009819002000007A440000C84200000000F8
:10274800D9F8FC301A78022A20D107EE90BAB8EEF0
:10275800E70A5FED077A93ED097A80EE270A30EEF3
:10276800070AB5EEC00AF1EE10FA07D4B4EE670A0C
:10277800F1EE10FAC8BFB0EE670A01E01FED110ACA
:1027880083ED090A0F2006F0E7FE0AE0997859441C
:10279800C829A8BFC82121EAE17199700F2006F065
:1027A800F1FEBAF10F0F00F0C181D9F8FC301A78A8
:1027B800022A1ED107EE90BAB8EEE78A5FED227AB8
:1027C80093ED080A88EE278A38EE000AB5EEC00AAB
:1027D800F1EE10FA07D4B4EE670AF1EE10FAC8BFAA
:1027E800B0EE670A01E01FED2B0A83ED080A1220FC
:1027F80056E159785944C829A8BFC82121EAE1718E
:102808005970122024E1D9F8FC301A78022A20D114
:1028180007EE90BAB8EEE70A5FED397A93ED0C7AD5
:1028280080EE270A30EE070AB5EEC00AF1EE10FA7C
:1028380007D4B4EE670AF1EE10FAC8BFB0EE670A23
:1028480001E01FED420A83ED0C0A102006F084FE19
:102858000AE0197B5944C829A8BFC82121EAE171B7
:102868001973102006F08EFEBAF1100F00F05E8189
:10287800D9F8FC301A78022A1ED107EE90BAB8EEC1
:10288800E78A5FED537A93ED0B0A88EE278A38EED4
:10289800000AB5EEC00AF1EE10FA07D4B4EE670AE2
:1028A800F1EE10FAC8BFB0EE670A01E01FED5D0A4D
:1028B80083ED0B0A1320F3E0D97A5944C829A8BF3D
:1028C800C82121EAE171D9721320C1E0D9F8FC309E
:1028D8001A78022A22D107EE90BA1FED6A0AF8EE9A
:1028E800E77A87EE800AD3ED0F7A30EE270AB5EE45
:1028F800C00AF1EE10FA09D45FED717AB4EE670AF6
:10290800F1EE10FAC8BFB0EE670A01E01FED750AD4
:1029180083ED0F0A112006F01FFE0AE0997D594445
:10292800C829A8BFC82121EAE1719975112006F0CC
:1029380029FEBAF1110F00F0F980D9F8FC301A78A5
:10294800022A20D107EE90BA1FED860AB8EEE78A70
:1029580088EE008A93ED0E0A38EE000AB5EEC00A3A
:10296800F1EE10FA09D45FED8C7AB4EE670AF1EE55
:1029780010FAC8BFB0EE670A01E01FED900A83EDB8
:102988000E0A14208CE0597D5944C829A8BFC821D3
:1029980021EAE171597514205AE0D9F8FC301A7807
:1029A800022A1ED107EE90BAB8EEE78A5FED9E7A4A
:1029B80093ED0A0A88EE278A38EE000AB5EEC00AB7
:1029C800F1EE10FA07D4B4EE670AF1EE10FAC8BFB8
:1029D800B0EE670A01E01FEDA70A83ED0A0A092095
:1029E8005EE0D9785944C829A8BFC82121EAE17115
:1029F800D97009202CE0D9F8FC301A78022A1ED1A7
:102A080007EE90BAB8EEE78A5FEDB57A93ED0D0A56
:102A180088EE278A38EE000AB5EEC00AF1EE10FA01
:102A280007D4B4EE670AF1EE10FAC8BFB0EE670A31
:102A380001E01FEDBE0A83ED0D0A0A2030E0597B44
:102A48005944C829A8BFC82121EAE17159730A204D
:102A580006F098FD6AE0D9F8FC301A78022A22D1EB
:102A680007EE90BA1FEDCD0AB8EEE78A88EE008A25
:102A780093ED100A38EE000AB5EEC00AF1EE10FA2E
:102A880009D45FEDD37AB4EE670AF1EE10FAC8BF45
:102A9800B0EE670A01E01FEDD70A83ED100A0B209C
:102AA80006F05AFD42E0D97D5944C829A8BFC8217B
:102AB80021EAE171D9750B20CAE7012936D1987846
:102AC800B84B33F91230B3F5617F05DB40F63302BA
:102AD8009342A8BF134601E04FF46173BAF10C0F9B
:102AE80024D14FF4966292FBF0F0AF4AA3F56173DC
:102AF80093FBF0F35FFA83F913784B4516D0B9F1DD
:102B0800040F34BF4B4602231370A84A0AFB035331
:102B180003F2A673136008F001FC5046494606F01C
:102B280031FD09F10100C0B206F002FF019A01234C
:102B3800934094F8F420134384F8F430019B013354
:102B48000193029B0C330293019B042B7FF40EAD7F
:102B5800C2E4D8F80030D80510D5954BDB786BB1B6
:102B6800336899070AD5BAF8003013F0010B0AD177
:102B78000EF078FD012008F0F5FA04E0012008F0D5
:102B8800E1FA012300E00023D9F8002052070DD50F
:102B980063B1012008F0D6FABAF800309B0708D4D0
:102BA8000EF060FD022008F0DDFA02E0022008F0D5
:102BB800C9FABAF800307F4A13F0030F4FF488417E
:102BC80014BF91611185326812F00A0F27D0D9F825
:102BD8000020D00609D559070AD4042008F0C2FA03
:102BE800754B1B88A4F8003102E0042008F0AAFA0B
:102BF800D9F800309A0607D5BAF800305B0606D433
:102C0800402008F0AFFA02E0402008F09BFAD9F81B
:102C18000030580642BF684B1B88A4F8023133685D
:102C2800990609D4D9F800301A0540F191804FF47B
:102C3800807008F097FA8FE0604B1B789B0753D59C
:102C48005F4B1B78042B4FD9D9F8003013F4007B65
:102C58000FD0BAF80030DE063AD4102008F082FA15
:102C6800202008F06FFA5748011D09F0E5FC0223FF
:102C78002AE0BAF8006006F01006B6B22EB11020AD
:102C880008F060FA012684F804B1D9F80030580534
:102C980012D5D4F808314C495A89B1F90030002BC3
:102CA800B8BF5B42934207DAB1F90230002BB8BFD4
:102CB8005B429342C0F2F880BAF80030990608D512
:102CC800202008F03FFA002384F80431012600E0B0
:102CD800002694F80C31BBB90E2006F003FE3B4BDE
:102CE800012283F80C210FE0BAF8003003F030031A
:102CF800002B97D0102008F025FA202008F022FA9F
:102D0800002384F8043101E0002E8BD0304B0020E2
:102D180003F1280603F150042E4A002122F810106E
:102D28002D4A596022F810100432716022F81010F0
:102D380000221A609A603260B26022606160A2600C
:102D480014331436143400287FF46CAF0120E3E701
:102D58004FF4807008F0F6F96B79082B01D00E2B30
:102D680002D1402008F0EEF9D8F800305A0540F1B9
:102D7800B18095F80C321BB93B7813F0040F03E0CF
:102D8800D9F8003013F4002F2AD0144B00221A70FF
:102D98003C2003F023FA002800F09C800CF010FA85
:102DA800F6E700BF982A0020702700207010002046
:102DB800782B002000100048E0100020D4180020D4
:102DC800DA18002078100020E4100020380E0020C7
:102DD800480F0020EE2B0020C00F00204D1A0020C5
:102DE8000EF04CF909B0BDEC028BBDE8F04F03F0D2
:102DF800F6B8012000E002205FFA80F909F1FF33FC
:102E080085F8A43708F0F0F908F0ACFA484606F05F
:102E18008FFDFFF703BBBAF1000F02D07E2B3FF402
:102E2800FBAA94F8B930972B06D12D4B4FF4C872F2
:102E3800A3F8BE20FFF7F2BAA72B06D1294A1378C8
:102E480043F004031370FFF7E9BA0022BB2B079283
:102E580001D1022303E0B72B04D14FF6FE73ADF87E
:102E68001E300AE0BE2B01D1022304E0BD2B7FF403
:102E7800D5AA4FF6FE73ADF81C30DBF80030BDF86C
:102E88001C10B3F858200A44A3F85820BDF81E10A7
:102E9800B3F85A200A44A3F85A2008F003FC002388
:102EA80084F8BA30FFF7BABABAF800309B063FF593
:102EB80010AF202008F056F90B480C4B011D1A687A
:102EC8005B684360026009F0B7FB054B012683F895
:102ED8000461FEE609B0BDEC028BBDE8F08F00BFCF
:102EE800380E0020D418002080100020DC180020A4
:102EF8002DE9F04FC14BB3F90610C14B2DED028BF4
:102F08001F687A8989B0914201930EDBB1F5FA6F97
:102F1800FC79BDBF8B1A6343A2F5FA64C4F164045B
:102F2800BCBF93FBF4F4643400E06424B54AB64BA8
:102F3800B2F896A192F95E211868049092B20592AF
:102F4800054600220293AD4B33F912300393CAEBC6
:102F5800030303F2F31640F2E63086424FEA420BCF
:102F680003D8002BB8BF5B4201E04FF4FA73022A82
:102F7800049E4FF064002FD096F811E1BEF1000FC7
:102F880004D07345CCBFCEEB03030023DFF8C0E2C7
:102F980093FBF0FC6FF063093EF81C809B4E09FB25
:102FA8000C390CF1010C3EF91CE00FFA88FCCCEB53
:102FB8000E0E0EFB09FE9EFBF0FEC64426F80BE043
:102FC800BE1836797343924E93FBF6F364339BB283
:102FD800634393FBF0F02EE096F812E1BEF1000F88
:102FE80004D07345CCBFCEEB03030023DFF84C823B
:102FF80093FBF0F06FF0630C0CFB003938F910E02C
:103008000130002B38F91000CEEB000000FB09F965
:10301800BDF8140099FBFCF9CEEB090919FB00F97E
:103028007A48A0F80490B879B8BF5B42434378481F
:1030380093FBF0F064306B78764E4FF0640E4343A8
:1030480093FBFEF3B354744EEB7A434393FBFEF3C6
:10305800B3546B7D6D4E5843704B90FBFEF0022AC3
:1030680098546F4B0FD183F802E0039B53450EDB56
:10307800644CB4F89821914215DBB1F5FA6FA8BFFA
:103088004FF4FA6110E09C54039B534504DA36F878
:103098000B305B4226F80B300132032A05F101059B
:1030A8007FF451AFE4E71146891A4FF47A73DFF8D9
:1030B800A4E1564D59436FF063036427C2F5FA62E1
:1030C800B1FBF2F191FBF7F23EF8120003FB02119B
:1030D800013203B23EF91220D21A514391FBF7F3A1
:1030E8000344F3804F4B1B885F0635D54E4B4F4A40
:1030F8001B881288DFED4E7A9B1A1BB208EE103A35
:10310800B8EEC88A28EE278AB0EE480A08F012F806
:10311800F0EE408AB0EE480A07F0ACFFB5F902308D
:1031280006EE903AB5F90030F8EEE66A07EE903A06
:1031380020EE667AF8EEE77AA7EEA87A67EE807A4C
:10314800BDEEC77AE6EEA87A17EE103AFDEEE77AFA
:103158002B8017EE903A6B80364D2B68980740F11C
:10316800A180354B354F1A687B6945F20721D31A80
:103178008B4240F397807A6103F0F4FC304BDFF820
:10318800D8901A78032A9846B9F8003022D10A2B29
:103198002AD90023282088F8003006F02EFA03F0F8
:1031A800E1FC284B18880DF0DDFC274B1A68D37812
:1031B80090FBF3F001300828244BA8BF08201870B2
:1031C800537980B213FB00F33B83137913FB00F0B0
:1031D800788309E00A2B07D803231C4A88F80030B3
:1031E800002313703B837B8398F80030144A012B2B
:1031F8003DD033D3022B4CD054E000BF982A002096
:1032080070100020EC10002050100020E410002066
:103218000CFEFFFFC81B0020D60F0020D01B00208B
:10322800501B002098190020E01000203A0F0020C1
:1032380035FA8E3CC4270020D42B0020C80F00206C
:1032480020190020C01A0020BC180020000100200E
:103258002A1C0020121C0020C01800203A8BB9F844
:1032680000309A421EDD012388F800300FE0B9F8DB
:1032780000107B8B8B4202DD022313700FE09F4B03
:103288001B8B0133994202DD002313700AE00820EA
:1032980006E07B8BB9F8002001339A42E3DC072073
:1032A80006F020FB2D68290577D5954B934F1A68B2
:1032B800FB69C3EB020845F2072398456DDD914B86
:1032C800B6F906B0D3F80090FA6199F80A30B4F864
:1032D8004E118D4E012B4FF47A70ABF57A7B98FB2B
:1032E800F0F803D042D3022B20D041E0874B396A53
:1032F8005A7B874B33F812204FF0080E92B291FB9D
:10330800FEF3C91A8B18BA843B6240F6E44293FB79
:10331800FEF39BB25343B9F80820C2EB133358436A
:10332800B9F9063090FBF3F0306021E0794BB9F839
:1033380008A01B78C6F800A05A0719D5764806F0E9
:10334800F0F820B915F0100F18BF4FF0000B32221B
:103358000BFB0BF393FBF2F3B9F906205B445A43DA
:103368004FF47A7392FBF3F3534400E00023336085
:10337800D7E90A013368694A03FB08F84FF47A73FE
:1033880098FBF3F810EB080041EBE8710023C7E95C
:103398000A010EF0B5FB624B1860624E3368DB041D
:1033A80027D52F0622D5604B1B789D071ED55F4B6E
:1033B800187804281AD900225D4BD7180521951CC6
:1033C8004FF00A0E122AD154E9B287F801E004D06E
:1033D800B0EB510F2A46EFD800E014215A183220DA
:1033E80002F8010CFF225A540F2000E00A2006F0D0
:1033F80079FA504D2A68002A50D04F4B4F4F186821
:1034080039688142984649D84D4BDFF84091197880
:103418005268E1B94FF0010A83F800A0B9F800300A
:10342800D35C23B3504606F03FFA464B83F800A01E
:103438000DF010FCB9F80030CBB92B681B78053BB0
:10344800534514D806F0B2F83F4B18600FE04FF020
:10345800000A83F800A0B9F80030D35C3BB15046AD
:1034680006F022FA374B83F800A00DF0F3FB2A6828
:10347800B9F8003052683548D25CFE2A01D10023E1
:103488000BE0FF2A02D106F015FA07E0D8F8005041
:103498000A2111FB02523A60013303801D4D2B783B
:1034A800580704D52A4B4FF488529A6166E032686F
:1034B800D1075CBF43F001032B701B4B1B781B0724
:1034C8005EBF2B7823F001032B70D70242BF2B7805
:1034D80023F001032B701F4B1A881A4B1AB11E4A8E
:1034E8001268960702D41D4A1288CAB302221A70BB
:1034F8002B7823F001032B7037E000BFC80F0020A2
:10350800D42B0020BC180020C8180020A81A0020BE
:10351800B81A0020F52B002074120020407E050008
:10352800CC18002014100020D4180020DA1800202D
:103538009C270020BC1C0020E8270020B41C002089
:10354800B01C00209C2B002094290020B81C0020CF
:1035580000100048F60E0020D0180020EC2B0020A8
:103568002978C80758BF02221A7006F01FF8B04B16
:103578001B68C01A002801DB0DF06CFBAD4F0DF085
:103588007DFD3E780397002E00F0A580AA4B1A68AF
:103598009846002A00F01287D8F8000006F03BFA97
:1035A800002800F00B87A44BA44C186806F030FAEA
:1035B800092801D03F284CD14FF0000A2668A04FB7
:1035C80055462EB19F483968324611F01FFA10B996
:1035D800BA4605B93D469C4B10379F42F1D3D5B149
:1035E8002F68DAF80090236817F803E019F8030049
:1035F800704510D15A1C934948B92D2B07D88F4FC5
:103608004FF0200E01F803E03A60885403E001F817
:1036180003E02260E7E723680BB1554510D08B48DB
:103628000BF0C8FE554507D855F8100B0BF0C2FE35
:1036380009200BF0B7FEF5E785480BF0BBFE002626
:1036480023689E42A8D27F4B985D0BF0ABFE0136F3
:10365800F6E72368002B40F09586042840F0D386CF
:10366800784809F051FE00F0A9BED8F80000DFF84C
:10367800F0A106F0D0F920B3DAF8000006F0C8F996
:10368800DBF8003093F848100746A1BB24286CD11A
:10369800012283F84820DBF800306E4F93F8482069
:1036A800062AE2D193F8490000F03AFF8346002841
:1036B80000F083800BF0D2FDD9F80030002283F8A7
:1036C8004820654B93F83530002B40F049864C363E
:1036D800982E00F07386614BF21892F84A1001296F
:1036E800F5D1DFF87091F358C9F800205C4ACB4651
:1036F80013609046B9E7012904D14D2814BF002270
:103708000222C6E7022904D13C2814BF0022032262
:10371800BFE703290CD140284FF0000102D983F8F4
:103728004810B8E758711971D97198710422B0E737
:10373800042907D1997983F8490080EA01029A712E
:103748000522A6E70529A6D15879197988429879DA
:1037580006D978409871481C18710B441F729AE773
:10376800B8420CBF0622002293E72B783D495B073D
:1037780091D42328DAF8003012D1039A0491012059
:1037880010702D4803603448036337480BF012FE6D
:103798002F480BF00FFE04990B7843F002030B70CF
:1037A800324B1B681B78BB4201BF314B314A1A6050
:1037B800314B04BF314ADA606DE73A6892F8493014
:1037C8004E2B00F0918400F28D80332B00F0B784EB
:1037D80021D8292B00F0558409D8252B00F02C84FA
:1037E800272B00F03084232B40F0098620E22D2B74
:1037F80000F0588407D82B2B40F001860BF000FD11
:10380800607100F0A8BD2F2B00F00685312B00F069
:10381800188500F0F4BD3E2B00F0E58043D8372B27
:1038280000F0C1842CD8352B00F03D8200F0E7BDB4
:10383800A02B0020F92B00208C270020EC2400204E
:1038480078640108BC24002038660108A37B0108BD
:10385800A87B010878190020C80F0020AC190020A7
:103868007C190020F52B0020D87B0108501A002075
:10387800FC9F0020EFBEADDE00ED00E00400FA057D
:10388800392B00F0ED833C2B40F0B985E14FD7F898
:1038980000A00BF0B5FC8AF800003B68187806F029
:1038A800F6FA00F058BD432B00F05A8406D8412B95
:1038B80040F0A5854FF0000800F046BC442B00F00E
:1038C800F5844C2B40F09B850BF09AFC84F8D601CC
:1038D8000BF096FC84F8D7010BF09CFCA4F8D801F7
:1038E80000F039BDD12B00F06B8319D8CC2B00F038
:1038F800018208D8C92B00F02B83CA2B7DD0C82B96
:1039080040F07D8552E0CE2B00F01583C0F00A838D
:10391800CF2B00F04082D02B00F0F98200F06FBD71
:10392800D82B00F005810BD8D32B39D025D3D42B35
:1039380000F07582D62B40F062854FF0000863E2F4
:10394800F22B00F0B98210D8EF2B40F05885B14F18
:10395800D7F800A00BF05EFCAAF85A003F680BF0FD
:1039680059FCA7F8580000F0F6BCF32B00F0A3842C
:10397800FA2B00F0E98200F042BD2B7803F0040333
:1039880003F0FF08002B40F0E6840BF039FC022816
:1039980084F8A40740F2C1829F4B83F8A487BCE255
:1039A8000BF038FC9D4B188000F0D5BC92F80580D0
:1039B8004FEA5808B8F1120F03D902F00BFC00F0D7
:1039C800CABC4FF0000AC24507D20BF023FC944B47
:1039D80023F81A000AF1010AF5E7924B012283F84D
:1039E800342000F0B8BC0BF00BFC84F8E0010BF0BD
:1039F80007FC84F8DF0100F0AEBC864B1A68127829
:103A0800022A4FF0000A984673D1D8F800700BF0DC
:103A1800F7FB07EE900AF8EE677AB2EE048AC7EE73
:103A2800887A07EB8A0BD8F80070CBED087A0BF090
:103A3800E7FB07EE900A9FED7C7AF8EE677A07EBD2
:103A48008A0BC7EE877AD8F80070CBED0B7A0BF0AB
:103A5800D7FB07EE900A9FED757AF8EE677A07EBC9
:103A68008A0BC7EE877A0AF1010ABAF1030FCBED88
:103A78000E7ACAD1BAF1070FD8F800701CD10BF032
:103A8800BFFB07EE900AF8EE677AC7EE887AC7EDB3
:103A9800117AD8F800700BF0B3FB07EE900AF8EE35
:103AA800677AC7EE887AC7ED127AD8F800700BF0FB
:103AB800A7FB87F84C0015E00BF0A2FB07EB0A0BFD
:103AC8008BF80100D8F800700BF09AFB07EB0A0B93
:103AD800D8F800708BF80B000BF092FB07EB0A0B81
:103AE8008BF815000AF1010ABAF10A0FC2D100F0E9
:103AF80032BCD8F800700BF083FB07EB0A0B8BF88D
:103B08000100D8F800700BF07BFB07EB0A0BD8F824
:103B180000708BF80B000BF073FB07EB0A0B0AF134
:103B2800010ABAF10A0F8BF81500E2D100F013BCB4
:103B38008246384F9FED3D8AD7F800B00BF06AFBFC
:103B480007EE900AF8EE677A0BEB8A0BC7EE887AD5
:103B5800B846CBED087AD7F800B00BF05BFB07EE60
:103B6800900AF8EE677A0BEB8A0BC7EE887ACBEDF2
:103B78000B7AD7F800B00BF04DFB07EE900AF8EE81
:103B8800677A0BEB8A0BC7EE887A0AF1010ABAF159
:103B9800030FCBED0E7ACCD1BAF1070FD8F800702D
:103BA8001CD10BF037FB07EE900AF8EE677AC7EEE8
:103BB800887AC7ED117AD8F800700BF02BFB07EE66
:103BC800900AF8EE677AC7EE887AC7ED127AD8F8C5
:103BD80000700BF01FFB87F84C0015E00BF01AFB88
:103BE80007EB0A0B8BF80100D8F800700BF012FBFA
:103BF80007EB0A0BD8F800708BF80B000BF00AFBE8
:103C080007EB0A0B8BF815000AF1010ABAF10A0F43
:103C1800C2D1A0E350100020EC100020380F002083
:103C2800982A0020C80F00200000C84200007A44EB
:103C38000BF0E6FA132883463FF6BFAEDFF834A34D
:103C4800DAF800700BF0DCFA0023C54A0C2101FBFE
:103C58000322117A814222D10FFA8BFB07EB8B08E2
:103C6800137888F879300BF0CBFA88F87A000BF0E3
:103C7800C7FA88F87B000BF0C3FABA4BBA4A1A6045
:103C880088F87C00B94BDAF8000018600021793018
:103C980005F036FCB64B80F0010018705BE3013389
:103CA8001C2BD2D189E60BF0ABFA0B2882463FF6E3
:103CB80084AEB04B1F680BF0A3FA03283FF67DAE25
:103CC800062303FB0A7888F8CE000BF099FA88F8E7
:103CD800C9000BF095FA88F8CA000BF091FA88F839
:103CE800CB000BF08DFA88F8CC000BF089FA88F835
:103CF800CD0030E35379092B7FF65FAE019BD3F8F3
:103D080000800BF07DFA019B88F80000D3F8008052
:103D18000BF076FA88F801000BF072FA019B642820
:103D28001B68A8BF642018710BF06AFA019B64280D
:103D38001B68A8BF642058710BF062FA019BFF282A
:103D48001B68A8BFFF2098710BF05AFA019B6428E2
:103D5800D3F8008028BF642088F807000BF050FAD9
:103D6800019B88F80200D3F800800BF049FA019B08
:103D780088F80300D3F800800BF04CFA3B68A8F8E9
:103D88000A005B790A2B40F2E6827B4B1F680BF036
:103D980037FA3872DFE20BF03DFA6FF4AF6E00EBE2
:103DA8000E039BB2C62B98BFA4F896010BF032FA0B
:103DB800A4F840010BF02EFAA4F842010BF02AFAFD
:103DC800A4F844010BF026FAA4F8D8010BF018FA6D
:103DD80084F8ED010BF014FA0BF012FA84F8EE01F6
:103DE8000BF00EFA84F885010BF00AFA84F89201B8
:103DF8000BF006FA5F4B1F680BF00CFA00EB800023
:103E08004000A7F856002BE10BF004FA5B4B23F8AF
:103E1800180008F10108B8F1080FF5D19BE25379B1
:103E28000F2B7FF4CAAD0BF0EBF9072880463FF65D
:103E3800C4AD029B1F680BF0EDF90E2303FB08F8D5
:103E480007EB080A029BAAF819011F680BF0E2F9B0
:103E580007EB080A029BAAF81B011F680BF0DAF9A6
:103E680007EB080A029BAAF81D011F680BF0C8F9A6
:103E780007EB080A029B8AF81F011F680BF0C0F9BC
:103E880007EB080A029B8AF820011F680BF0B8F9B3
:103E980007EB080A029B8AF821011F680BF0B0F9AA
:103EA80007EB080A029B8AF822011F680BF0BCF98D
:103EB800B844C8F823014EE20BF0A2F90F28804657
:103EC8003FF67BADC8EBC8080BF09AF904EB080382
:103ED80003F1D00883F8D0000BF092F988F80100BC
:103EE8000BF08EF988F802000BF08AF988F80300C5
:103EF8000BF086F988F804000BF082F988F80500C1
:103F08000BF07EF988F8060005F034FF23E22B78E1
:103F18005F0700F120820BF053FC07F065F907F00A
:103F280021FA18E22B78580700F11582144B4FF448
:103F3800C8721A800FE22B78590700F10C82114AD7
:103F4800137843F0040339E02B785A07E5D556E295
:103F58000BF056F90B4B1A78B0B142F0020215E09B
:103F68009C5C0108300F00202C120020340F002028
:103F7800020000205010002070100020722700203E
:103F8800F60E0020D418002022F002021A700BF05E
:103F980037F9D94BD94F18700BF046F938600BF048
:103FA80043F978600BF036F9D54B18800BF032F9ED
:103FB800D44BD54A1880137843F002031370CAE132
:103FC8000BF01EF980460BF02FF983460BF02CF905
:103FD80082460BF029F907460BF01CF90BF01AF989
:103FE8000BF00EF9B8F1000F12D1C84B1020C3F82E
:103FF80000B0C3F804A007F0A5F8C54A137843F049
:1040080001031370002F00F0A681C24B1F60A2E1CC
:10401800B8F1100F40F09F81BF4BC3F800B0C3F850
:1040280004A00FB1BB4B1F60BB48BC4B0222011D53
:104038001A7008F001FB8EE1A0600BF0F5F8A36898
:104048001843A06087E10BF0E5F8A4F858010BF0DD
:10405800E1F8A4F85A010BF0DDF8A4F85C017AE164
:104068000BF0CEF884F87A010BF0CAF884F87E01D8
:104078000BF0C6F884F87D010BF0C2F884F87F01D4
:1040880069E10BF0C7F8A4F880010BF0C3F8A4F8B5
:1040980082010BF0B5F884F884010BF0BBF8A4F8A2
:1040A800860158E10BF0ACF884F890010BF0B2F8F7
:1040B800A4F89A010BF0AEF8A4F896010BF0AAF850
:1040C800A4F898010BF09CF83B6884F891015B799F
:1040D800082B40F240810BF09DF8A4F89C010BF0EE
:1040E80099F8A4F89E0136E192F805800323B8FBFD
:1040F800F3F8B8F1120F3FF660AC894F8246C2451B
:1041080080F029810BF07CF887F8A0010BF082F889
:1041180040F2ED22904205DD40F6CA029042A8BF67
:10412800104601E040F2EE20A0F2EE2019220AF13A
:10413800010A90FBF2F0023787F89F01DFE70BF0E6
:104148005FF884F8920106E10BF05AF804EB0803D3
:1041580008F10108B8F1080F83F88801F4D1FAE0F2
:104168000BF04EF8C4F808B060710BF05DF8A36866
:104178001843A0600BF044F884F890010BF04AF85B
:10418800A4F858010BF046F8A4F85A010BF042F8CD
:10419800A4F85C010BF03EF8A4F880010BF03AF8A3
:1041A800A4F88201D7E053794FF0070AB3FBFAF27B
:1041B800C2EBC2029A1A12F0FF0F7FF4FEABB3FBF8
:1041C800FAFA0AF1FF3A5FFA8AFABAF1FF0F00F039
:1041D800C2800BF015F85FFA80FB4FFA8BF005F000
:1041E800BFF8804600283FF4E8AB80F800B00BF039
:1041F80011F8A8F802000BF003F888F804000AF098
:10420800FFFF88F805000AF0FBFF88F807000AF0AE
:10421800F7FF88F80600D4E7DFF8048108F1400AC0
:104228000AF0F8FFA8F89C020AF0EAFF88F89E0254
:104238000AF0E6FF08F1040888F89B02D045EFD1A0
:1042480089E00AF0DDFF1F2880463FF6B6ABD9F8B3
:1042580000305B79082B7FF4B0AB0AF0DBFF08F184
:10426800860804EB880800F03F00A8F806000AF06A
:10427800D1FFB8F80630800100F4FE501843A8F8C2
:1042880006000AF0BDFF000188F804000AF0B8FF34
:1042980098F8043000F00F00184388F804000AF07A
:1042A800AFFF88F805000AF0B7FA54E01D4B012269
:1042B80083F835204FE00AF0A3FFFF28824635D166
:1042C80000238DF81F309DF81F30052B43D89DF82B
:1042D8001F00154A9DF81F3052F8300002EBC30347
:1042E80001215B68994089B2042204F065FF9DF8BA
:1042F8001F300133DBB2E4E7DA180020DC180020B5
:10430800D8180020D6180020761000207810002039
:10431800D418002088100020801000203C0F0020B6
:10432800EC100020C80F0020607F010805283FF628
:1043380044AB00200AF0B6FF0AF090FFD8F800005E
:1043480005F060FB18B9322005F057F9F6E74FFA87
:104358008AF004F03FFF00200AF0A4FFFFF7AAB993
:104368005C4B985905F04EFB18B9322005F045F919
:10437800F6E705F0BFFC06F00DFF574B574ADA6029
:10438800FFF7A5B90C2840D00A2842D1544D55480A
:104398000BF010F82846232110F021FB08B1401B30
:1043A80020602368002B37D14D482360002130223C
:1043B80010F0DFFA039B1B78002B5ED14A4B1B6879
:1043C8009B0615D5494B4A491B688A6B9A1A002ADD
:1043D8000EDB484A1278042A0AD9474A03F51233F1
:1043E80003F5F8738B63938A9BB283F488439382B3
:1043F800424B9B68002B67D04148984764E001F026
:10440800E9FEFFF757B90C2845D13E480AF0D2FF1C
:1044180033E00D2833D1B9E75A1EA95C202901D110
:104428001346BFE72E4A23600021D154364B374D3F
:10443800D3F800A0D5F800B0294F584610F0DDFA9F
:10444800064632463846594610F0E0FA304A20B956
:10445800BB5D53445B78590703D010359542E9D3C7
:1044680006E0954204D2701CEB683844984702E095
:1044780028480AF09FFF002396E7274807E07F288F
:104488000DD1013B164A254823600021D1540AF07A
:1044980091FFFFF781B87F2804D1FFF77DB82F2B54
:1044A8003FF67AA8A0F12002D2B25E2A3FF674A89D
:1044B80013B920283FF470A85A1C2260084AD05427
:1044C8000AF070FFFFF768B809B0BDEC028BBDE8D1
:1044D800F08F00BFAC19002000ED00E00400FA05E1
:1044E800BC24002051890108D0180020D42B0020BA
:1044F800C80F0020DA18002000100048AC2B00205C
:10450800E2100020AD7B010810010020786401084A
:1045180038660108B87B0108A87B0108D47B01082C
:104528002DE9F0474D282DED028B044600F0358625
:1045380000F29480302800F0CF8651D8222800F06D
:104548006F8423D8032800F0CB8114D8012800F009
:10455800BB81022840F0FE8604200AF0A3FE432017
:104568000AF06BFE4C200AF068FE46200AF065FE51
:104578004C2000F038BE042800F0BB81052840F02C
:10458800E9861A200AF08EFE0024DBE1282800F0D4
:10459800C38515D8242800F0A685262840F0DA8699
:1045A800DC4C06200AF07EFEB4F858010AF07DFEC5
:1045B800B4F85A010AF079FEB4F85C0100F090BD35
:1045C8002C2800F0BC852E2800F05A862A2840F0B6
:1045D800C18601200AF066FECE4B587900F003BE72
:1045E8003B2800F016841AD8362800F02A860BD803
:1045F800322800F0F285342840F0AC8648200AF0D2
:1046080051FE002500F02EBC382800F072853A28AB
:1046180040F0A08604200AF045FE00F096BE42282D
:1046280000F0EE850BD83D2800F0B082402840F01D
:10463800918608200AF036FE002400F0D7BD4628EF
:1046480000F06F864B2800F09985452840F0828657
:1046580013200AF027FE002400F06DBE702800F039
:10466800ED8200F2E480692800F04A8200F2B68008
:10467800662800F0A48100F2A680642800F07B81FF
:10468800652840F06786A44C0B200AF00BFE2088B2
:104698000AF00BFE6268A14B9A420CBF2089608920
:1046A80080B20AF002FE9E4B1B68C3F3C000C3F33E
:1046B8008002800040EA4200C3F340021043C3F383
:1046C800401240EAC20003F0100318430AF0EDFD5F
:1046D800944B1A88E368247C02F0080103F44759D4
:1046E80049EA010903F4804149EA010903F4004158
:1046F80049EA010903F4803149EA010903F4003168
:1047080049EA010903F4802149EA010903F4002177
:1047180049EA010903F4801149EA010903F0007329
:1047280049EA0303DFF8189299F8009012F0010F94
:10473800C9F3800914BF4FF002084FF0000843EA9C
:10474800090312F0020F43EA080314BF4FF0040CE8
:104758004FF0000C12F0040F43EA0C0C14BF4FF09A
:10476800100E4FF0000E12F0400F14BF2027002744
:104778004CEA0E0E12F0100F14BF4FF4007600260C
:104788004EEA070712F0200F14BF4FF4806500258A
:104798003E4312F4807F14BF4FF40060002035437D
:1047A80012F4007F14BF4FF400110021284312F4C3
:1047B800806F41EA000114BF4FF08063002300209E
:1047C80019430346E7E0672800F02181682840F094
:1047D800C18510200AF066FD002488E16C2800F0ED
:1047E800A28117D86A2800F001846B2840F0B285AE
:1047F80005200AF057FD4C4B18880AF056FD4B4B24
:1048080018880AF052FD444B93F86E0000F001003E
:1048180000F0E9BC6E2800F0938100F2C281062006
:104828000AF040FD00200AF049FD00F058BC782845
:1048380000F0FA8018D8742800F035830AD8722856
:1048480000F09483732840F0858508200AF02AFD3B
:104858000124C4E3762800F0E98300F25D832F2069
:104868000AF020FD324CCCE2A42800F0058414D8CC
:104878007B2800F06C82A02840F06C850C200AF0A0
:1048880011FD2C4B18680AF019FD2B4B18680AF01B
:1048980015FD2A4B186800F059BDF12800F0008179
:1048A800FE2800F01084F02840F054851A4C0420AB
:1048B8000AF0F8FCA36CB3F85A000AF0F6FCA36CF3
:1048C800B3F8580000F00CBC03200AF0EBFC002001
:1048D8000AF0B3FC20460AF0B0FC0D2000F083BCBF
:1048E8000AF0E0FC01200AF0A8FC0A200AF0A5FC66
:1048F800C0E306200AF0D6FC53200AF09EFC4420B0
:104908000AF09BFC46200AF098FC33200AF095FC3C
:10491800E5E300BFEC100020081000200054004020
:10492800D0180020981900204E1900205019002096
:104938006B5C0108ACF7FF1FB0F7FF1FB4F7FF1F50
:10494800F52B0020AC4B185D01340AF076FC0B2CDB
:10495800F8D10024A94B185D01340AF06EFC082C2C
:10496800F8D10024A64B185D01340AF066FC072C28
:10497800F8D100F0EDBC07200AF094FCE7200AF01B
:104988005CFCA04B58790AF058FC00200AF055FC52
:10499800042000F0DBBCA3420AD29B4A9D5C0122A2
:1049A80002FA05F50D421CBF9A4010430133F2E7A5
:1049B8000AF084FC934B93F8A40700F014BC12206F
:1049C8000AF070FC914B1B88B3F5806F8CBF0825EB
:1049D800012500248E4B33F9140090FBF5F00134C7
:1049E80080B20AF062FC032CF4D18A4CA08D0AF044
:1049F8005CFCE08D0AF059FC208E0AF056FC608EB3
:104A08000AF053FCA08E0AF050FCE08E68E31020F8
:104A18000AF048FC0024804B185D01340AF00DFCB4
:104A2800102CF8D100F094BC70200AF03BFC002652
:104A3800784D0E24AB6C744323440136B3F8190146
:104A48000AF033FCAB6C2344B3F81B010AF02DFCCD
:104A5800AB6C2344B3F81D010AF027FCAB6C23446C
:104A680093F81F010AF0E9FBAB6C234493F820018B
:104A78000AF0E3FBAB6C234493F821010AF0DDFB59
:104A8800AB6C234493F822010AF0D7FBAB6C1C44AF
:104A9800D4F823010AF012FC082EC9D100F058BC42
:104AA8007020584C0AF0FEFB04F1700594F8D00011
:104AB8000AF0C3FB94F8D1000AF0BFFB94F8D200C7
:104AC8000AF0BBFB94F8D3000AF0B7FB94F8D400C3
:104AD8000AF0B3FB94F8D5000AF0AFFB073494F85A
:104AE800CF000AF0AAFBAC42E0D100F031BC4B4B3E
:104AF800185D01340AF0A1FB102CF8D100F028BC95
:104B0800474D2878400000F0FE000AF0CBFB002457
:104B18002B789C4280F01C84424B33F814000AF036
:104B2800C4FB0134F4E7404C06200AF0BBFB2088A4
:104B38000AF0BBFB60880AF0B8FB3C4B1888CFE250
:104B480007200AF0AFFB3A4B1888FF28A8BFFF20C0
:104B5800C0B20AF072FB374B186880F3100080B2BD
:104B68000AF0A3FB2B4BB3F864000AF09EFB254B1D
:104B780093F88521304B186822B10A23584380F3F3
:104B8800100001E000F30F0080B2A9E21D4C0220E2
:104B98000AF088FB94F8E0010AF04FFB94F8DF0173
:104BA80021E31C4C0B200AF07DFBA36E18780AF059
:104BB80044FBA36E58780AF040FB00262546AB6EEE
:104BC800144C3344013618790AF037FB032EF6D11A
:104BD800A36ED8790AF031FBA36E98780AF02DFB02
:104BE800A36ED8780AF029FBA36E58890AF05DFBFA
:104BF800A36E187AF7E200BFE0780108EC780108A4
:104C0800C1780108EC1000201910002004000020D1
:104C1800DA10002008100020401000205410002056
:104C2800481A0020982A0020BC270020E010002005
:104C3800C0180020CC180020C8180020C64C1E2020
:104C48000AF030FBA36C1B78022B4FF000056BD1E8
:104C5800A36C03EB850393ED080AB2EE048A20EEF9
:104C6800080A10F095F880F30800C0B20AF0E5FAD7
:104C7800A36CDFEDBA7A03EB850393ED0B0A20EE04
:104C8800270A10F085F880F30800C0B20AF0D5FAB8
:104C9800A36CDFEDB37A03EB850393ED0E0A20EEE8
:104CA800270A10F075F880F30800C0B201350AF041
:104CB800C4FA032DCCD1072DA36C23D193ED110A8F
:104CC80020EE080A10F064F880F30800C0B20AF079
:104CD800B4FAA36C93ED120A20EE080A10F058F803
:104CE80080F30800C0B20AF0A8FAA36C93F84C301D
:104CF80000EE103AB8EE400A10F04AF880F30800C7
:104D0800C0B20BE02B4458780AF097FAA36C2B44F6
:104D1800D87A0AF092FAA36C2B44587D01350AF030
:104D28008CFA0A2DC7D113E3A36C2B4458780AF0E8
:104D380084FAA36C2B44D87A0AF07FFAA36C2B442C
:104D48000135587D0AF079FA0A2DEDD100E33C20AF
:104D58000AF0A8FA0024804D9FED818AAB6C03EB22
:104D6800840393ED080A20EE080A10F011F880B2C7
:104D78000AF09BFAAB6C03EB840393ED0B0A20EE6D
:104D8800080A10F005F880B20AF08FFAAB6C03EB52
:104D9800840393ED0E0A20EE080A0FF0F9FF0134A0
:104DA80080B20AF082FA032CD5D1072CAB6C16D14D
:104DB80093ED110A20EE080A0FF0EAFF80B20AF01C
:104DC80074FAAB6C93ED120A20EE080A0FF0E0FFBC
:104DD80080B20AF06AFAAB6C93F84C000BE02344FB
:104DE80058780AF062FAAB6C2344D87A0AF05DFA74
:104DF800AB6C2344587D01340AF057FA0A2CD4D1FD
:104E0800A6E214F8010F002800F0A2820AF015FAB1
:104E1800F7E701200AF046FA4F4B9B6C1878E2E15D
:104E280050200AF03FFA00254B4B9C6C4D4B04EB8D
:104E380085040C2194F8792001FB0233013593F89D
:104E480038000AF0FAF994F87A000AF0F6F994F8BA
:104E58007B000AF0F2F994F87C000AF0EEF9142DC0
:104E6800E2D175E23C4B9C6C062303FB05440135FB
:104E780094F8CE000AF0E1F994F8C9000AF0DDF9D7
:104E880094F8CA000AF0D9F994F8CB000AF0D5F9D9
:104E980094F8CC000AF0D1F994F8CD000AF0CDF9D5
:104EA8000C2DDFD154E24FF00008012600272A4BD1
:104EB8001A7C974227DA11330024FA5C294D0C2317
:104EC80005F130016343595C914207D12B44586B7B
:104ED8000FF093FD82462EB9B14605E001341C2C33
:104EE800ECD10EE080440CE0D1450ADA0C2303FB38
:104EF80004535B6B13F809000AF09FF909F10109E3
:104F0800F2E70137D3E7002E00F022825FFA88F03B
:104F18000AF0C8F90026C9E70F4D287C0AF0C2F943
:104F280000242B7C9C4280F013820F4BE65C00210E
:104F38000C480C2200F1300702FB01F3DA5DB242A3
:104F480005D1034493F838000AF077F902E00131FB
:104F58001C29EDD10134E4E7081000200000C84204
:104F680000007A446C5C010819100020CF4C162010
:104F78000AF098F9B4F896010AF097F9B4F84001E4
:104F88000AF093F9B4F842010AF08FF9B4F8440131
:104F98000AF08BF9B4F8D8010AF087F994F8ED0112
:104FA8000AF04BF900200AF048F994F8EE010AF0EB
:104FB80044F994F885010AF040F994F892010AF04E
:104FC8003CF900200AF039F9B94B9B6C0A20B3F977
:104FD800563093FBF0F080B20AF067F98DE0E0B24A
:104FE80001340AF02AF9092CF9D1B1E110200AF0AC
:104FF80059F9B04BB04C187800F002000AF01DF9CE
:10500800AE4B18780AF019F920680AF057F9606869
:105018000AF054F9AA4B18880AF047F9A94B1888DE
:105028000AF043F9A24BB3F86C0059E00AF0E8F82B
:10503800074612200AF036F99D4C17B9266F656F9E
:1050480005E0102F13BF0025A66FE56F2E463846E2
:105058000AF0F3F830460AF031F928460AF02EF93A
:10506800D4F880000AF02AF900200AF01EF900207E
:105078000AF01BF90020B6E08D4D95F884008000F9
:105088000130C0B20AF00EF995F884000AF0D5F89C
:1050980000242E4696F884309C4280F059818A4D2F
:1050A800285D0AF0CAF805F11003185D0AF0C5F882
:1050B80005F120033035185D0AF0BFF8285D0AF0C5
:1050C800BCF80134E6E708200AF0ECF800200AF002
:1050D800ECF800200AF0E9F800200AF0E6F80020D1
:1050E8000AF0E3F834E104200AF0DCF86F4B986822
:1050F8002CE104200AF0D6F86C4C94F87A010AF0F6
:105108009CF894F87E010AF098F894F87D010AF06A
:1051180094F894F87F0166E0644C07200AF0C2F81E
:10512800B4F880010AF0C1F8B4F882010AF0BDF8B9
:1051380094F884010AF081F8B4F88601D0E75B4C52
:105148000C200AF0AFF894F890010AF076F8B4F859
:105158009A010AF0AAF8B4F896010AF0A6F8B4F889
:1051680098010AF0A2F894F891010AF066F8B4F8E8
:105178009C010AF09AF8B4F89E01B1E74B4C042060
:105188000AF090F894F8D6010AF057F894F8D70185
:105198000AF053F8B4F8D801A2E74C4C4C4D2078EB
:1051A80000EB4000C0B20AF07DF8002623789E424A
:1051B80005F1020580F0CC8015F8020C0AF03DF8E4
:1051C80015F8010C00EB800000EB800000F2EE20E7
:1051D80080B20AF06AF80136E8E701200AF062F8BE
:1051E800324B93F892010AF028F8B1E02F4B234490
:1051F800013493F888010AF020F8082CF6D1A7E0CA
:105208002A4C10200AF04EF860790AF016F8A068C7
:105218000AF054F894F890010AF00FF8B4F858011D
:105228000AF043F8B4F85A010AF03FF8B4F85C0100
:105238000AF03BF8B4F880010AF037F8B4F88201B4
:105248004EE71B4B194C93F8C500C0EBC000C0B229
:105258000AF028F804F118051E4A94F8F40192F9A6
:10526800001043B2994277D092F90C10994273D04A
:1052780092F918209A426FD00834AC42ECD167E01A
:1052880040200A4C0AF00EF804F14005B4F89C02DC
:105298000AF00BF894F89E0209F0CFFF043494F852
:1052A8009B0209F0CAFFAC42F0D151E0EC1000209B
:1052B80008100020D4180020DC180020DA1800207C
:1052C800D8180020D61800208D100020481A002079
:1052D8008C120020541A0020E0202D4C09F0E2FF27
:1052E80004F18005B4F81E0200F03F0009F0DDFF6C
:1052F800B4F81E02C0F3861009F0D7FF94F81C0218
:10530800000909F09AFF94F81C0200F00F0009F058
:1053180094FF043494F8190209F08FFFAC42E1D1EC
:1053280016E00D2009F0BEFF002009F086FF0020DE
:1053380009F0C4FF06E0174B185D013409F07DFF42
:105348000B2CF8D1002009F0B9FF002009F0B6FFB6
:10535800012018E0002016E009F06FFFB4F8F6010C
:1053680009F0A3FF94F8F80109F067FF94F8F90130
:1053780009F063FF94F8FB0109F05FFF94F8FA0164
:1053880009F05BFF78E7BDEC028BBDE8F08700BF52
:10539800EC100020E07801082DE9F047C14CC24E1E
:1053A800237886B00746002B00F0038232686368D2
:1053B800D31A7C2B40F2FD81237A62600133237279
:1053C800002505F12400DFF8DC82C0B20BF046FEB0
:1053D80008F10A0333F9153007EE903AB34B1B88EE
:1053E800B8EEE77A07EE903AF8EEE77A0135C7EEBD
:1053F800277A9FEDAF7A67EE877AFDEEE77ACDEDF3
:10540800037ABDF90C000BF017FE032DD9D130201B
:105418000BF024FE00200BF00FFE0BF017FE98F89F
:10542800085015F0030520D1D8F8042041F288333C
:105438009A420BD910200BF011FE28460BF0FCFD08
:1054480021200BF00BFE28460BF0F6FD14200BF084
:1054580005FEB4F910000BF0EFFD1C200BF0FEFD6B
:1054680000200BF0E9FD0BF0F1FD237ADFF8348220
:105478005B0740F07B8102200BF0F0FD0A23B8F9AE
:10548800120090FBF3F00BF0D7FD0320B8F91A5087
:10549800DFF830920BF0E2FD864B1B7813F0040F17
:1054A8004FF0050A95FBFAF5ADB20DD008F5D270AC
:1054B800394604F036F828B9D9F8003013F0100F3F
:1054C80018BF002528B205E0D8F8EC379889B0FB5A
:1054D800FAF000B20BF0B0FDD9F800309F0740F1A8
:1054E8008A80DFF8E491B4F8F27799F80030B4F8DC
:1054F800F0276C4D3F014FF06408BFB208FB023241
:105508005B00B2FBF3F347EA0327BFB2C3F30323FD
:105518001F4306200BF0A2FD38B20BF08DFDB4F846
:10552800F23799F8001001339BB293FBF1F201FBBB
:105538001233A4F8F237D4F8F4379B7B012B05D14A
:1055480039200BF08BFDB5F9F0071AE0B5F8F057E4
:105558006E233A205D4315270BF080FD95FBF7F588
:10556800AFB2B7FBF8F528B20BF066FD08FB15756E
:105578003B200BF073FDA8B2451D0A2095FBF0F007
:1055880000B20BF059FD28200BF068FDD4F8F8376D
:10559800444D0A2093FBF0F000B20BF04DFD0420BF
:1055A8000BF05CFDD4F8EC37D5F8FC079A894FF678
:1055B800FF739842A8BF1846C2B10028ACBF131A9F
:1055C800134607EE903A9FED3C7AF8EEE77A67EEDD
:1055D800877A07EE102AB8EEC77AC7EE877AFDEE0B
:1055E800E77A17EE900A6428A8BF642020EAE070E2
:1055F80000B20BF021FDD4F800382A4F9D0640F187
:10560800AA8097F8043898071DD511200BF026FDBD
:10561800B7F80608294B4FF4F365684390FBF3F09D
:1056280000B20BF009FD19200BF018FDB7F80608B9
:105638004543642095FBF0F595FBF0F300FB135010
:1056480000B20BF0F9FC94F80438B4F8085813F0D9
:10565800020F08BF002501200BF000FD28B20BF057
:10566800EBFC09200BF0FAFC00200BF0E5FC144BD6
:1056780094F80A581A88B2F5967F0AD9094B1B7A0A
:1056880003F00F03072B04D842F20F75954228BF89
:10569800154605200BF0E2FCD4F8F4375B7BBBB968
:1056A80028B232E0D0100020E827002004000020B3
:1056B80000007A44F52B00200000C842A0860100B3
:1056C80002010020C4270020000100206666E63F92
:1056D800A5F1200307EE903A1FED047AF8EEE77A79
:1056E800F6EE006AC7EE877ABEEE007AF5EEC07A6B
:1056F800F1EE10FA58BFB0EE667A77EE877AFDEED3
:10570800E77ACDED037ABDF90C000BF095FC94F81F
:105718000428C94B910703D493F80B28012A04D114
:10572800012384F80B38C5481CE0D3F8F437DFEDC3
:10573800C46A93ED017AD3ED027A27EE267A67EEF2
:10574800A67ABDEEC77AFDEEE77A8DED047ACDED47
:10575800057A04A806E0BB4A92E8030004AB83E894
:105768000300184602F0C6FF0BF070FC237A282BC2
:105778001FD1B14B00221A723C2733684FF47A705C
:10578800B3FBF0F817200BF069FCB8FBF7F5B5FB95
:10579800F7F007FB1050000200B20BF04DFC182088
:1057A8000BF05CFC07FB158000B20BF045FC0BF01E
:1057B8004DFC94F81438A04D002B00F0628103F0E2
:1057C800F5FED5F81838A04AC31A9342074640F2A6
:1057D800C680002385F81E3885F82038B5F8F037DC
:1057E800DAB21B0A85F83A2885F83B3885F830285C
:1057F80085F83138D5F8482833689A1AD5F84C38DE
:10580800D97B4FF47A734B439A420ED38F4B1B6864
:10581800C5F8483895F85038013B012B9FBF102335
:1058280085F81E38022385F820380A20D4F8F8278E
:1058380092FBF0F284F83828121284F8392894F888
:105848000428D4F8FC3793FBF0F384F83C381B1297
:1058580084F83D38920794F80A38774984F86B3809
:1058680003D42D2381F86C3877E0042BD4F80C98F6
:10587800D4F81068DFF8E481754A8CBF33233223EB
:1058880081F86C384FF0060C724B99FBF3F096FBDD
:10589800F3F308FB009108FB036803EB83030CFB9D
:1058A80001F103EB830391FBF2FE642502FB1E1159
:1058B8009B0091FBF5F184F85D1809120CFB08FCBC
:1058C80084F85E189CFBF2F143FA81F39BB202FB69
:1058D80011C292FBF5F284F86228121284F860383B
:1058E80084F863281B0AB4F8062884F8613824234E
:1058F800534393FBF5F5B4F87E3884F8643800EB2D
:1059080080001B0A00EB8000800084F865380A22BA
:10591800B4F80838B3FBF2F303F5FA739BB240FA14
:105928008EF080B284F866381B0A4FEAD97984F879
:105938005B08F60F000A84F8585884F86738C5F3EE
:105948000725B4F8803884F85A9884F85C0884F8F5
:105958005F6884F8595884F86D38C4F8187894F852
:105968008288354DB8F1000F0DD1D5F8880804F0BC
:1059780052F8012807D90228374E00F0568202F063
:10598800ABFE0123B370D4F88C282B4D002A78D0B5
:1059980095F882683EB1D5F8943840F6B731FB1ACD
:1059A8008B4219D86DE00123D5F8880885F882382C
:1059B80003F0A7FCD5F8983893F9000002238DE886
:1059C8004800082132464FF4964303F020FE85F83C
:1059D8009C68C5F8880852E095F89068CEB9D5F863
:1059E8008808C5F88C6885F8826803F08AFCD5F8C1
:1059F800983893F9000001238DE8480008213246C1
:105A08004FF4964303F003FEC5F8880802F064FEDD
:105A180035E0013EF6B285F8906895F89C1895F83F
:105A28009D38EEB94A1C013385F89C2885F89D38C5
:105A3800D5F8880821E000BFD0100020DC1800202D
:105A48008096184BF85D01083F0D0300E8270020F9
:105A580040420F008096980004000020806967FF8C
:105A680012F8016BC5F88C28701885F89C0801336A
:105A7800D5F8880885F89D38314603F0CFFFC4F87B
:105A8800947894F89E389C4DDBB1D5F8A038C3B112
:105A9800D5F8A438ABB1C5F8A8381B68974AC5F83B
:105AA800AC38D5F8B0381344187AFEF739FD09F048
:105AB800D5FBD5F8B0380133092B88BF0023C5F8CA
:105AC800B0388F4D94F8B4282E688B4B002A00F01C
:105AD800E781D3F8B828002A00F0E28193F8BC38AF
:105AE800013B012B00F2DC81D4F8B808824F03F0A7
:105AF80092FFE0B1D7F8B80803F08AFF97F8BD38ED
:105B0800D5F800907E2B80460ED102231B2887F8FB
:105B1800BC3809D1D7F8B80803F07DFF20B90123B4
:105B2800C7F8C09887F8C43884F8BD88DCE7D7F888
:105B3800C0282B689B1A41F6583293421ED903237A
:105B480087F8BC38ACE16F4A32F8130010B9034645
:105B58004FF403600133B0F5C06FDBB271D01ED9CA
:105B6800B0F5006F77D033D9B0F5036F40D184F822
:105B7800C538D4F80038604F9A0640D494F8C41851
:105B880094F8C538002900F04D812A68921B012A33
:105B9800D9D984F8C538002384F8C43880E1B0F531
:105BA800007F44D008D8B0F5807F00F08780B0F53A
:105BB800887F00F08380E5E7B0F5806F00F0A6806D
:105BC800B0F5826F00F0EB80B0F5047FDAD123E006
:105BD800B0F5E26F00F08280B0F5E46F00F08380EA
:105BE800B0F5E06FCED184F8C538B4F90A107EE07C
:105BF800B0F5046F6BD0B0F5026FC3D1FBE097F836
:105C080004389B07BAD5B7F8061824234B43123338
:105C1800642193FBF1F1FFE084F8C5383A4B364F25
:105C28001B689907AAD5B7F8F0370A21F3E084F87A
:105C3800C538354B304F1B681A059FD5D7F8F8176C
:105C4800EAE084F8C538304B2B4F1B681B0595D507
:105C5800D7F8FC17E0E0D4F80018274A84F8C538CC
:105C680088068BD592F80418890787D5DB0712D5E3
:105C7800D2F8103883EAE371002BA1EBE37101EB52
:105C880051014FF01902B1FBF2F1ACBF41F00041F4
:105C980041F040410FE0D2F80C3883EAE371A1EB00
:105CA800E371002B01EB51014FF01902B1FBF2F146
:105CB800B8BF41F080414FF400608BE084F8C538EC
:105CC800D4F800385F077FF559AF002160E0B4F9D8
:105CD800101084F8C538642359437BE084F8C5382C
:105CE800B4F90C1003E0B4F90E1084F8C5382C236D
:105CF80091FBF3F16EE000BFD0100020F85D0108C1
:105D0800E8270020F67C0108C427002084F8C5385D
:105D180094F8C638644A0133DBB2032B88BF0123E9
:105D280082F8C63894F8C61842F2107359435F4B8C
:105D38001B78D80748BF01319A0748BF02315F076F
:105D4800B4F8C83848BF0431D80748BF0A319A07A1
:105D580048BF14311F0648BF2831D80548BF28312D
:105D68005A0748BF64311F0748BFC831980548BF64
:105D780001F5C8719A0648BF01F57A71DF0648BF78
:105D880001F5FA61580648BF01F57A614FF4806061
:105D980002F06EFC444B002283F8C428EEE6D4F8E7
:105DA8000018DFF8048184F8C53811F0200717D0EF
:105DB80098F8042812F0020F14BF4FF47A710021EA
:105DC80012F0010F14BF4FF4FA6300230B4494F848
:105DD8000A18194402F04CFC002384F8C438CDE6B4
:105DE800334B1B6819067FF5C9AE394602F040FCF3
:105DF80088F8C478C2E684F8C538D4F800382A4F41
:105E08009A067FF5BBAE97F804389B077FF5B6AEC8
:105E1800B7F808386421594302F02AFC002387F8B0
:105E2800C438ABE684F8C5383AE0B37823B1C5F88E
:105E3800847886F80280A6E5D5F88438FB1AB3F58D
:105E48007A6FFFF4A0AD0123D5F88808B37003F08A
:105E5800DFFD0646D5F8880803F0DAFD76067FF4FC
:105E680092AD8A2802D08E280DD08CE5D5F800385E
:105E780099067FF588AD95F88238002B7FF483ADBD
:105E880005F6510306E095F88238002B7FF47BADC8
:105E980005F61C03C5F88C382D2385F8903872E573
:105EA80006B0BDE8F08700BFD0100020F52B002019
:105EB800C4270020704708B51F4A18B95368022242
:105EC8001A8208BD0020516810800B7813F07F03F8
:105ED8000DD14B7A990644BF0221117013F0400F7F
:105EE800137814BF43F0010323F0010315E0012BDD
:105EF8001FD0022B1ED14B7913F0800F03F00F0334
:105F08004FEA830303F1804303F5B8431B6806D0C7
:105F180003F03003102B07D10123137004E003F4BE
:105F28004053B3F5805FF6E793681B6998470248CA
:105F380008BD104608BD00BFA019002010B5064CCA
:105F480018B9636801221A8210BDA3689B68984734
:105F580060680C3010BD00BFA019002010B5064CB9
:105F680018B9636801221A8210BDA3681B68984794
:105F780060680A3010BD00BFA0190020084BDA681D
:105F8800D10709D4DA68D20608D4DB6813F0040F05
:105F980014BF032004207047012070470220704777
:105FA8000020024010B50446B0F9000009F08BFF4C
:105FB800B4F9020009F087FFB4F90400BDE8104005
:105FC80009F081BF10B50446006809F07CFF6068DD
:105FD80009F079FFA068BDE8104009F074BF2DE909
:105FE800F74F012003F0FCF9002488B3012C2FD8C7
:105FF800194E4FF04C0909FB04FA06EB0A0808F1A0
:106008005407BD7815B10134E4B2EEE790F90030D9
:1060180090F804E01846114B03228DE82400012172
:106028002A4653F82E3003F0F2FA834660B106F19F
:106038000C00504429464A460EF09BFC01231C44A0
:10604800C8F80CB0BB70E4B2012003F0AFF9CCE79C
:1060580003B0BDE8F08F00BFA0190020105E010852
:1060680010B5184C002120461A220EF082FCA4F527
:10607800F970142380F8F43105230022042180F8F4
:10608800F83180F8FA3180F8003280F8023280F86E
:10609800083280F80A325223012480F8F91180F876
:1060A800FB2180F8011280F8032280F8091280F899
:1060B8000B2280F8F23180F8FC2180F80442A0F825
:1060C800F64110BDDE12002010B5FFF757FF4FF460
:1060D8003024012806D11CB1FFF750FF013CF8E736
:1060E800052010BD002C08BF052010BD70B5064660
:1060F800441E14F8011F89B1094D28460EF06FFCA3
:106108000028F6D005F1080398423FBF054B401B15
:10611800C018A31B38BF80F88831EAE770BD00BFFC
:10612800167D0108EC100020031EB8BF2D2210B503
:10613800B8BF58420C46B8BF01F8012B0A2204F038
:1061480007FE00230370204610BD07B51C4B03F162
:10615800A802C3F8A4201B4A92F890215AB1012A38
:1061680014D1032183F8AA10072183F8AC2083F8FF
:10617800AB100C2208E0022183F8AA10032183F84F
:10618800AC2083F8AB10072283F8A8200E4B0F4AE7
:106198001A60402003F024F970B10122002390F91D
:1061A800000040218DE80C00094A4FF4E13303F068
:1061B8002EFA003018BF012003B05DF804FB00BFC1
:1061C800A0190020EC100020080000204508010854
:1061D800D90901080120002109F046B8F0B51C4A88
:1061E80092F8AD30D2F8B05092F8B47092F8C0601E
:1061F80092F8CCE0022B0ED805EBC304591CA31C63
:10620800C9B206D02346A48814F0010F01D0204259
:1062180005D10B46EEE782F8AD300020F0BD93F9CA
:1062280002307CB29C4201D1002307E074B29C4248
:106238000CD04FFA8EF49C42EBD1022382F8AD10B9
:106248000C2101FB0322D2F8B800F0BD0123F5E7C9
:10625800A019002030B5002202F1805303F5B8538D
:106268009B0042F400441D6840F60F7144F080041E
:10627800294001322143042A1960EDD1024B40F034
:106288008000186030BD00BF4C5C00402DE9F84329
:10629800324D6E68328A377ABAB9042F15D1304830
:1062A8000378012B0CD12F4B19682F4B89B20B4463
:1062B8005B0019681A603023A5F8D830027049E0ED
:1062C8001023A5F8D830072744E0B48AB369A2425E
:1062D80094BF04270227944228BF14461FFA84F863
:1062E800404698471F4A13689BB203F1005303F5D1
:1062F80040535B0004F1010E1B689BB203F100538D
:1063080003F540534FEA6E0E5B000021714500F122
:10631800020009D010F8019C10F802CC4CEA092CB4
:1063280023F821C00131F1E712680F4B92B21344F0
:106338005B001A681C60338AC8EB03033382738AD4
:1063480098443023A5F8D8304FF44053A6F812806B
:10635800A5F8DA306B681F72BDE8F883A019002031
:10636800F62B0020505C0040023000200E4B0F4AF4
:106378001B689BB203EBC00002443E294FEA42026D
:1063880009D94B09C80604BF03F1FF339BB29B022E
:1063980043F4004304E04B08C90748BF01339B029C
:1063A80011681360704700BF505C00400630002041
:1063B80008B50B4B002093F83010FFF7D7FF094BB7
:1063C8005A68107A082801BF4FF48052A3F8DA20DF
:1063D8001022A3F8D820A0F109035842584108BD5B
:1063E80008000020A019002038B5444D6A681078CC
:1063F80010F07F0004D1537A23F02003537238BD84
:10640800022879D15388002B77D11379002B74D1C6
:10641800537923F08000840004F1804101F5B841EC
:1064280013F0800F096814BF01F0300101F44051E6
:10643800032861D800295FD0927A002A5CD004F141
:10644800804404F5B8441906226825D502F03002C4
:10645800102A4CD103F07F039B0003F1804303F51E
:10646800B8431A68510641BF196840F60F720A40CE
:1064780042F4004244BF42F0C0021A601A6822F493
:10648800E04222F0400292B282F0300242F400422E
:1064980042F080021A602AE002F44052B2F5805FAE
:1064A80025D128B9164B93F83010FFF75FFF11E09C
:1064B8009B0003F1804303F5B8431A68520441BFB7
:1064C800196840F60F720A4042F4404244BF42F055
:1064D80080021A60236823F4804323F070039BB280
:1064E80083F4405343F4004343F080032360AB68D4
:1064F8005B699847002038BD022038BDA0190020EC
:1065080008000020002303604360836083810361E7
:1065180043618361C36103624362836270478A682F
:10652800036810B50C6A14430A6914434A69144392
:106538008A691443CA6914434A6A14438A6A23F469
:10654800FF4323F070032243134303608B894360A6
:106558000B6883604B68C36010BD02684FF6FE731A
:10656800134003600023036043608360C360294BCA
:10657800984201D1284A27E0284B984201D1264A5F
:106588002AE0274B984201D1234A2DE0254B984217
:1065980001D1214A30E0244B984201D11E4A33E010
:1065A800224B984204D11C4A536843F470032EE0EE
:1065B8001F4B984204D1184A536843F0706326E091
:1065C8001C4B984204D11C4A536843F00F031EE049
:1065D8001A4B984204D1184A536843F0F00316E066
:1065E800174B984204D1144A536843F470630EE081
:1065F800144B984204D1104A536843F4704306E0A0
:10660800114B984204D10C4A536843F470235360E9
:10661800704700BF08000240000002401C00024012
:106628003000024044000240580002406C00024022
:106638008000024008040240000402401C0402409A
:10664800300402404404024058040240036A23F024
:1066580001030362036A70B5446882690D6822F415
:10666800803222F0730215438A8923F00203134310
:106678008A881343134A90420FD002F50062904271
:106688000BD002F54062904207D002F5806290423A
:1066980003D002F5806290420DD1CA89CE8823F0DA
:1066A800080313430A8A24F4407414434A8A23F0E3
:1066B8000403334314438A68446085614263036278
:1066C80070BD00BF002C01409D4A536803F00C03C5
:1066D800042B2DE9F04105D0082B06D0994901601B
:1066E800B3B916E0974B036012E053685468C3F3DC
:1066F8008343991CE30349BFD36A934B914C03F03E
:106708000F0344BF0133B4FBF3F34B43036000E0D2
:10671800002351688D4FC1F30311394491F8345067
:106728000168EDB221FA05F444605668C6F3022602
:106738003E4496F8346024FA06FEC0F808E056682D
:10674800C6F3C2263E4496F83460F6B2F440C460FC
:10675800D2F82C80C8F3041808F00F0C07EB4C0C87
:1067680018F0100FBCF844C01FFA8CFC07D0BCF11D
:10677800000F04D0B3FBFCFCC0F810C000E00161BE
:10678800D2F82CC0CCF3442C0CF00F0807EB4807C8
:106798001CF0100FB7F84470BFB204D01FB1B3FBA0
:1067A800F7F7476100E04161176BFF065ABF654F75
:1067B80087618161176BBF065ABF624FC761C161AC
:1067C800176B7F065ABF5F4F07620162176BFF05A1
:1067D80006D5994204D1AE4202D14F00476200E08B
:1067E8004462176BFF0406D5994204D1AE4202D128
:1067F8004F00876200E08462176BBF0506D5994297
:1068080004D1AE4202D14F00C76200E0C462176BE8
:106818007F0506D5994204D1AE4202D14F004764A4
:1068280000E04464176B3F0506D5994204D1AE4297
:1068380002D14F00876400E08464176BBF0406D55B
:10684800994204D1AE4202D14B00C36400E0846493
:10685800156B3B4BAD0701D1046315E01C6B04F0CD
:106868000304012C01D101630EE01C6B04F0030446
:10687800022C02D14FF4004305E01B6B03F0030325
:10688800032B01D12F4B0363146B2D4B14F4403FA2
:1068980002D1C0F834E018E01C6B04F44034B4F5BD
:1068A800803F01D1416310E01C6B04F44034B4F51F
:1068B800003F02D14FF4004306E01B6B03F4403362
:1068C800B3F5403F01D11F4B4363146B1C4B14F4C9
:1068D800402F02D1C0F838E018E01C6B04F44024C3
:1068E800B4F5802F01D1816310E01C6B04F44024BF
:1068F800B4F5002F02D14FF4004306E01B6B03F4FC
:106908004023B3F5402F01D10E4B8363146B0C4B1E
:1069180014F4401F02D1C0F83CE021E01C6B04F4E1
:106928004014B4F5801F01D1C16319E01C6B04F455
:106938004014B4F5001F0BD14FF400430FE000BF23
:106948000010024000127A0000093D0008000020F3
:106958001B6B03F44013B3F5401F01D1134BC36302
:10696800126B134B12F4400F03D1C0F840E0BDE89E
:10697800F0811A6B02F44002B2F5800F02D1016473
:10698800BDE8F0811A6B02F44002B2F5000F02D1A3
:106998004FF4004306E01B6B03F44003B3F5400FCC
:1069A80001D1024B0364BDE8F08100BF00127A00F8
:1069B80000100240F0B500230E681C460125A540D2
:1069C80005EA060EAE452BD10F797A1E012A15D895
:1069D800856803229A4025EA020282604D7982681E
:1069E8009D4015438560828892B222EA0E02828019
:1069F8008A798588A2402A4392B282800322056858
:106A08009A40D2431540056005689F402F430760B0
:106A1800C7681740CA7902FA03F547EA0502C26057
:106A28000134102C03F10203C8D1F0BD38B52DEDA7
:106A3800048B4A4C0368C4F8DC308388A4F8E0303F
:106A4800013A0D46072A42D8DFE802F0040A101876
:106A580022292F35B4F8DC300B80B4F8DE3013E08F
:106A6800B4F8DE300B80B4F8DC3005E0B4F8DC3084
:106A78005B420B80B4F8DE305B4205E0B4F8DE30F0
:106A88005B420B80B4F8DC306B80B4F8E0301DE07A
:106A9800B4F8DC305B420B80B4F8DE3012E0B4F8B6
:106AA800DE300B80B4F8DC300CE0B4F8DC300B805E
:106AB800B4F8DE3005E0B4F8DE305B420B80B4F8A1
:106AC800DC305B426B80B4F8E0305B42AB80244B37
:106AD80093F86430002B3ED1B5F9003094ED3C0AB0
:106AE800D4ED397A09EE103AB5F9023008EE103AC9
:106AF800B8EEC88AB5F90430B8EEC99A28EE000A8B
:106B080008EE903AA7EE890AF8EEE88AD4ED3F7AC3
:106B1800A7EEA80A0EF03CF994ED3D0AD4ED3A7AB6
:106B2800288028EE000AA7EE890AD4ED407AA7EE5D
:106B3800A80A0EF02DF994ED3E0AD4ED3B7A688050
:106B480028EE000AA7EE890AD4ED417AA7EEA80A32
:106B58000EF01EF9A880BDEC048B38BDA0190020EA
:106B68000800002008B50A4890F8093100EB4303F3
:106B78000A22B3F8181189B2A0F8201100F5947010
:106B880002F04FFF80B209F0EDFF024B188008BDFC
:106B9800A0190020C01800202DE9F04F2DED028B20
:106BA80085B080460293934B1B889807934637D548
:106BB800109B9148DC89B0F900301B1B03F2F315D8
:106BC80040F2E632954203D8002BB8BF5B4201E0A1
:106BD8004FF4FA73B0F90220121B02F2F31440F2D8
:106BE800E630844203D8002AB8BF524201E04FF48D
:106BF800FA729342B8BF1346C3F5FA73052293FBA2
:106C0800F2F30A22643B534398F81C20D2105343F2
:106C1800642293FBF2F3134423EAE373DBB200E04C
:106C280064230093CB1C019347460025019BDFF8A2
:106C3800E8A113F8016F0193022D4FEA450905D128
:106C4800BAF904301B365E43761148E06B493AF8CE
:106C5800152031F91510022012FB0011CBF10002AA
:106C6800914203DB59450A46A8BF5A466449029B2C
:106C780031F90940141B33F9152014440AF0FEFABF
:106C880088B107EE904A5F4AB8EEE70AB2EE048A86
:106C9800505D80EE080A09F08FF920EE080AFDEE33
:106CA800C07A17EE904A534A1288D10713D43AF99A
:106CB80009301B365E4393074FEA26160FD598F81E
:106CC80012305C439DF900305C43642394FBF3F479
:106CD80006EB241603E098F80860744326114A4B23
:106CE800042433F9093093FBF4F4341B474EAB5DAD
:106CF8009A467B78524663435343022D4FF0640211
:106D080093FBF2F34FEAE31308EE103A304609D149
:106D1800B8EEC80A04301E21D6ED030A03F0FAFEC5
:106D2800BDEEC08A394A308AFE7A02F1140E00FBA1
:106D380004F35EF82510DB1206FB0316B6F5001FF8
:106D4800334BA8BF4FF4001602F120019E42B8BF92
:106D58001E4651F8253041F82540E31A4FF6FF71D9
:106D68000009B1FBF0F098F850104EF82560584330
:106D780083114FEA850C761300EE103A79B102F1CF
:106D88002C00B8EEC00A00EBC500D2ED030ACDF81E
:106D98000CC003F0BFFEDDF80CC0BDEEC00A7B7D61
:106DA80010EE102A18EE101A534352465A4313464F
:106DB8003144642293FBF2F3164A1B12194422F859
:106DC800091018EE100A02F1080101354CF801000B
:106DD80002F114012032032D4CF801604CF8023006
:106DE80007F101077FF422AF05B0BDEC028BBDE8C7
:106DF800F08F00BF98190020982A0020EE2B002061
:106E0800BC270020345E010834100020501B0020ED
:106E18000000E0FF941B0020E41000202DE9F04F53
:106E28002DED028B87B000260593C14B0491B3F971
:106E38000270B3F900300292002FB8BF7F42002BD6
:106E4800B8BF5B429F42B8BF1F46B7F5FA7F80467E
:106E5800A8BF4FF4FA770090B3460196B24634467D
:106E6800B44D2B8899075AD0B14BB34A33F8143034
:106E780032F91420022013FB0022029B5B429A4243
:106E88004FEA440103DB029B9342A8BF1346AB4A77
:106E980031F90290059A32F91420C9EB030303EB88
:106EA80002090AF0EBF988B107EE909AA44BB8EE04
:106EB800E70AB2EE048A185D80EE080A09F07CF849
:106EC80020EE080AFDEEC07A17EE909A98F808307E
:106ED800642203FB09F393FBF2F398F81C206FF08C
:106EE800040A0AFB02FA534504DB02EB820A9A45BC
:106EF800A8BF9A46934A52F8241009EB010342F2BC
:106F080010718B42A8BF0B468F498B42B8BF0B4606
:106F180042F8243098F8122053431B1301932D880C
:106F280005F00303012B38D0814B884933F914B09D
:106F3800009B51F824E093F801C0854B33F9140005
:106F480080EAE073A3EBE073B3F5206F4FEA8406A1
:106F580016DC0BEB8B031A0192FBFCF3042290FB6B
:106F6800F2F0181A8644BEF57A5FA8BF4FF47A5E2D
:106F7800784B9E45ACBF41F824E041F8243002E04C
:106F8800002341F824308B597D2693FBF6F6009BAD
:106F9800DB7A7343402693FBF6F6AA0711D50198CE
:106FA800C7F5FA7307FB0BF907FB06F54FF4FA71FF
:106FB80003FB0A9903FB005599FBF1F295FBF1F5E8
:106FC80005E0EB074DBF019D35465A465246DFF8AE
:106FD80088E1630003930EF178015D4B615C33F83F
:106FE80014004FF0040C03B293FBFCF909FB01F108
:106FF8006FF04F0991FBF9F991440EF17C0232F9D7
:10700800141022F814005B1A98F8501093FBFCF344
:1070180000EE103A59B10EF12C00B8EEC00A00EBA0
:10702800C400DEED030A03F075FDBDEEC00A4A4A4E
:10703800039802F1800110EE103A11F804C002F131
:10704800440E09EB05010CFB03F34FF0200C93FBF6
:10705800FCF3C91A20F80E1002F1640002F14C0189
:107068005B4240F82430009B41F8249002F158011B
:10707800013341F8245000930CB90124F0E62C4B5D
:10708800D469B3F90410049B9B790F335B004B431D
:107098005B112F49002BB1F904104FF0040091FB4C
:1070A800F0F0A3EB0000B8BF5B42322B98F80D104C
:1070B8000BDC2A4B01FB00418B42A8BF0B46284939
:1070C8008B42ACBFD361D16101E00023D36198F852
:1070D800031001FB00F32349097803294FEAA3139E
:1070E8000CD9B8F84E10B1F5FA7F07D2484283425E
:1070F80003DB8B42A8BF0B4600E00346D16953650A
:1071080041F34F31B1F5807FA8BF4FF480716FF024
:10711800FF008142B8BF014658180023A2F8480072
:107128001166D36607B0BDEC028BBDE8F08F00BFD7
:10713800E410002098190020EE2B0020BC27002026
:10714800345E0108C01B0020F0D8FFFF641B00203C
:107158003410002080C1FFFF501B0020FEFFFF0FEE
:10716800020000F0F01C00202DE9F04F2DED028BFD
:1071780085B080460393AA4B02911C88019204F0C3
:107188000204A4B294B1A74BB3F90240B3F900309A
:10719800002CB8BF6442002BB8BF5B429C42B8BF0A
:1071A8001C46B4F5007FA8BF4FF40074C246002502
:1071B8009C4B9D4833F815209C4B50F8256033F9BB
:1071C800153083EAE377A7EBE37711B2B7F5206FC1
:1071D8004FEA450B4FEA41014FEA850911DC0427C4
:1071E80093FBF7F3CB1A1E44B6F57A5FA8BF4FF4AA
:1071F8007A568F4B9E42ACBF40F8256040F8253048
:1072080002E0002340F8253050F809609AF80B3066
:107218009AF80170F6115E43814B1B884F439B0718
:107228004FEAA6164FEAA71756D0824B33F90B3010
:10723800022112FB0132019B5B429A4203DB019B54
:107248009342A8BF13467C4A3BF902209A1A039B33
:1072580033F91530D31808EE103A0AF00FF868B170
:10726800B8EEC80A754BB2EE048A80EE080A585D7B
:1072780008F0A2FE20EE080ABDEEC08A704918EE9A
:10728800102A59F8013042F2107013448342A8BF03
:1072980003466C4898F808208342B8BF034649F86B
:1072A800013018EE101A4A4398F81C1001EB8101BE
:1072B800D2114842824203DB8A42A8BF0A461046DE
:1072C80098F8122053431B13F61A3F1A6643674374
:1072D80003EB662600EB6727DFF86CE1534B0EF1F2
:1072E800780C3BF803101CF805C00BB2042093FB84
:1072F800F0F202FB0CF2A7EBA2170EF184023BF9A5
:1073080002C02BF8021098F85010CCEB030393FB43
:10731800F0F300EE103A59B10EF12C00B8EEC00AA5
:1073280000EBC500DEED030A03F0F4FBBDEEC00A76
:10733800454A02F1800110EE103A485D43435B1163
:1073480002F14400B919C91A2BF8001002F14C01D6
:107358005B4249F8017002F158010AF1010A49F843
:10736800016002F1640149F801300DB901251FE7F8
:107378002C4BD469B3F90410029B9B790F335B0043
:107388004B435B112949002BB1F904104FF004005D
:1073980091FBF0F0A3EB0000B8BF5B42322B98F8EA
:1073A8000D100BDC294B01FB00418B42A8BF0B469B
:1073B80027498B42ACBFD361D16101E00023D3617F
:1073C80098F8031001FB00F32249097803294FEAD2
:1073D800A3130CD9B8F84E10B1F5FA7F07D248427A
:1073E800834203DB8B42A8BF0B4600E00346D1690A
:1073F800536541F34F31B1F5807FA8BF4FF48071D9
:107408006FF0FF008142B8BF014658180023A2F868
:1074180048001166D36605B0BDEC028BBDE8F08F5D
:1074280098190020E4100020641B0020341000206C
:1074380080C1FFFFEE2B0020BC270020345E01082E
:10744800C01B0020F0D8FFFF501B0020FEFFFF0FDD
:10745800020000F0F01C00202DE9F04F2DED028B0A
:1074680085B000260293A94B0192B3F90270B3F9D3
:1074780000300096002FB8BF7F42002BB8BF5B4298
:107488009F42B8BF1F46B7F5FA7F8046A8BF4FF4A2
:10749800FA778146B346B24634469D4D2B88990704
:1074A8005AD0022C58D0994B9A4A33F8143032F9F2
:1074B8001420022013FB0022019B5B429A424FEAF0
:1074C800440103DB019B9342A8BF1346924A8A5E9C
:1074D8009B1A029A32F91420134408EE103A09F064
:1074E800CDFE68B1B8EEC80A8C4BB2EE048A80EEC5
:1074F800080A185D08F060FD20EE080ABDEEC08A93
:1075080018EE102A98F808305343642293FBF2F3DC
:1075180098F81C206FF0040A0AFB02FA534504DBB2
:1075280002EB820A9A45A8BF9A467D4A18EE101ABD
:1075380052F8243019440B4642F210718B42A8BF0E
:107548000B4678498B42B8BF0B4642F8243098F86E
:10755800122053431B1300932B8803F00302012AC4
:1075680001D1022C3FD17048684A30F914006F49A4
:1075780032F914B099F8016051F824E080EAE07516
:10758800A5EBE075B5F5206F4FEA84021EDC022CEE
:1075980016D00BEB8B01090191FBF6F6042190FB49
:1075A800F1F0361AB644BEF57A5F60496048A8BF64
:1075B8004FF47A5E8645ACBF42F801E0505007E0D0
:1075C8008BEAEB75A5EBEB75642DE2DD00208850A6
:1075D80056497D26525892FBF6F699F80B207243CD
:1075E800402692FBF6F69A0713D5022C11D0009B81
:1075F800C7F5FA7207FB06F507FB0BF002FB0A005A
:107608004FF4FA7102FB035290FBF1F092FBF1F593
:1076180008E0DB0704D5022C02D0009D504601E0AB
:1076280035465846404BDFF810E133F9141004236F
:1076380091FBF3F30EF17801022C615C03FB01F37B
:107648006FF04F0193FBF1F303444FEA440208EE55
:10765800103A0CD1B8EEC80A0EF104001E21DEED76
:10766800030A039203F056FA039ABDEEC08ADFF8C4
:10767800C8E02D4B0EF18801D05A535E505298F84D
:1076880050100FFA80FCC3EB0C034FF0040C93FB73
:10769800FCF300EE103A69B10EF12C00B8EEC00A06
:1076A80000EBC400DEED030A039203F033FA039AF9
:1076B800BDEEC00A1F4910EE103A085D00FB03FC3E
:1076C80018EE103A4FF0200E58199CFBFEFCA1F161
:1076D8003C0ECCEB000022F80E00A1F1340209F1B7
:1076E800010942F82430A1F128031C3943F8245039
:1076F800CCF1000341F824300134032C7FF4CDAEE3
:1077080005B0BDEC028BBDE8F08F00BFE41000208F
:1077180098190020EE2B0020BC270020345E0108B9
:10772800C01B0020F0D8FFFF34100020641B00208D
:1077380080C1FFFFD01B0020501B00202DE9F04F17
:107748002DED0A8B85B08246039390F85030029154
:1077580090461BB1322BA8BF322300E0012307EE6D
:10776800903AB8EEE7BADFEDD97AD94BDFEDD9BA5E
:107778001B88D94C019487EE8BBA002B08BF0123D4
:10778800D64D07EE903AF8EEE79A238869EEABBA41
:1077980013F0020F3BEE2BBA8BEE8BBA26D0B5F95D
:1077A8000030B5F9022083EAE37182EAE270A1EBC6
:1077B800E371A0EBE27088420646B8BF0E46B6F504
:1077C800E17F16DA8842DFEDC6AA05DD002AD8BFB8
:1077D800524207EE902A04E0002BD8BF5B4207EE26
:1077E800903AF8EEE77AC7EEAAAA04E0DFEDBDAA60
:1077F80001E0F7EE00AA9FEDBB9ABB4C56464FF04E
:10780800000BB0EE49AADFF8189339F91B300CEEDB
:10781800103AB8EECCCAF5EE047A35F91B302CEEE6
:1078280027CA08EE903A019BBDEECCCA1988F8EE3B
:10783800CC7A9FEDAECA89074FEA4B0727EE8CCA70
:10784800F8EEE88A00F08580A94931F91B3007EE87
:10785800903AF8EEE77AB0EE007AE8EE877AC8F167
:107868000000FDEEE77A17EE901A814203DB4145EE
:10787800A8BF414608469F49039B795E401A33F9E1
:107888001B10084407EE900AB8EEE78A09F0F6FCE8
:1078980050B19949B2EE049A88EE090A11F80B0022
:1078A80008F08AFB20EE098A9AF81C30DFED936A0B
:1078B8000AEE103A9AF8083007EE903AF8EE677A2E
:1078C800B8EE4AAA68EE277AB1EE047A67EEA67A8D
:1078D8002AEE077AFDEEE77A17EE901AF1EE477A6C
:1078E800BDEEE7AA1AEE103A994208DBBDEEC7AA28
:1078F8001AEE103A8B42A8BF0B460AEE103A80499E
:1079080001EB8B01D1ED007AE8EE2B7ABBEE0E7A13
:10791800F4EEC77AF1EE10FAB8EECAAA09D4B3EEBB
:107928000E7AF4EE477AF1EE10FAC8BFF0EE477A15
:1079380001E0F0EE477AC1ED007A9AF8123009EECC
:10794800103AB8EE499A67EE897A9FED6E9A27EE5B
:10795800899A019B1988CA0750D439F90700002869
:10796800B8BF4042B0F5206F02DD0020206025E05E
:107978009FED657A737868EE877A07EE103AB8EE6D
:10798800477A87EE877AD4ED007A37EE4C7AE7EEBD
:107998002B7A9FED5E7AF4EEC77AF1EE10FA09D4ED
:1079A8009FED5B7AF4EE477AF1EE10FAC8BFF0EE7D
:1079B800477A01E0F0EE477AC4ED007AF37AD4ED25
:1079C800007A08EE103AB8EE488A8B0768EE277AF4
:1079D8009FED508A27EE888A14D578EECA8AF0EE91
:1079E8004A7AEAEEA87A38EE498AF0EE678AF0EE2B
:1079F800497AEAEE887AB0EE678A03E0B0EE498AFF
:107A0800F0EE4A8ADFF81C919FED437A09F178017C
:107A180009F1A4001BF8013007EE903AF8EEE77A76
:107A28004FEA8B0167EECC7A0844E7EE878A043484
:107A3800013690ED007A80ED00CA3CEE477A09F1F4
:107A4800AC0087EE2B7A0144D1ED007A37EE677AE5
:107A5800F0EE68CAEBEE077A3CEE880AC1ED007AD0
:107A680009F180011BF8013008EE903AF8EEE88A37
:107A780067EEA87ADFED298A67EEA88A30EE680AF1
:107A88000DF086F909F14401FDEEECCAC8531CEE6D
:107A9800903A09F14C01BDEEC88AF1EE688A41F8C6
:107AA8002B30FDEEE88A09F1580118EE103A41F83A
:107AB8002B3009F1640118EE903A4F4641F82B300B
:107AC800BBF1000F30D14FF0010B9CE683F9223E49
:107AD80008100020BD37863598190020E4100020D2
:107AE8000000E14300000000E01B0020CDCC4C402A
:107AF800EE2B0020BC270020345E01086F12033CE7
:107B0800EC1B00200AD7A33D0000A043000040C39F
:107B1800000040430AD7233CA69B443BF7CC92384D
:107B280034100020501B0020029AB5F904309479D3
:107B3800640028345C434B4BB3F9043000EE103A30
:107B4800BAEECF0A0DF024F96411201A002C07EEC2
:107B5800900AB8BF6442322CF8EEE76A03DD0023CE
:107B6800C9F81C3029E0FDEEE99A19EE903A23F0A5
:107B7800030307EE903AF8EEE79ADFED3B7A9AF8BE
:107B88000D30C9EEA77A07EE103AB8EE477AD9F861
:107B98001C3026EE877A67EE277AFDEEE77A17EE35
:107BA800902A1344314A9342A8BF1346304A93425D
:107BB800ACBFC9F81C30C9F81C20FB695B13B3F5CE
:107BC800807FA8BF4FF480736FF0FF029342B8BF65
:107BD800134607EE903AF8EEE78AFDEEE67A9AF851
:107BE800032017EE903A53439B1107EE903A214B2E
:107BF8001B78032BB8EEE78A14D9BAF84E20B2F5F1
:107C0800FA7F0FD2FDEEC87A534217EE901A9942C6
:107C180004DB914217EE903AA8BF134607EE903A5C
:107C2800B8EEE78A38EE280ABDEEC00A8DED010AE3
:107C3800BDF9043000EE103AB8EEC00A0DF0A8F80D
:107C4800BDEEC88AFDEEE88A0023A7F8480087ED54
:107C5800158AC7ED188AFB6605B0BDEC0A8BBDE82E
:107C6800F08F00BF3410002000803B45FEFFFF0F5F
:107C7800020000F0F01C00202D4B2E4A1B681268F1
:107C880010B51A602C4A1168596051689268DA6018
:107C98002A4A996011681961516892689A61284A5C
:107CA80059611168D961516892685A62254A196206
:107CB80011881985518859859188D288DA85224A90
:107CC8009985118819865188598692889A861F4AFB
:107CD8001188D986518819871946928821F83A2F30
:107CE8001B4A10780022824206DA1A4C34F81240F5
:107CF80021F8024F0132F6E7174A1288A3F86420E8
:107D0800164A1288A3F86620154A1188A3F8681045
:107D180051889288A3F86C20124AA3F86A10128836
:107D2800A3F86E20104A5289A3F85E2010BD00BF48
:107D380020280020D42B00209C1B0020A81B0020FA
:107D4800B41B0020E410002034100020DA100020BA
:107D5800F01C002054100020C01A0020EC0F002056
:107D68003A1000206C100020401000202DE9F84344
:107D78000E4B93E8800305460E460024B44213DAFE
:107D88007B1933F9140008EB050333F9142009EBC8
:107D9800050333F914301344022293FBF2F3C01A9B
:107DA80008F091F80134E9E7BDE8F88320280020BD
:107DB80070B5472007F0D6FF174B1B681B0307D584
:107DC800164B174A5B6810681B68C01A08F06CF8F5
:107DD800144E154C154D307808F066F8236828685D
:107DE800C01A08F070F863686868C01A08F06BF881
:107DF8000F4B188808F058F80E4B188808F054F8FC
:107E08000D4B188808F050F8337823742B68A3605A
:107E18006B68E36070BD00BF802900202028002027
:107E2800D42B0020DA1800200C280020DC180020B1
:107E3800D8180020D6180020741000207FB5264CD2
:107E4800264E274D2749284A284B20B12848008824
:107E5800B0F5805F31D23088ADF8040028781E4D27
:107E680091F8201012788DF806008DF807108DF81B
:107E780008201B788DF8093001A8294606220CF045
:107E88005DFD30B30198BDF808302860AB80532001
:107E980007F068FF208808F007F8A07808F004F8D1
:107EA800E37801932379029301A86379039307F098
:107EB80061FF0F4B00221A800BE03088208091F878
:107EC8002010287812781B78A070E17022716371F5
:107ED800DDE704B070BD00BF041C00209819002025
:107EE800D4180020782B0020630E0020C80E002034
:107EF800A0290020A0F17D03012B70B504460D4692
:107F08000A4E05D830687D2101F088FD84F02004F0
:107F18003068214601F082FD35B12B881C4404EB02
:107F2800142404F0FF042C8070BD00BF88190020C1
:107F38000A4A138801331380094A1368013313600E
:107F4800084A138801339BB2202B01BF00231380FA
:107F5800054A138808BF013313807047A029002001
:107F6800882900208C2900208E29002038B53A4B1A
:107F78001B78083B012B05460C466BD8452007F0BB
:107F8800F1FE284607F0EEFE0C2D23D004D80A2D6A
:107F98000AD014D835B138BD0E2D4BD02ED3FF2DB5
:107FA80050D038BD206849E0207807F0DBFE6279C0
:107FB8006378002A14BF80200020184300E020784E
:107FC80007F0D0FEA07807F0CDFEE07807F0CAFEF3
:107FD80020793BE0B4F9000007F05CFFA07807F0D7
:107FE800C1FEE07807F0BEFEB4F9040007F052FFC6
:107FF800B4F90600BDE8384007F04CBF6378207834
:108008008BB180F0800007F0ADFEA468E0B207F005
:10801800A9FEC4F3072007F0A5FEC4F3074007F044
:10802800A1FE200E12E007F09DFE6068BDE8384012
:1080380007F049BF206807F037FF6068BDE838409F
:1080480007F032BF054807F06BFE0020BDE8384056
:1080580007F088BE38BD00BF042800202B7D01082A
:108068002DE9F04FB84BB94F1A888BB00193002A0D
:1080780040F09D80B7F8CA07B54E42F20103C41A12
:1080880060426041FFF7DAFEFFF7F6FD34684920E9
:1080980007F068FEAF4B2546186807F005FF55F84E
:1080A800040B07F001FF2846FDF78CFF04F11000D0
:1080B800FDF788FF04F11C094FF01008A64D0123B5
:1080C8002A6803FA08F3134203D0D9F8000007F02E
:1080D800FAFE08F10108B8F1130F09F10409EDD10E
:1080E80004F12800FDF75EFFB7F84031B4F92E001F
:1080F800C01A07F0D9FE2B68D90408D5974BB4F8F5
:1081080064001B88181AC0F30D0007F0CDFE2B6819
:108118009A0403D5B4F8660007F0C6FE2B685B0521
:1081280003D504F16800FDF73DFF2B68180403D55B
:10813800B4F86E0007F0B8FE04F13000A046FDF771
:1081480031FF04F13600FDF72DFFB7F8403138F95B
:108158003C0FC01A07F0A8FE0127814B1B789F42ED
:1081680008DA38F9020FB4F93C30C01A07F0ABFE50
:108178000137F2E72B68990505D5B4F95E00A0F23E
:10818800DC5007F0A0FE326876487260B260121ABE
:108198001111754A4A43531C032293FBF2F202EB76
:1081A80042029A1A702303FB02033360C0E16F4B4B
:1081B8006F4A1B6811688B4206D00AA9002041F853
:1081C800203D1360FFF7D2FE019B97F8CA171B8862
:1081D80097F8CB070B44013BB3FBF0F200FB1233DB
:1081E8008B4280F070815A4F0120FFF727FEFFF77E
:1081F80043FD50203E687D6807F0B4FDBA683B68CF
:1082080010681B687A6803441068A3EB400007F005
:108218005AFE6A6873689B1A0293AA68B3689B1A25
:108228000393EA68F36802A89B1A0493FDF7CAFE51
:108238002A6933699B1A02936A6973699B1A0393C3
:10824800B369AA6902A89B1A049307F093FD06F183
:108258001C0B05F11C0810243F4901220B68A240A1
:108268001A428A4606D0DBF80000D8F80030C01A57
:1082780007F029FE0134132C0BF1040B08F1040854
:10828800EAD106F1260005F12601002331F9024F53
:1082980030F9022F121B02AC44F823200133042BBF
:1082A800F4D103214FF000094FEA89035FFA83F9FB
:1082B80002AB53F821206AB102F108000F2802D856
:1082C80049F0010906E08032FF2A94BF49F002090B
:1082D80049F0030911F1FF31E6D2484607F042FDA3
:1082E80000240DF1080BA04609F00302022A16D05B
:1082F800032A1DD0012A4ED1B8F1000F05D1DBF8B1
:1083080000402401E4B2904645E0DBF8000000F0AC
:108318000F00204307F026FD4FF000083BE0B8F1BE
:10832800000F0CD0DBF80000C0F3031020432CE052
:10833800B8F1000F1ED19BF8010007F013FD9BF860
:10834800000007F00FFD26E08C290020EC1000202B
:108358002028002088290020802900207C2900204E
:10836800F01C00202C280020B76DDBB694290020D3
:1083780090290020DBF80000C0F30330204307F009
:10838800F1FCDBF80000C0F3071007F0EBFCDBF8AA
:1083980000402401E4B20BF1040B06AB9B454FEA05
:1083A8009909A1D1B8F1010F02D1204607F0DAFCF2
:1083B800DAF8001011F480541FBFB6F86430B5F82D
:1083C80064209B1A029318BF01248A040AD50AABB9
:1083D80003EB8402B5F86600B6F866301B1A42F85B
:1083E800203C01344B0513D502AB03EB840C06F19A
:1083F800660E05F1660000233EF9022F30F9028F60
:10840800C8EB02024CF823200133032BF4D10334C8
:1084180008040BD50AAB03EB8402B5F86E10B6F866
:108428006E305B1A42F8203C013400E0FCB1012CAC
:1084380003D1029807F047FD19E0631E002002AA45
:10844800400052F82320C0B20AB140F00100013BBD
:10845800F5D507F087FC4FF0000802AB53F8280069
:1084680008B107F030FD08F10108A045F5DB302020
:108478000321FFF77BFC36200321FFF777FC2F4B06
:108488003C201978FFF772FCDAF80030990506D518
:10849800B6F95E00B5F95E30C01A07F014FD3A6807
:1084A80027487B687A60121A1111264ABB604A4332
:1084B800531C032293FBF2F202EB42029A1A702336
:1084C80003FB02033B60204B1B681A0630D51F4C88
:1084D8001F4D22682B689A420BD162686B689A42DA
:1084E80007D1019B1B88102B11D11A4B1B885B06E7
:1084F8000DD1482007F036FC206807F0E4FC6068DE
:1085080007F0E1FC23682B6063686B600EE0124A99
:108518000F4B11782A7C914208D1104A996810684B
:10852800884203D15268DB689A4201D0FFF740FCC9
:1085380007F0E8FB0BB0BDE8F08F00BFF01C00208F
:108548002C280020B76DDBB6C42700207810002047
:108558000C2800208E290020DA180020DC180020C2
:108568002DE9F84F0C9E3A4CC2EB030B0B9BF61A05
:108578006368002914BF4FF0060A4FF0040A01335C
:108588000546904613D1236853455ED2314A324896
:1085980052F82320032B98BF294607F0D1FB6368C4
:1085A800013363602D4B002205469A7113E00025C4
:1085B80011E02B4A1278954240DA0B9BE3B109FB94
:1085C80006F2995C01228A40264909680A4213D1B9
:1085D800636801336360D4F804900A9B1C4F994583
:1085E800E7DB2BD10A2007F0BDFB3B6801333B607A
:1085F8004FF0FF337B6021E0184A917921B12C209C
:1086080007F0B0FB013501E001219171226809FBF7
:108618000BF308EB030752B958F8030007F080FB87
:1086280097F904104B1C0544D2D00F4802E03A4495
:108638000E48117907F084FB0544C9E720685045C6
:108648002CBF00200120BDE8F88F0020BDE8F88F7E
:1086580098290020385E0108367D0108041C002096
:108668000C01002080290020457D01080D880108A3
:1086780030B585B004AC002524F8025D0091ADF852
:10868800060021461020FFF735FC9DF8060021461C
:10869800FFF730FC9DF807002146FFF72BFC9DF8FB
:1086A80000002146FFF726FC9DF801002146FFF750
:1086B80021FC9DF802002146FFF71CFC9DF80300F1
:1086C8002146FFF717FC9DF80E00C043C0B22946AB
:1086D800FFF710FC05B030BD10B5054C206801F05F
:1086E8009AF918B1206801F093F9F6E710BD00BFB8
:1086F8005819002013B5044601A9006808F072FC57
:10870800132008F0ABFCBDF9040008F095FC1B2011
:1087180008F0A4FCBDF9060008F08EFC232008F040
:108728009DFC2368002BB4BF53204E2008F084FC26
:1087380001A9606808F056FC122008F08FFCBDF90A
:10874800040008F079FC1A2008F088FCBDF906003E
:1087580008F072FC222008F081FC6368002BB4BF8B
:108768005720452008F068FC02B010BDF8B5044653
:108778000E4617460025204620210CF030F9044605
:10878800D0B1013420460CF08FF9B0F5617F05DBDC
:1087980040F634039842A8BF184601E04FF46170D0
:1087A800A0F56170192390FBF3F00DB9307000E06B
:1087B80070703B7801333B700DB90125DBE720462B
:1087C800F8BD30B505460C461346294622460248F0
:1087D800BDE8304002F0BDBB3C7E01087FB504789F
:1087E8000646E4B9354B1B6803EB8403192193F85B
:1087F8007B0093F87C6093F8792093F87A304FF4F3
:10880800617511FB005011FB0651009001912C4835
:108818002146013402F09DFB142CE3D14BE00CF00F
:1088280043F91328054641DC244B701C1C682021A1
:1088380000238DF80F300CF0D2F81E35064670B1C3
:10884800013630460CF030F91A289FBF04EB850337
:1088580058709DF80F30013398BF8DF80F303046AF
:1088680020210CF0BCF8064670B1013630460CF0F9
:108878001BF90D289FBF04EB850398709DF80F30F6
:10888800013398BF8DF80F3004EB85043046E11CA6
:108898000DF10F02FFF76AFF9DF80F30042B0AD085
:1088A800601C002104220CF064F804E00548002153
:1088B8001322FFF786FF04B070BD00BF50100020E0
:1088C8005B7E0108707E0108014806F073BD00BF99
:1088D800767E01082DE9F04304788FB00546002C18
:1088E80059D17B4B0021142209A807AED3F8008088
:1088F8000CF03FF80722304600210CF03AF805A8A2
:108908000023A700059308EB070583801A467149E1
:10891800B5F802E031F813C01CEA0E0F0AD00DF1C9
:10892800380C0E3102F1010E6244595C02F81C1C2D
:108938005FFA8EF20133072BE9D100210B46664A14
:10894800B5F802E011F802C01CEA0E0F0AD00DF1CA
:10895800380C063203F1010E63448A5C03F8242CB8
:108968005FFA8EF301310629E9D118F807305B491F
:108978008DE841006A78029209A81A0903F00F03EA
:1089880007F02EFD2146564809AA013402F0E1FA03
:10899800202CA6D198E00CF087F81F28044600F395
:1089A800868028462021E4B20CF019F81F2C02D941
:1089B800FFF78AFF88E0464B1B6803EB8404451CDD
:1089C8000021204604220BF0D4FF0027454B09AEB6
:1089D800304600210A2217F803905FFA87F80BF057
:1089E800C8FF002315F8012B32B10A2B04D04A45E1
:1089F80002D0F2540133F5E74A455ED108F1FF335E
:108A0800032B09D8DFE803F01005023F0DF123011D
:108A180034E00DF123011EE030460CF045F82378D0
:108A2800C0B243EA001006E030460CF03DF8237867
:108A380000F00F001843207031E00133062B0AD0F4
:108A4800244800F11B069E5D9642F6D103445A7DE8
:108A580063881343638011F8012F02B30023EFE703
:108A68000133072B0AD01B4800F10E069E5D964283
:108A7800F6D130F8132063881343638011F8012F6F
:108A88006AB10023EFE730460CF00EF80F2804DC3B
:108A980030460CF009F8607001E00023637001377C
:108AA800052F93D1012405F0B7FE6CB980E70E4875
:108AB80000211F22FFF785FE06E020460021042240
:108AC8000BF057FF0024EEE70FB0BDE8F08300BFBE
:108AD8000C1C0020505E0108655E0108847E0108B8
:108AE800937E0108715E0108707E0108F8B504786C
:108AF800064674B9304DB5F8C421B5F8C6312F48CB
:108B08002146013402F025FA042C05F10405F2D1BE
:108B1800F8BD2B490BF036FFA8B9274B4FF47A71F3
:108B28004FF4FA62A3F8C411A3F8C621A3F8C81138
:108B3800A3F8CA21A3F8CC11A3F8CE21A3F8D01129
:108B4800A3F8D221F8BD30460BF0AEFF0328054646
:108B58002BD8304620210BF042FF044630B10134B7
:108B680020460BF0A1FF0126074600E006462046F6
:108B780020210BF034FF10B9BDE8F840A4E601301D
:108B88000BF092FF012EF7D1A7F2EE2240F2DC5350
:108B98009A42F1D8A0F2EE229A42EDD8064B7035EF
:108BA80003EB85039F80D880F8BD06480021032287
:108BB800BDE8F84005E600BFEC1000209F7E0108E4
:108BC800B27E0108778A01082DE9FF41047805463D
:108BD800002C39D17348744D06F0ECFBD5ED047ABE
:108BE800F5EE407AF1EE10FA00F0D88021466F4891
:108BF80002F0AFF995ED040A684602F03FF8014625
:108C08006B4802F0A6F995ED050A684602F036F8B9
:108C18000146674802F09DF995ED060A684602F09C
:108C28002DF80146624802F094F995ED070A684666
:108C380002F024F8013401465E4802F08AF90C2C4F
:108C480005F11005CAD1A9E05B4905220BF0DEFE4B
:108C580040B9554B03F1C002002143F8101F93425D
:108C6800FAD19BE02846554904220BF0CFFE044672
:108C78002846002C40D120210BF0B1FE002800F03E
:108C88008D80451C28460BF0B8FE07464C4B53F820
:108C980024601EB94B4806F08DFB7FE0284631461C
:108CA800FAB20BF0B3FE01340028EFD13E4B03F1CA
:108CB800C0029E46002143F8101F9342FAD1424B4E
:108CC80003EBC4029846D2F804C0BCF1000F04D1EB
:108CD80031463E4802F03DF957E0002718F8343095
:108CE8009F42F5DA3B010EEB030563440FCB1035C9
:108CF80085E80F000137F1E70BF0D6FE0B28064692
:108D080047DC284620210BF06AFE054650B10135A4
:108D1800284601F029FF244B03EB061383ED040AD0
:108D2800012400E00446284620210BF058FE0546A1
:108D380048B10135284601F017FF1B4B03EB06131A
:108D480083ED050A0134284620210BF048FE05462C
:108D580048B10135284601F007FF134B03EB061312
:108D680083ED060A0134284620210BF038FE10B99D
:108D7800FFF7AAFD12E0013001F0F6FE0A4B032CC2
:108D880003EB061686ED070AF2D11148FFF71CFF20
:108D980004E0104801210C22FFF713FD04B0BDE8E0
:108DA800F08100BFB87E0108EC100020D37E0108D6
:108DB800D97E0108F5870108B27E0108DD7E010829
:108DC80038660108E27E01086C7D0108F17E010821
:108DD800D77B0108707E0108F0B5047887B0064695
:108DE8001CBB514B1968062303FB0411192091F889
:108DF800CA5091F8CB7091F8CE2091F8C9304FF451
:108E0800617610FB056510FB07600095019091F8ED
:108E1800CC000290C8314548497903912146013474
:108E280002F097F80C2CDCD17CE00BF03DFE0B280F
:108E3800044672DC3C4B701C1D68202100238DF811
:108E480017300BF0CCFD064680B1013630460BF0EA
:108E58002BFE03289FBF062303FB045383F8CE0091
:108E68009DF817309CBF01338DF81730304620210C
:108E78000BF0B5FD074680B1013738460BF014FEFC
:108E88000D289FBF062303FB045383F8C9009DF8F0
:108E980017309CBF01338DF8173006266643A91991
:108EA8003846CA310DF11702FFF760FC20210BF09C
:108EB80096FD074670B1013738460BF0F5FD1428CA
:108EC8009FBF9DF817307619013386F8CC0098BFFC
:108ED8008DF81730384620210BF081FD78B101302C
:108EE8000BF0E2FD0D289FBF062303FB045383F814
:108EF800CD009DF817309CBF01338DF817309DF8D1
:108F08001730062B0ED0062202FB04500021C93070
:108F18000BF02FFDFFF7D8FC04E0054800210B22D9
:108F2800FFF74FFC07B0F0BD50100020FD7E010890
:108F3800707E0108F0B5027887B0AAB94C4C04F1EC
:108F480018064C4B94F9F41193F900208A4272D018
:108F580093F90C208A426ED093F918308B426AD06C
:108F68000834B442EDD180E0002204920592451CF9
:108F78000BF09AFDC4B260B200F0F2F9074618B1DE
:108F88008DF81040012400E00446284620210BF00B
:108F980026FD054638B1013528460BF085FD01341C
:108FA800ADF81200E4B20026284620210BF017FD88
:108FB800B0B3451C28460BF077FD00222E4951F826
:108FC800223083425FFA82FE04D00132082AF5D1AA
:108FD800002300E0734651F82320824220D1022E5C
:108FE8000FD0032E12D05A1E012ED2B204D0042A5A
:108FF80013D88DF814300EE0042A0ED88DF81530E9
:1090080009E0052B09D88DF8173004E09A1E052AC7
:1090180003D88DF816300134E4B20136042EC3D1DA
:10902800052C03D807B0BDE8F0404DE404AB03CBF2
:109038003860796019E094F8F9010F4B94F8F85109
:1090480053F82000B4F8F621009094F8FB0153F887
:109058002000019094F8FA0153F82000029053F888
:109068002530064801F075FF7AE707B0F0BD00BF6C
:10907800EC100020541A0020105E01081D7F010822
:109088002DE9F347047807464CB9204601A9FDF7B6
:109098004BF80134FFF7F4FF122CF6D17EE00BF009
:1090A80003FDC5B2112D74D8781C20210BF097FC54
:1090B8003C4C3D4F05F1D006034614F8168030B9F4
:1090C800A8F10202D2F1000848EB020846E007F1D5
:1090D800260800F1010A597840460BF080FC68B177
:1090E800032D8CBF03230023C8EB00003B4453FA35
:1090F80080F090F82A90B9F1030F02D1FFF7E4FB52
:109108004CE0A9F10203D3F1000850464FF02001CA
:1091180048EB03080BF063FCD8B1B8F1000FEDD0B1
:1091280001300BF0C1FC40F2ED2380B2984205DD1E
:1091380040F6CA039842A8BF184601E040F2EE2064
:1091480004EB4603A0F2EE20192290FBF2F05870CF
:1091580002E0B8F1000FD1D104F8169014F81630D7
:109168001F4497F82620B8F1000F0DD00D4B0F487B
:1091780003EB46062946737840F2EE24192505FBD1
:10918800034301F0E6FE09E02946094801F0E1FE43
:1091980004E0084800211122FFF713FB02B0BDE8E4
:1091A800F08700BFEC100020505E01083C7F0108EA
:1091B8004E7F0108778A010807B50123ADF804102E
:1091C80001A98DF806208DF8073004F03BFE03B0A6
:1091D8005DF804FB2DE9F843404B414C9A6A42F490
:1091E80000129A629A6A22F400129A625A6942F448
:1091F80000125A6106464FF4A06120460122FFF78B
:10920800DBFF4FF4A063238572B6364D02214FF081
:109218000809298528460422A5F82890FFF7CCFFDD
:10922800284601224946FFF7C7FF2F4850F8364025
:1092380000EBC600236842680126570006FA07F8C3
:1092480048EA030396402360A661C5F818902B8A64
:109258009B07FCD4236848EA03032360214B0822B8
:10926800B1B221851A854FF48072A3F828284FF4EB
:109278008062C3F8182840F605531A48028A9507F1
:1092880011D4013BF9D122680323BB4022EA03032E
:10929800236008210222FFF78FFF62B63220BDE863
:1092A800F84300F0AAB90422A6612046FFF784FF1C
:1092B8000B4B4FF480621A850A4B1A8A9207C9D55C
:1092C800228A92B21642064A4FF008004FF4807183
:1092D80015BF9861188511859161EDE7001002406E
:1092E8000010004800080048607F010810B50446D7
:1092F800204600F087FB18B90A2000F07EF9F7E74E
:1093080010BD0C4B5A6882421A4607D01B6983422B
:1093180006D0D36983420BD1022302E0002300E088
:1093280001230021C1620C2000FB0323197259603C
:10933800704700BF541A0020034B4FF4085208B17D
:109348009A6170471A85704700100048034B4FF424
:10935800085208B11A8570479A6170470010004892
:109368000C4B1B6893F90220824209D093F90A201A
:10937800824207D093F91220824208D1022002E0EB
:10938800002000E0012003EBC000023070470020FD
:10939800704700BF501A002038B1438811EA030013
:1093A80003D08B420CBF01200220704730B50A4B16
:1093B8000A491C680A78022A0AD8134604EBC30330
:1093C800551CEAB29D882842F5D00A70981C30BD19
:1093D8000A70002030BD00BF501A0020101C002069
:1093E800014B00221A70E1E7101C00202DE9F0471C
:1093F800877890F803C0214DBBB2C7F1640E03EB28
:1094080083065C42C3F178005FFA8EFE7600CCF1E9
:109418006408A4B280B2A3B20FFA83F9B9F1000FBD
:1094280005DC002B14BFBA464FF0010A00E0F246F3
:1094380013FB03F303FB0CF21AFB0AF392FBF3F39F
:10944800434403FB09F30A2293FBF2F333449BB230
:1094580025F8023FB1F800904A880A34C9EB020A9D
:10946800A4B21AB202FB0AF24FF47A73844292FB56
:10947800F3F34B442B80CED1BDE8F087101C0020BD
:1094880010B544780078002202FB02F3193B6343CD
:1094980003F6C413534340F6C411434393FBF1F35B
:1094A800034921F812300132072AEDD110BD00BF5F
:1094B8002A1C00200430114B33F91000B0F5617FED
:1094C80010B506DB40F6330398420246A8BF1A4699
:1094D80001E04FF461720C78192340F2833013FBDA
:1094E8000404944207DA497813FB01039342B4BF9A
:1094F8000020012010BD002010BD00BF982A0020C8
:1095080010B500F1500302788A4203D18478C278FA
:10951800944204D304309842F5D1002010BD0120B4
:1095280010BD0B4B1B6813F4805F0A4BB3F9063070
:1095380005D0C089421A934207DD084400E0008A3A
:109548008342B4BF0020012070470120704700BF4C
:10955800C4270020982A00201FB5094B1B681B034D
:109568000AD58DF8040001230D2001A98DED030A09
:109578008DF80530FEF7FAFC05B05DF804FB00BF76
:10958800C42700201FB5084B1B681B0309D58DF89D
:109598000400029100230D2001A98DF80530FEF783
:1095A800E5FC05B05DF804FBC427002010B50A4AA5
:1095B8000A4B11689B6800BF12689142F7D1084AAC
:1095C800946A4FF47A7000FB04F2D31AB3FBF4F3F5
:1095D80000FB013010BD00BFE827002010E000E0CC
:1095E800101C002038B50446FFF7E0FF0546FFF7DA
:1095F800DDFF401BA042FAD338BD10B504462CB19C
:109608004FF47A70FFF7EEFF013CF8E710BD2DE943
:10961800F04F06468A4890F9004087B0B442884621
:109628009DF8445011461A469DF8403009D090F9EB
:109638000C40B44207D090F91840B44209D102272F
:1096480002E0002700E001270C2404FB0700047A4D
:109658000CB10020F0E0012E00F0DD80142E05D0C2
:10966800002E40F0E88000957648D6E0DFF814A296
:10967800DAF8183043F00103CAF81830DAF8143071
:109688004FF0904543F40033CAF814304FF0010905
:1096980003224FF4805B04A94FF090408DF8152009
:1096A8000392CDF810B08DF814908DF816908DF8BF
:1096B8001740FDF77FF9A5F828B0C820FFF79DFFF0
:1096C800C5F818B0DAF81430039A43F40033CAF82E
:1096D800143028464FF4C0534FF0020B04A90493EA
:1096E8008DF815208DF814B08DF816408DF81740B8
:1096F800FDF760F96B6A23F470436B626B6A43F49D
:1097080060436B626B6A23F470236B626B6A43F489
:1097180060236B624C4B4D4D4FF480221A6002F16E
:109728008042A2F53F3212236B67082385F879300F
:10973800136885F87A9023F480231360536823F420
:109748008023536095F8783003F1804303F5823322
:109758001A6842F480221A606A6F3D4B22F01F009B
:1097680002F01F02C15809FA02F221EA0202C250AD
:109778006A6F384922F01F0002F01F0250F801E01A
:1097880009FA02F22EEA020242506A6F22F01F0121
:1097980002F01F02C85809FA02F20243CA502E4BBF
:1097A8002E4A1C60DAF81C3043F40003CAF81C3057
:1097B8002B4B04A8DA608DF810608DF811B08DF885
:1097C80012408DF8139006F0ADFB2A238DF8103067
:1097D8009DF813308DF811908DF812401BB104A834
:1097E80006F0A0FB04E01F4B4FF48062C3F884200E
:1097F8001D4B1E4C1C60022385F884301C4A1D4BEF
:109808001D49C5F8983011601B6898471B4BEB62DF
:10981800A4F1500006E01A48009503F08BF90028DF
:109828003FF417AF064B06710C2202FB073787F887
:109838000880786000E0204607B0BDE8F08F00BFE0
:10984800541A00200038014014040140101C002064
:10985800080401400C040140D80042420005FA0502
:1098680000ED00E000E100E0A41900208C1C0020BD
:10987800A81900200C000020700000204063010897
:109888000044004000100240024A1368013313608C
:10989800704700BFE8270020024BD3F89C3003B183
:1098A80018477047101C0020014B1B68184700BF61
:1098B800D82B002010B50020FFF7F6FF074B002437
:1098C8001C7007F0C7F9064B83F8A040C3F8A44002
:1098D800A3F8A840C3F8AC4010BD00BF9C2B0020E3
:1098E800101C002010B510B9BDE81040E2E70023B5
:1098F8000C225A430C4C1119125D824203D00133D9
:10990800102BF5D110BD094BD3F8AC0018B14A782B
:109918004078824206D20022C3F8AC10A3F8A820EF
:10992800C3F8A42010BD00BF88680108101C0020DF
:1099380010B540001428A8BF14200023074A0221AC
:1099480099540B4499181424834201F8014CF5DB0F
:10995800FF21D1540F20BDE81040C3E79C27002009
:109968002DE9F84380460B25013D3FD0224B4FF4AB
:1099780088429A614FF488521A8508F10106322705
:109988004FF005091C4CA38A9BB283F48843A38239
:10999800A38A9BB283F48853A3820120FFF784FF34
:1099A8003846FFF72AFEA38A9BB283F48843A38232
:1099B800A38A9BB283F488530020A382FFF774FF25
:1099C8003846FFF71AFEB9F1000F08D0B9F10109BE
:1099D800D8D14FF4FA70FFF710FEFA27D2E7013E0C
:1099E800D0D14FF47A70FFF708FEBDE7034B044A65
:1099F800DA60BDE8F88300BF0010004800ED00E021
:109A08000400FA0503681B6918470368DB681847F0
:109A180003689B68184703685B68184703681B68F6
:109A280018472DE9F84FB0F90230934218BF0023C8
:109A38002DED048B18BF0370057804460E46914639
:109A4800002D40F0978007EE902ADFED7D8AF8EE32
:109A5800E77AB6EE009A67EEA88ADFED7A7A68EEC2
:109A6800A78AA04668EE898A2746B0EE680A01F000
:109A780001FBB0EE408AB0EE680A01F05BFB88EEAD
:109A8800000A40F2DC5363651023A4F8523018230F
:109A9800A4F85030DFED6C6A60EE266AB7EE006A13
:109AA800B0EE667AA0EE007AD0EE006A37EE067A5B
:109AB80076EE866AC6EE077A84ED046A27EE807A27
:109AC800B0EE498A27EE007A77EE075A84ED017ADC
:109AD800C4ED025A70EE005A84ED037AB8EE007AAB
:109AE800A5EE807A27EE877A67EEA67A84ED057A66
:109AF800C4ED067ADFED557A98ED047A27EE277AD9
:109B0800F0EE678AB5EEC07AF1EE10FA4CBF77EE48
:109B1800487A77EE087A013517EE900A08F00CF8C3
:109B2800D8ED017A67EEA87AC7E90E01F5EEC07A9A
:109B3800F1EE10FA4CBF77EEC87A77EE887A08F122
:109B4800040817EE900A07F0F7FF032DC7E908018C
:109B580007F10807CED1A6F2DC531B042367E3679D
:109B68006367C4F88030A367C4F884300123A4F87D
:109B780002902370D4F85490B4F95280636A276A2B
:109B8800206FE26FD4F840C0D4F88010C4F8802069
:109B9800C9EB060606FA08F64FEAE67B734307FBAD
:109BA8000B332667A7FB06671F44636C656F606706
:109BB8004FEAE27B53430CFB0B3EACFB022373449E
:109BC800B61A67EB0307E36AA26AC4F884104FEA7F
:109BD800E07B434302FB0B3EA2FB00237344B61811
:109BE8005F41E36CA06CB4F95020A5674FEAE17BB4
:109BF8004B4300FB0B33A0FB01011944636B361A7E
:109C0800206B4FEAE57B05FB03F300FB0B3367EBA7
:109C18000107A0FB050119448019794107F05AFD95
:109C280008F1FF3201239340E067C01841EBE3716C
:109C3800424607F04FFDBDEC048B4844BDE8F88F61
:109C48006F12833ADB0F4940F404B53F0000804BA4
:109C58002DE9F8430024244B93F8E060E0B2B042C9
:109C68000DD203EB8003214AD3F8B03032F810103C
:109C78001BB10B2801D8DB6898470134EBE71C4B74
:109C88001B685B032DD500242346E2B2B24228D2DA
:109C9800DFF8549009F1B0074FEA840857F82420F8
:109CA80055689D4215D0284604F096FCEFF31283C0
:109CB800502282F3128828216A6A01FB009001323F
:109CC800C0F808216A6942F001026A61DBB283F3D5
:109CD800118857F808301B6800221A6001342B4697
:109CE800D3E7BDE8F88300BF101C00205410002003
:109CF800C427002008B50E4B1B6813F4805F0D4B7A
:109D080014BFD3F8FC21D3F8002293F8E01092880E
:109D18000023D8B2884204D2074820F81320013320
:109D2800F7E7FFF795FF3220BDE8084065E400BF7C
:109D3800C4270020101C0020541000200A4B1A6869
:109D48000A4B30B502F48052D3F8FC41D3F80052E4
:109D580000230AB1A18800E0A988054820F813105B
:109D680001330C2BF5D130BDC4270020101C002076
:109D78007227002070B5124D0024214605F20520F7
:109D8800702285F804420AF0F4FD2146D5F87832AD
:109D98000B4A0B4493F9020080B102F205241E68B5
:109DA8000E5108199C8884809B79837192F804323B
:109DB80007310133702982F80432E7D170BD00BF42
:109DC800101C0020094B1A680E2303FB0020437A5D
:109DD800FF2B07D0064A12789A4203D9054A32F86F
:109DE800130000E0808800B2704700BFF424002010
:109DF800481A0020982A0020D0ED024A91ED016A05
:109E080090ED015A91ED027AD0ED005AD1ED007A29
:109E180066EE646AE5EE076A27EE657AC2ED006AC7
:109E2800A4EEA77A67EEC57A82ED017AE5EE867A26
:109E3800C2ED027A7047D0ED017A91ED017AD1ED49
:109E4800026A91ED006A37EE877AD0ED027A77EEF2
:109E5800A67AD0ED006A82ED017A76EE866AC2EDC6
:109E6800027AC2ED006A704790ED017AD0ED027A6D
:109E7800D0ED006A20EE077A60EE277A26EE800A97
:109E880081ED017A81ED000AC1ED027A704701384F
:109E98000A4B042804D8DFE800F00507090B0D0079
:109EA800074A08E0074A06E0074A04E0074A02E0D2
:109EB800074A00E0074A1A60704700BF0401002003
:109EC80061740008A16B0008A912010871710008EB
:109ED800256E00084577000813B5062204460321BD
:109EE8001E206B4604F0C4F800283DD09DF80020E1
:109EF8009DF801309DF8021043EA02231BB21B4A69
:109F080007EE903A92ED007AF8EEE77A012067EED4
:109F1800877A92ED027AFDEEE77A17EE903A23807F
:109F28009DF8033043EA01231BB207EE903AF8EE9E
:109F3800E77A9DF8041067EE877A92ED017AFDEED4
:109F4800E77A17EE903AA3809DF8053043EA01239B
:109F58001BB207EE903AF8EEE77A67EE877AFDEEE5
:109F6800E77A17EE903A638002B010BD94000020A3
:109F780013B506220446A82119206B4604F078F888
:109F8800F8B19DF800309DF8012043EA0222022131
:109F98009DF8033012B292FBF1F222809DF8022064
:109FA80042EA032212B29DF8053092FBF1F2628078
:109FB8009DF8042042EA03231BB2012093FBF1F32E
:109FC800A38002B010BD08B524218022192004F016
:109FD800CBF86420FFF711FB20219722192004F009
:109FE800C3F80A20FFF709FB10222321192004F0E7
:109FF800BBF86420FFF701FB024B4FF480521A8034
:10A0080008BD00BF040000202DE9FF41634B1B6819
:10A0180093B11A681AB16249486902434A619A8839
:10A02800ADF8042002228DF807209868002201A9C3
:10A038008DF8062003F006FF3220FFF7DEFA002134
:10A0480011221E2004F090F8012160221E2004F045
:10A058008BF86420FFF7D1FA02A8FFF73DFF002430
:10A068000A2726462546022101221E2004F07CF8F4
:10A078003220FFF7C2FA02A8FFF72EFFBDF9082029
:10A08800BDF90A10BDF90C308A421444A8BF0A462B
:10A0980093421D44A8BF134613F5805F0E440ADDA2
:10A0A800404A938A9BB283F48843013F9382DAD172
:10A0B8004FF0010801E04FF000081E200021122295
:10A0C80004F052F80A27022101221E2004F04CF85D
:10A0D8003220FFF792FA02A8FFF7FEFEBDF908202A
:10A0E800BDF90A10BDF90C308A42A4EB0204A8BFDE
:10A0F8000A469342A5EB0305A8BF134613F5805FF4
:10A10800A6EB010608DD274A938A9BB283F48843AD
:10A11800013F9382D7D101E04FF0000807EE904A43
:10A128009FED217A214FF8EEE77A0021C7EE277AD2
:10A1380070221E20F0EEE77AC7ED007A07EE906AEB
:10A14800F8EEE77AC7EE277A9FED197AF0EEE77A0C
:10A15800C7ED017A07EE905AF8EEE77AC7EE277A4C
:10A16800F0EEE77AC7ED027A03F0FEFF0121202224
:10A178001E2003F0F9FF1E200221002203F0F4FF45
:10A188006420FFF73AFAB8F1000F04D14FF07E537C
:10A198003B607B60BB6004B0BDE8F081FC0200203E
:10A1A800001002400010004800406F469400002054
:10A1B80001C05E46154B37B5082205461A85E820CA
:10A1C80005F088FE0024002005F084FE0DF8040048
:10A1D8000134062CF7D10D4B08229A619DF8002016
:10A1E8009DF8013043EA02232B809DF802209DF858
:10A1F800033043EA02236B809DF804209DF8053064
:10A20800012043EA0223AB8003B030BD00100048B0
:10A218002DE9F04F944D954C2B68954E9BB22380B9
:10A22800228831880A40900585B007D54FF6FF533C
:10A23800904A2B6013780133DBB2137023880B40EC
:10A24800190440F143830023ADF80A302B6887498D
:10A258009AB21804228040F139830B8803F00F0367
:10A268008B70002B40F00483834A844F1368844822
:10A278009BB23B803B8803F0300303803B8803F4A8
:10A2880040533B80D2F800E04BF6BF730EEA03035D
:10A2980083F4005383F0200343F4004343F0800326
:10A2A80013600B8813F0100F804626D1116848F60A
:10A2B8000F730B40734913600B681A7A022A894698
:10A2C80001D0042A05D1FBF7E1FFD9F800301B7A49
:10A2D8003FE1062A6ED15A78052A09D11A78520622
:10A2E80006D1D878FBF7B6FF674B1B681B6A9847FF
:10A2F800664B1B689B6898475CE013689BB2ADF897
:10A308000A30BDF80A301B0540F1F38111685D4839
:10A3180040F68F730B405E4913600A685D4B92B23A
:10A3280013445B0081461A68036893F808E0BEF19D
:10A33800090F8A4617D092B2520002F1804202F504
:10A34800C04211781970517859709188C8B2090AB9
:10A3580041EA002159801189C8B2090A41EA00215D
:10A3680099809289DA8001221A72DA8893F801B00A
:10A37800002A40F0F1801A7812F07F0250D1BBF128
:10A38800090F10D1DA78012A00F2CA8099780029D9
:10A3980040F0C6809988002940F0C2809A723A4BF2
:10A3A8001B685B68BAE0BBF1050F10D193F9032075
:10A3B800002A01DA0823CCE09A78002AFAD19A8890
:10A3C800002AF7D19B7A002B00F0B480F2E7BBF1AA
:10A3D800030F0FD1DA78012A40F0A2809A88002A68
:10A3E80040F09E805A7A42F020025A72264B1B682F
:10A3F800DB6993E0BBF1010F40F09280DA78012A23
:10A4080040F08E809A88002A40F08A805B7A98060D
:10A4180040F18680FBF7E8FF002800F08B807FE0A2
:10A42800012A39D1BBF10B0F7AD1184A5879126831
:10A43800D97892699047D9F800309A7A002A6FD073
:10A4480000286DD11A79002A6AD19B78002B67D130
:10A458000D4B1B68DB6898470A4B1B685A79DA7200
:10A46800DA781A7366E000BF445C00408C1E002056
:10A47800A42B0020F72B0020005C00407A1A002053
:10A48800781A0020A4190020A8190020A81C002070
:10A49800505C004004300020022A41D1BBF1010F7A
:10A4A800B8D0BBF1030F3BD1587920F0800E4FEAAA
:10A4B8008E0202F1804101F5B84110F0800F096861
:10A4C80014BF01F0300101F44051BEF1030F27D849
:10A4D800B3F802E0BEF1000F22D109B39B7AFBB1B9
:10A4E80002F1804202F5B842010613684BBF23F41B
:10A4F800E04323F4804323F0400323F070034BBF71
:10A508009BB29BB283F0100383F4805343F400435F
:10A5180043F080031360A94B1B689B69984709E0C7
:10A52800A74B1B6858465B699847032810D000283A
:10A538007FF440AFDAF80020A24B92B213445B00DC
:10A548001A6800221A603023A8F80030062300E0B9
:10A558000923D9F8002065E1BBF1060F13D11A7859
:10A5680050067DD19A78964B012A02D11B68DB6987
:10A578006AE0022A02D11B681B6A65E0032A6FD1D0
:10A588001B685B6A60E0BBF1000F3AD1598800296B
:10A5980066D15A6822F47F42B2F5003F60D11A783A
:10A5A80012F07F0204D19B88002B00F0F48157E061
:10A5B800012A0AD1824A587912689269904700287C
:10A5C8004ED1D9F800309B7A17E0022A48D15A793F
:10A5D80002F00F010BB29B0003F1804303F5B8436F
:10A5E80012F0800F1B6814BF03F0300303F44053CC
:10A5F800032935D812F0700F32D1002B40F0CB81EF
:10A608002EE0BBF1080F04D11B78590600F0C58174
:10A6180026E0BBF10A0F23D11A7802F07F02012A43
:10A628001ED19A7AE2B15988D1B95A6822F47F4288
:10A63800B2F5803F14D1624A5879126892699047FE
:10A64800002800F0AC810BE053B1D9F800204FF09E
:10A65800000AA2F812A093615046984750460BE0B2
:10A66800574BD9F800201B6850781B699847032876
:10A6780002D1554B1B6806E0D9F800301A8A4FF60C
:10A68800FF718A4201D1092203E0022800D012B9E1
:10A6980008221A72C7E093F90010002923DAD98832
:10A6A80003910398DFF818E1824202D9039A1A82CB
:10A6B80011E08A420FD2DEF8001091F82C00824295
:10A6C80001D2002105E092FBF0F100FB112212B942
:10A6D80001213E4A1170DEF8002092F82C209A825F
:10A6E800FBF7D4FD9FE003221A724FF440533B80DE
:10A6F80099E0BDF80A301BB2002BBFF6A7AD116870
:10A7080040F68F730B4013602F4AD2F8009099F8E7
:10A718000830022B934600F08280042B7FD0032B55
:10A7280001D0052B75D1D9F81830B9F810209BB98C
:10A73800B9F81020002A4FD04FF440533B80244BE7
:10A748001968204B89B20B445B0019680021196015
:10A758003023A8F800303FE0002AE9D0B9F814A067
:10A76800924528BF92461FFA8AF2104601929847EE
:10A77800019AB9F810309B1AA9F81030B9F81230BC
:10A788001344A9F81230124B1A68124B92B21344B0
:10A798005B000AF1010A1B689BB203F1005303F541
:10A7A80040534FEA6A0A5B0000215145C0D053F874
:10A7B800212020F811200131F7E700BFA819002057
:10A7C800A81C002002300020A4190020F62B00202D
:10A7D800505C004004300020B9F814309342DBF894
:10A7E800003001D8032201E012B105221A720CE0F0
:10A7F800062119726C4B19686C4B89B20B445B00CB
:10A8080019681A603023A8F80030DBF800301B7A8A
:10A8180006E0072B03D1664B1B68DB6898470823C3
:10A82800DBF800201372FBF7C3FD624B1A684BF686
:10A83800BF7313403A88D2043A8848BF83F48053E0
:10A848009004B8F8002048BF83F40053D106B8F844
:10A85800002048BF83F01003920648BF83F020030E
:10A8680043F4004343F08003524A9BB213602DE047
:10A878009A0002F1804202F5B842116889B2ADF837
:10A888000A10BDF80A1009B2002909DA106840F662
:10A898008F7101401160013B474A52F823309847B5
:10A8A800BDF80A301F067FF5D1ACA1788B0003F103
:10A8B800804303F5B84348F60F72186802401A60DF
:10A8C8003D4B03EB81039B699847BFE4228833889B
:10A8D8001340590505D54FF6FF332B60374B5B689E
:10A8E8009847228831880A40920444BF4DF6FF7386
:10A8F8002B602388324A0B40DB0452D54EF6FF7397
:10A908002B600023D370D378052B41D8DFE803F000
:10A91800030D1418222DA368294D1BB901F0B6FFA9
:10A92800062300E00523EB703BE001F0AFFF0423B2
:10A93800E3700123A36034E002232371032328E09A
:10A948002379013BDBB22371237953BB1C4B0422CF
:10A95800DA7026E01B4A13689BB243F010031360B9
:10A968000523E3700A2323711BE02379144A013B72
:10A97800DBB22371237903F0FF0093B911490C6806
:10A988004FF6EF7323400B600623D370906008E006
:10A998000623E37005E00C4B57E60C4B55E60C4BD1
:10A9A80053E605B0BDE8F08F505C0040023000204F
:10A9B800A81C0020005C0040606301080C00002017
:10A9C8008C1E0020405C0040BF5E0008655F0008E8
:10A9D800455F0008704770477047FEE7FEE7FEE7EF
:10A9E800704730B50024E3B293420DD2030F092B10
:10A9F80094BF3033373301F8143001EB440300259A
:10AA080000015D700134EEE730BD00BFF0B50124F0
:10AA1800B0FBF4F58D4201D34C43F9E70026D4B1DD
:10AA2800B0FBF4F504FB1500B4FBF1F41EB9002DDE
:10AA380001DC002CF3D1092D03F1010EEFB204DD86
:10AA4800002A14BF3725572500E030253D441D70E6
:10AA580001367346E3E71C70F0BDF0B50124B0FB86
:10AA6800F4F58D4201D34C43F9E70026D4B1B0FB8D
:10AA7800F4F504FB1500B4FBF1F41EB9002D01DC5C
:10AA8800002CF3D1092D03F1010EEFB204DD002AE9
:10AA980014BF3725572500E030253D441D70013689
:10AAA8007346E3E71C70F0BD03685A1C0260197016
:10AAB80070472DE9F843089E002B07468846144640
:10AAC80014BF4FF030094FF02009334613F8012B1B
:10AAD8000AB9254603E0002CFBDD013CF6E7002D12
:10AAE80004DD38464946C047013DF8E724EAE474E6
:10AAF8003546A01B284415F8011B11B13846C0473C
:10AB0800F7E7BDE8F883024B1868FEF787BF00BF78
:10AB1800F80F002090ED017A07EE901AB5EE407A12
:10AB2800F1EE10FA01BFF8EEE77A9FED0E7A67EEC4
:10AB3800877AB7EE007A04BFC7EE277AC0ED017AAC
:10AB480090ED017AD0ED007A30EE877A30EE670A20
:10AB5800C0EE870AE0EE807AB0EE670AC0ED007AB0
:10AB6800704700BFDB0FC94010B50278202A0346A2
:10AB780000F10100F9D0092AF7D02D2A03D10346A4
:10AB8800BFEE000A04E02B2A08BF0346B7EE000A0E
:10AB9800DFED387A1A46134612F8010BA0F130019E
:10ABA800CCB2092C0AD807EE101AB8EEC77AF2EE22
:10ABB800046AA7EEA67AF0EE477AECE72E2816D1BB
:10ABC800F2EE046A1146B0EE666A0B4611F8012BE4
:10ABD800303AD0B209280AD807EE102AB8EEC77A58
:10ABE80087EE267A66EE866A77EE877AEDE71A7838
:10ABF80002F0DF02452A35D15A782D2A02D10233D4
:10AC0800012004E02B2A14BF013302330020013B4A
:10AC1800002213F8011F3039CCB2092C03D80A24BA
:10AC280004FB0212F5E7B2F59A7F28BF4FF49A7237
:10AC38001346B7EE007A072B05D9DFED0F6A083BFC
:10AC480027EE267AF7E702F007032BB1F2EE046A43
:10AC580027EE267A013BF8E7F0EE476A20B1C7EE07
:10AC6800877A03E0F7EE006A67EEA67A20EE270AF5
:10AC780010BD00BF0000000020BCBE4C30B52DED5B
:10AC8800028B87B0B0EE408A0C220021054603A84B
:10AC980009F06FFEB5EEC08ADFED2A7AF1EE10FA00
:10ACA800CCBF38EE278A38EE678ADFED277A28EEA0
:10ACB800278A6946FDEEC87A17EE904A84EAE4705E
:10ACC800A0EBE470FBF730FA002CACBF20232D2357
:10ACD80068468DF80C3009F090FE012807D1302322
:10ACE8008DF80D308DF80E308DF80F300CE00228FD
:10ACF80005D130238DF80D308DF80E3004E003288F
:10AD080004BF30238DF80D30694603A809F058FEBA
:10AD180003A809F072FE0338C4B2224603A92846E4
:10AD280009F098FE00232B552846084909F048FEEB
:10AD380003AB2846191909F043FE284607B0BDECB5
:10AD4800028B30BD6F12033A00007A44907F0108ED
:10AD580070B5064615460846B6FBF2F414B120460F
:10AD6800FFF7F6FF05FB1464024B1B5D00F8013B7F
:10AD780070BD00BF927F01082DE9F04F814689B070
:10AD88008A4616461C4600253178002900F0DD80E9
:10AD9800252902D00136484675E07278302A08BF66
:10ADA800B278A2F1300319BFB71C4FF0000BF71CA3
:10ADB8004FF0010B092B4FF0000819D8A2F130030E
:10ADC800D9B2092905D80A2202FB083817F8012B3D
:10ADD800F4E7A2F16103052B02D8A2F1570305E0BD
:10ADE800A2F14103052B03D8A2F137030A2BEADDB0
:10ADF8006C2A31D13A78642A07F1010600F0838081
:10AE08000BD8252A3DD003D8002A00F09E80BBE746
:10AE1800582A0CD0632A19D0B6E7732A22D002D850
:10AE28006E2A37D0B0E7752A5CD0782AACD1271DB6
:10AE38002068A2F1580462424FF01001624155E0C7
:10AE48002CD9582A32D0632A2AD13E46484621783E
:10AE5800271DD04701350FE0642A64D00ED9732A24
:10AE680014D13E4623680093484651464246002383
:10AE7800FFF71FFE271D05443C4685E7252ADFD13D
:10AE88003E4648462521D04701357DE70AD86E2A37
:10AE980006D13E46236804341D6075E7002A54D065
:10AEA8003E4671E7752A26D0782AF9D1A2F15803CF
:10AEB80004F1040C5A422068CDF80CC04FF0100180
:10AEC8005A4105ABFFF7A2FDDDF80CC03E466446CB
:10AED80005AB00934846514642465B46FFF7E9FDFD
:10AEE800054451E72068271D0A21002205ABFFF71A
:10AEF800B4FD3C46ECE704F1040CCDF80CC0206826
:10AF08000A210022DDE72068002804F1040708DA96
:10AF18002D238DF8143040420DF115030A2100222B
:10AF2800E5E705ABFAE72068002804F1040C0ADA23
:10AF38002D238DF8143040420DF11503CDF80CC0C7
:10AF48000A210022BEE705ABF8E7284609B0BDE8AC
:10AF5800F08F0FB413B50B4904AB08680A4953F8CE
:10AF6800042B09680193FFF707FF0446074B18688D
:10AF7800FEF748FD0028F9D0204602B0BDE8104091
:10AF880004B070478401002080010020F80F0020E1
:10AF9800B0EEE06AF0EEC05AB4EEE56AF1EE10FAEF
:10AFA800D4BFF0EE656AF0EE466AF5EE406AF1EE5F
:10AFB80010FA0BD0B4EEE56AF1EE10FA54BFF0EED9
:10AFC800657AF0EE467AC7EEA66A01E0DFED1F6A01
:10AFD800DFED1F7A9FED1F7A9FED1F5AA6EEA77A25
:10AFE800DFED1E7AE7EE267A9FED1D7AA7EEA67AA8
:10AFF800DFED1C7AE7EE267AF4EEC65AB1EE677AF0
:10B00800DFED197AA6EEA75AF7EE007AE5EE267A72
:10B01800F1EE10FAC7EE277AC8BF9FED147AF5EE65
:10B02800C00AC8BF77EE677AF1EE10FA48BF9FED05
:10B03800107AB5EEC00A48BF77EE677AF1EE10FADB
:10B0480048BFF1EE677AB0EE670A7047000000006B
:10B0580039094E3DE3B59EBE69A2163E88FA16BE72
:10B0680045FE7FBFA7DFA8B499FB243FDB0FC93F8C
:10B07800DB0F4940FDEEC07A17EE903A2033402BA3
:10B0880043D8DFED237AB4EEE70AF1EE10FA04DDD7
:10B09800DFED207A30EE670AF3E7DFED1F7AB4EED2
:10B0A800E70AF1EE10FA04D5DFED1A7A30EE270A36
:10B0B800F3E7DFED1A7AB4EEE70AF1EE10FA04DDF1
:10B0C80030EE670A37EEC00A0AE09FED157AB4EE53
:10B0D800C70AF1EE10FA44BF30EE270A37EE400AED
:10B0E80060EE007ADFED0F6A9FED0F7AA7EEA67A81
:10B0F800DFED0E6AE7EE876A9FED0D7AA7EEA67A76
:10B1080020EE276AA6EE070A70479FED060A7047E9
:10B11800DB0F4940DB0FC940DB0F49C0DB0FC93FDC
:10B12800DB0FC9BF0000000092E741B99730083C27
:10B1380015A82ABEDFED027A30EE270A9AE700BF8B
:10B14800DB0FC93F064B1A8822EA0000904210B56F
:10B1580018801C4602D00120FEF7EAFB208810BDAB
:10B1680098190020064B1A881043904210B5188091
:10B178001C4602D00120FEF7DBFB208810BD00BF73
:10B1880098190020024A936823EA000090607047EB
:10B19800EC10002008B5104B1A780023D9B2914260
:10B1A80007D20E4951F823100968002008600133BE
:10B1B800F4E73220FEF721FA094B1B685A0309D538
:10B1C800084B9B685B0305D440F2DC50BDE808409F
:10B1D800FEF713BA08BD00BFF01C0020C01C0020F9
:10B1E800C4270020EC1000202DE9F34105F010FDE4
:10B1F800454A6C2313704FF4FA635380BE231371CE
:10B20800EF2382F8CD37002382F8CE371946164649
:10B21800F25C0133B3F5FA6F81EA0201F8D13A4BD7
:10B2280083F8CE17394B1A69120604D5384A5A6082
:10B2380002F188325A6004270020013F17F0FF0707
:10B248004FD0324B3422DA60002444B1002356F840
:10B2580004800193FAF738FF0428EED117E0FAF7D3
:10B2680033FF0428E9D1294D2B6943F002032B61F0
:10B27800284B6B612B6943F040032B61FAF724FFDD
:10B288002B69042823F002032B61DFD0D5E71F4D7B
:10B298002B6943F001032B6104F1006303F57E334E
:10B2A8001FFA88F21A80FAF70FFF042810D11A4BF8
:10B2B80023440193019B4FEA1848A3F80080FAF74A
:10B2C80003FF2B69042823F001032B6105D0B4E7A1
:10B2D8002B6923F001032B61AFE70434B4F5FA6F4F
:10B2E800B3D10A4A1369042843F08003136102D1D9
:10B2F80004F044FA10B90520FEF732FB05F072FCA1
:10B3080002B0BDE8F08100BFEC1000200020024030
:10B318002301674500F8030802F8030810B50E4C2E
:10B328002068FEF7ADF82068047A002202FB02F3D9
:10B33800193B634303F6C4135343192193FBF1F3F9
:10B34800064921F812300132072AEFD10449BDE835
:10B358001040FEF74BB800BF70100020C80F002047
:10B368002C1200202DE9F04104F008FA10B904204D
:10B37800FEF7F6FAAD4CAE4D05F04AFCAD494FF478
:10B38800FA62204609F0EAFA94F8A437022B84BF3F
:10B39800002384F8A43794F8A4274FF4CC7101FB58
:10B3A80002F3E018234400F53770286093F830035F
:10B3B80003F54A73022801FB024284BF0020187279
:10B3C80092F830339C4A13700C2202FB03439B4AC9
:10B3D80003F2A6731360A36846F209021A401AB969
:10B3E800924A43F400539360A368D80703D54FF4F7
:10B3F8000050FFF7C7FEA368590409D50820FFF7D6
:10B40800C1FE4FF40050FFF7BDFE0120FFF7BAFE62
:10B41800A3681A0706D54FF40050FFF7B3FE0120C2
:10B42800FFF7B0FEA3689B0406D54FF48030FFF702
:10B43800A9FE4020FFF7A6FE012284F80D2294F809
:10B44800DE217A4B2AB193F8E22112B1002283F867
:10B45800E2217B4B7B4E1E604FF0000C674604EBED
:10B468000C03B3F8F6E14FEA5E0101F077314FEAD9
:10B478009E0303F03333C1EB0E00C11A4FEADE031B
:10B4880003F01133CB1A03EB23131EF0010803F06A
:10B498000F324FF0FF0392FBF3F3C3EB032318BF04
:10B4A8000137A2EB030318BFFFB2012B0ADD022B01
:10B4B80040F0B980B8F1000F00F0B5801EF0BC0F65
:10B4C80000F0B1800CF1080CBCF1180FC7D1013F96
:10B4D800012F00F2A880FFF721FF302200215A48EF
:10B4E8005A4F09F046FA5A4BD5F800801F60594B5D
:10B4F800002108F17900C3F80080FEF701F8564BE7
:10B5080080F001001870554B07F128021A60544B5F
:10B5180007F1CC021A6098F80000FEF7B8FC28681A
:10B52800504B00F5C5721A6001F0D0F84E4B94F8F4
:10B53800D601DFED4E6A07F196021A6064214C4B82
:10B54800C82211FB00225A6000229A60DA601A6150
:10B558005A619A61DA6183F8202083F82120454BEB
:10B5680007F12E021A602A68434B92ED187A02F20C
:10B5780019111960414B02F289111960404B07F10A
:10B58800080119603F4B1F603F4B07F1A20119608A
:10B5980067EE266A3D4B07F1AC01B6EE007A1960FA
:10B5A80087EE267A3A490E60B4F86411181D07EE42
:10B5B800901AB4F86611F8EE677AC3ED027A07EECE
:10B5C800901A92F85C10197192F87810597194F8E1
:10B5D800E1111974F8EE677AB2F81611C3ED037A1F
:10B5E80007EE901A2B49F8EEE77A08605A6183ED66
:10B5F800077A9FED297A1A62C7EE277A02F1640169
:10B6080099612649DF62BDE8F0419FED257A67EE32
:10B61800877AC1ED007A02F1680102F211125962CB
:10B628009A6205F0DFBAFAF71BFD54E7EC10002028
:10B638005010002000F80308702700207010002028
:10B648006C2B002074120020FC0E00202C1200200D
:10B65800300F0020340F002002000020CC0600200C
:10B668004C060020400F0020CC2B0020DB0F494067
:10B67800782B002034070020F424002068090020DB
:10B688000C1E0020101E00207C080020981E0020A0
:10B6980040090020A8070020000061447808002025
:10B6A8004C3D0F4408B5FFF79FFDFFF75BFE0120F7
:10B6B800BDE80840FEF73CB92DE9F74FA44CFDF76B
:10B6C80075FF26686568A768861BF643451BC71B78
:10B6D800ED43FF43F60F8046ED0FFF0F2EB93FB93C
:10B6E800002D00F07E82B9462CE04FF0000929E0D9
:10B6F800B14627E003EB8A0BBBF8023019050ED4DC
:10B7080013F4805F1DBF934A9BF801101268924A98
:10B71800924B14BF52F82120126843F82A20BBF834
:10B728000230DA0516D49B050AD58D4B1B7813F029
:10B73800040F0CBF8B4A8C4A884B126843F82A20A6
:10B7480009F10109207B89495FFA89FA82450B686A
:10B75800D0D320E050465946854A02F0EDFF854B8C
:10B768001B88580603D550465946834A10E05907A6
:10B7780003D550465946814A0AE09A0703D55046F0
:10B7880059467F4A04E0DB07DAD57E4A50465946D7
:10B7980002F0D2FFD4E7DFF804E20093BEF90630E6
:10B7A8007822A3F57A7353434FF47A7293FBF2F33A
:10B7B80003F22B1301930022F3465FFA82FE8645BB
:10B7C80017D2009B03EB820EBEF802E01EF4806FD6
:10B7D8000DD0DFF88891019B39F822E040F2671A12
:10B7E8009E449EFBFAFC0AFB1CEE29F822E001327B
:10B7F800E3E74DB308F5C333A0336360637B544A72
:10B8080013BB9373604B1B6813F0020F0AD0DFF869
:10B8180090E19EF800E0BEF1000F03D04FF0010E5A
:10B8280082F80EE0DA0506D5584BDB781BB1A37B0E
:10B8380043F00203A3734A4B1B7813F0050F02BFB2
:10B84800A37B43F00403A37394F80EE0BEF1000F4A
:10B8580003D13F4B5B7B002B4FD094F80DC01CF0FD
:10B86800010FACF10C031DD1BCF1030F07D8DFF8B1
:10B87800E8903C4A1EF0040F08BF4A4600E0364AEA
:10B88800ACF1040CBCF1070F05D8DFF818C11EF0A5
:10B89800010F18BF6246DBB2032B0ED81EF0020F51
:10B8A8003B4B06E0DBB2032B06D82F4B2A4A1EF08F
:10B8B800020F18BF1A4600E0274A4FF0000C5FFA43
:10B8C8008CF383420DD20B6803EB8C035B881B0659
:10B8D80042BF224BD2F8009043F82C900CF1010C97
:10B8E800EDE785B1BEF1000F08D0637B184A01333C
:10B8F800DBB2142B06D1002304E025B1637B002BB7
:10B90800F3D100E05373002E50D0224AB2F902500E
:10B91800B2F90020002DB8BF6D42002A4FF0320363
:10B92800B8BF524295FBF3F592FBF3F2EDB2D3B2F6
:10B93800AB4238BF2B46184A13B192FBF3F300E031
:10B94800134643442360E37B014A6BBB01232CE08D
:10B95800C81E0020F024002088780108B20D0020BD
:10B96800F52B002090770108807701080C1C002037
:10B9780098630108981900209E630108A4630108D0
:10B98800AA630108B0630108C4270020782B0020AF
:10B9980098770108E4100020400D0300982A002041
:10B9A80020190020A07701080023D3738E4D8F4BF8
:10B9B8002D78E27BADB9002F00F00E818C4B267BF1
:10B9C8001A788C4B8C4D93F800C08C4BD3F800E060
:10B9D8000B6802F004020021D2B203EB86060F4680
:10B9E800B5E01AB9864A1A61002508E0854AFAE7DF
:10B9F8000A68AB00D6187688760604D40135EBB20F
:10BA08008342F5D3D7E7804EB6F90060192E25DDBD
:10BA180012F803E094F814C026690EF00F09E14506
:10BA28000CDCDFF8C8C19CF815C0BCEB1E1FDEBFDC
:10BA3800DFF8D8E1D6F800C043F80EC012F803E0EA
:10BA480094F816C00EF00F09E14533DBDFF89CC10E
:10BA58009CF815C0BCEB1E1F2CDC26E0193629DA31
:10BA680012F803E094F814C026690EF00F09E145B6
:10BA78000CDCDFF878C19CF817C0BCEB1E1FA2BF16
:10BA8800DFF888E1D6F800C043F80EC012F803E0EA
:10BA980094F816C00EF00F09E1450BDBDFF84CC136
:10BAA8009CF817C0BCEB1E1F04DBD6F800E0574E0D
:10BAB80043F806E0544EB6F90260192E1BDD12F861
:10BAC80003C094F814E026690CF00F09F1450CDC6A
:10BAD800DFF8189199F81590B9EB1C1FDEBFDFF855
:10BAE8002CC1D6F8009043F80C90D25C02F00F0CF1
:10BAF800F4451EDD82E7193680DA12F803C094F89F
:10BB080016E026690CF00F09F1450CDBDFF8DC9034
:10BB180099F81590B9EB1C1FDEBFDFF8F0C0D6F816
:10BB2800009043F80C90D25C02F00F0CF445FFF63D
:10BB380065AF94F817E0BEEB121FA2BF334A366810
:10BB48009E505BE75888000504D404330435B3429B
:10BB5800F8D122E04AB101EB0C0A06209AFBF0F971
:10BB680000FB19A001280DDC01E057B9012793F863
:10BB780001900EEB89003EF829A090F80290C07859
:10BB880003E01746002081468246013125F802ACC1
:10BB980085F800906870C9B2D7E7164A1378013B58
:10BBA80013F0FF0308BF06231370114B1B785B07C4
:10BBB80041BFBBF90630A3F57A7303EBC3034FF417
:10BBC8007A7243BF93FBF2F30133DBB20123104ACD
:10BBD80092FBF3F34344A36003B0BDE8F04F02F0D7
:10BBE80053B803B0BDE8F08F630E0020C81E0020D4
:10BBF800F52B0020A0000020B40D0020F024002028
:10BC08009C77010888780108E4100020B20D002014
:10BC1800400D0300012380F8453070472DE9F043BB
:10BC280090F84410002380F84430002953D02E4C5B
:10BC38002268002A52D02268052A52D12B4C20298A
:10BC48000D4628BF20256E1C27687610DFF8A8E06F
:10BC5800DEF800309BBBDFF8A4C000F132033246A7
:10BC680013F8019C13F8028C013A48EA09282CF8C9
:10BC7800048C03F102030CF1040CF1D11C4B1A687B
:10BC88001C4B92B213445B002A46D3F800C01D60D7
:10BC9800DEF800302B44CEF80030DFF864E0DEF840
:10BCA800003023F4E04323F040039BB283F03003D9
:10BCB80043F4004343F08003CEF8003000E0002254
:10BCC8008A4203D02368DB1B312BBFD9531A584251
:10BCD8005841BDE8F0830120BDE8F0831046BDE877
:10BCE800F0831846BDE8F083DC2B0020E82700200D
:10BCF800505C00400A300020E01E002084610040B3
:10BD0800045C0040002280F8452087E790F8442032
:10BD1800531C0244DBB280F8443082F8301090F8AB
:10BD280045200AB1132B00D978E77047014B5868B2
:10BD3800C0B27047E01E002001207047704770476E
:10BD480020B9034B1B6808221A82704701487047C4
:10BD5800A4190020A400002020B9034B1B68082266
:10BD68001A82704701487047A4190020A4000020D7
:10BD780021B901288CBF022000207047022070479B
:10BD880010B5094B1A68D378042B0BD8074C518A85
:10BD9800DB00234418B99B895B1A138210BD9B688A
:10BDA800581810BD002010BDA4190020A4000020C0
:10BDB800054B1968054B4A8A18B99B8D9B1A0B824B
:10BDC8007047986A10447047A4190020A400002006
:10BDD800054B1968054B4A8A18B99B8E9B1A0B822A
:10BDE8007047186B10447047A4190020A400002065
:10BDF800074B1B681B7803F07F03212B06D100F04B
:10BE0800DF00022814BF022000207047022070477C
:10BE1800A4190020212810B508D1114B1B681B78E4
:10BE280003F07F03212B10D0022010BD2028FBD166
:10BE38000B4B0C4A1B681B78107003F07F03212BF7
:10BE4800094B18BF00230BB9EEE7084B044A1268E8
:10BE580000249361548220469847204610BD00BFB5
:10BE6800A4190020F82B002049BD000861BD000876
:10BE7800704707EE900AF8EEE77ADFED0C6A9FED5F
:10BE88000C0AF5EEC07AF1EE10FAD4BFB1EE677A7B
:10BE9800C7EEA67A08B5D8BFC7EE267A27EE800A7D
:10BEA800FFF748F9034B83ED000A08BD8096184B4D
:10BEB80035FA8E3CF8000020F7B51C4B5A681D4631
:10BEC8000AB95C6800E00124187A0021CAB2A242CB
:10BED80001F1010107D202AE2F1816443A44527AF2
:10BEE80006F8042CF2E75A68121B5A601A7A5D6841
:10BEF80022441A729DB903204021FAF737FA0C4AF6
:10BF0800136823F4804323F070039BB283F44053F7
:10BF180043F4004343F080031360044B1D72002C6C
:10BF2800CBD09DF8040003B0F0BD00BFE01E002098
:10BF38000C5C0040F8B5A84B1B680546187818B18A
:10BF4800012800F0838106E3242DA44C0CD006D8E8
:10BF58000A2D00F0EC800D2D00F0E9805CE12A2D1F
:10BF680009D02C2D07D057E184F8490084F84A00FD
:10BF780084F84B0066E19A4B94F84A1094F849709B
:10BF8800964A0020585447BB197882F84C704729C4
:10BF980023D15978502920D19978472908D1D978BF
:10BFA800472905D11979412902D1012182F84C107C
:10BFB80099788B4A522903D1D1784D2900F0CD8246
:10BFC8009978874A472908D1D178532905D1127918
:10BFD800562A04BF032284F84C2094F84C207F4E44
:10BFE800022A3BD0032A50D0012A40F08A80BA1E88
:10BFF800072A00F28680DFE802F004080F131A25EA
:10C00800842B04F067F920657BE01B78532B78D1EB
:10C01800236D5B42236574E004F05CF9606570E0B1
:10C028001B78572B6DD1636D5B42636569E01B78A4
:10C03800302B6C4B1A788CBF42F0020222F00202BD
:10C048001A705EE0002004F0A5F984F8580058E062
:10C05800002004F09FF9A4F85A0052E0072F07D0F7
:10C06800082F4ED1012004F095F9A6F85E0048E0AB
:10C07800012004F08FF941F2184358434FF47A73C2
:10C08800B0FBF3F0A6F85C003BE0022F07D0032FCB
:10C098000BD1002004F07EF9534B187031E00020DA
:10C0A80004F078F986F860002BE02AD93A1F92103C
:10C0B80096F860300132D2B2013B02EB8303DBB267
:10C0C800102B1ED8F91EC2F1010201EB8202D2B276
:10C0D800012A0BD0042A11D100205E1E04F05AF95F
:10C0E800424B9855424B00229A5507E05E1E414A42
:10C0F8000020935504F04EF93F4B9855636E013379
:10C108006366364B2A2D18BF93F84B2007F10107B9
:10C118004FF000000CBF0122554084F8497084F8A4
:10C128004A000CBF83F8682083F84B508AE094F8E3
:10C13800680000284CD0314B13F8012D30495A7053
:10C148008B42F9D1264A254D13785278402B85BF6A
:10C15800373B1B011B01DBB298BF03F0F003402AF9
:10C168008CBF373A303AD2B2134494F84B20DBB242
:10C178009A422AD121230B7095F84C00EB6E204A85
:10C1880001330128EB660CD0022820D172231370EA
:10C198001C4BB5F85C201A801B4BB5F85E201A8042
:10C1A80015E0672313700F4B1B789F0710D5174BAB
:10C1B8002A6D1A606A6D5A60154B95F858201A70E6
:10C1C800144BB5F85A201A8002E03F230B70002068
:10C1D800002384F8683035E0C4060020E01E002003
:10C1E800F0270020D41800208C100020BD1000205B
:10C1F800AD1000208D1000209D100020200300208D
:10C208000C030020D618002074100020DC18002031
:10C21800DA180020D818002094F84A3094F86800FA
:10C228000E2B9FBFB14A591C82F84A10B04A98BFDA
:10C23800D554AE4A28B992F84B305D4082F84B503D
:10C2480000E00020003018BF0120F8BDA74B93F88C
:10C2580070100022082900F27E81DFE801F0050C49
:10C26800101A2B3C63828F00B52D40F0748183F83F
:10C278007120012253E0622D08BF02224FE0032201
:10C2880083F8702083F8725083F8735083F87450E1
:10C2980061E1042283F8702093F8732093F87410F6
:10C2A80083F875502A44D2B283F873200A4483F87D
:10C2B800742050E1052283F8702093F8732093F8D6
:10C2C8007410A3F876502A44D2B283F873200A4433
:10C2D80083F874203FE1062283F8702093F87320D6
:10C2E80093F874102A44D2B283F873200A4483F86E
:10C2F8007420B3F8762002EB0525ADB2B5F5AC7F16
:10C3080088BF7A4AA3F8765084BF012182F8711059
:10C318000022A3F87820002D40F01D81072283F821
:10C32800702018E193F8732093F874102A44D2B25D
:10C3380083F873200A4483F87420B3F87820B2F5A0
:10C34800AC7F3CBF6949891802F1010238BF81F806
:10C358007C50B3F8761092B29142A3F87820DDD9D8
:10C36800F9E0082283F8702093F87330AB4200F0AC
:10C37800F2805E4B012283F871200FE05D4C83F858
:10C38800702014F8012D62705B4A9442F9D193F839
:10C398007410564AA94206D03F232370574A53685F
:10C3A80001335360D7E0D16E92F871000131D16644
:10C3B80010B13E232370CEE02121217092F8751030
:10C3C800062944D004D8022907D0032926D0F8BD6D
:10C3D80012295CD030296CD0F8BD50212170484911
:10C3E800D2F880404C60D2F884400C60D2F88C10AF
:10C3F8004FF47A7491FBF4F1424C218092F8D411F5
:10C40800414A19B1117841F0020102E0117821F096
:10C4180002011170012283F8D5218EE05321217089
:10C4280092F88110CE0705D592F88020D51E6A4271
:10C438006A4100E0024602F0010183F8D411002AA3
:10C448007BD131490A7822F002020A7075E04F2147
:10C45800217092F88710CC0705D592F88620D11E56
:10C468004A424A4100E0024602F0010183F8D41131
:10C4780022B925490A7822F002020A70234A93F861
:10C48800AB101170224AB3F8A810118055E056215C
:10C4980021702049D2F890400C8042F21074D2F8F2
:10C4A800941091FBF4F11C4C2180012182F8D611E3
:10C4B80043E04921217092F88010184A102988BF5A
:10C4C80010211170164914780022A24232D2154D5B
:10C4D8000E7A5655144D4E7A5655144DCE7A5655F9
:10C4E800134D11F80C6F56550132EEE7E01E00208F
:10C4F800F0270020200300200C030020A4060020C1
:10C50800DC180020D8180020D4180020DA180020E1
:10C5180002010020D6180020741000208C10002082
:10C528005C1F00208D1000209D100020AD10002001
:10C53800BD1000205A6E01325A6693F8D5310B4A65
:10C548009BB192F8D63183B1002182F8D51182F8D7
:10C55800D6111846F8BD0020F8BD1279432A7FF499
:10C568002FAD022284F84C202AE5F8BDE01E0020F9
:10C578000449054B0968187000225A6199611A77B5
:10C58800704700BFE8270020A406002010B5121A43
:10C5980007EE902A5B1A2DED028BF8EEE78A07EE7C
:10C5A800903A184B059CB8EEE78AD3ED007A28EE4E
:10C5B800278A28EE080AA8EEA80A08F0C1FCDFEDD1
:10C5C800127A049B20EE270AF0EE480ABCEEC00A55
:10C5D80083ED000AB1EE680AFEF7DAFCDFED0B7AAC
:10C5E8009FED0B7AE0EE077ABDEC028BFDEEE77A61
:10C5F80017EE903A002BBCBF03F50C43A033236021
:10C6080010BD00BFF80000202C7D8E3F00A00C4616
:10C61800A00CB34544F25063984203DDA0F50C40EA
:10C62800A0387047034B9842BCBF00F50C40A030BF
:10C63800704700BFB0B9FFFF73B51A4C0368236099
:10C648000B686360184D0068184EFFF712FC184B12
:10C65800009395E8030094E80C000196FFF796FF15
:10C66800144B32681A606868636813491B1A07EE2E
:10C67800903A124B286893ED007A23681B1A0B60D6
:10C688000F4BF8EEE77A1A600E4B67EE877A1B6855
:10C69800FDEEE77ADA880C4BC1ED017A1A8002B018
:10C6A80070BD00BF10270020DC1800201C270020C8
:10C6B800182700205827002020270020F8000020F5
:10C6C80050270020400F00204C2700204279DFED42
:10C6D8002A5A2A4B9FED2A5A07EE902AF8EE677AD3
:10C6E800C27BC7EEA57AB2EE047AC3ED007A07EEF4
:10C6F800902AF8EE677A234ADA60C7EEA57AC3ED86
:10C70800017A8179204B07EE901AF8EE677A017C5E
:10C71800DA60C7EE877AC3ED007A07EE901A817E59
:10C7280006EE101AF8EE677AB8EE466AC7EEA57AF2
:10C7380086EE056AC3ED017A83ED026AC179134B6F
:10C7480006EE901A417CDA60F8EE666AC6EE876AF1
:10C7580007EE101AC17EC3ED006A07EE901AB8EE14
:10C76800477AF8EE677A87EE257AC7EE857A83ED01
:10C77800017AC3ED027A70470000C84228270020DA
:10C7880000007A440000FA44382700205C27002083
:10C7980010B50C4C23789B0713D50B4B1B78042B37
:10C7A8000FD90A4A0A4B106852685A601860FFF796
:10C7B80060FB084B1A88084B1A80237843F0010362
:10C7C800237010BDD4180020DA180020DC180020CF
:10C7D80078100020E01000206C2700201C4B1B68FC
:10C7E8001B0307B530D51B4A1B4BD2ED007A1B78CB
:10C7F8008DF80030B2EE047A67EE877A174B9FED1A
:10C80800187A1B788DF80130FCEEE77A0A2017EECB
:10C81800903AD2ED017A8DF8023067EE877A694650
:10C82800FCEEE77A17EE903AD2ED027A8DF80330F3
:10C83800FCEEE77A17EE903A8DF80430094B1B7836
:10C848008DF80530FBF792FB03B05DF804FB00BFE1
:10C85800C4270020D8270020B6270020D42700208E
:10C8680000007A44BA270020054A137883F00103B0
:10C878001370044A00231360034A1360AEE700BF35
:10C88800BA270020D0270020CC2700200A4B10B55B
:10C8980019684FF6FB720A401A60084A927A1C46D9
:10C8A800074B0AB1052200E001221A6003F0DCF907
:10C8B8004FF43643236010BD405C00408C1C0020C0
:10C8C800DC2B002010F80A3C0133DBB20A2B84BFB2
:10C8D80010F8131C044A00F80A3C82BF002322F80F
:10C8E800113000F80A3C7047BC2A0020334A136C08
:10C8F80090681944081A40F68C23984270B513467C
:10C908009160D06051603BD9127893F945108A4202
:10C9180010460BD1111F082908D893F8461018297A
:10C9280001D8013103E083F8442002E0002183F8B4
:10C93800461093F944402149A24219D191F8474041
:10C94800B4B10C310024944206DA1D4D51F8046F3D
:10C9580025F814600134F6E70C2805D0184900249E
:10C9680021F810400130F7E71648017801310170CD
:10C9780083F84520002201211A7083F8471070BD02
:10C9880092F84710C9B1A0F2EF2440F2DA518C4274
:10C9980008D811780B2905D80B1D0131117042F800
:10C9A800230070BD002283F84720074B03F13002B3
:10C9B800002143F8041F9342FAD170BDB001002052
:10C9C800BC2A002074060020BC010020024A136C17
:10C9D8000133194411647047B0010020024B53F829
:10C9E80020301B6819607047C01C0020064B53F8A4
:10C9F80020301A681B89A1F57A7159434FF47A736C
:10CA080091FBF3F111607047C01C0020F0B5046D74
:10CA18008668236823F0010323608379054613F0B1
:10CA2800020F40790CBF4FF0000E4FF4005E13F078
:10CA3800040F14BF4FF48067002710F0010F14BFD4
:10CA4800042100218307206820F00100206062682B
:10CA580022F440524EEA02026260226822F4B05385
:10CA680023F00C0348BF41F008013B430B4323600C
:10CA7800A36895B023F44073A3606846F9F724FED1
:10CA8800284B9C4201D10C9B0EE0274B9C4201D1C4
:10CA98000D9B09E0254B9C4201D10E9B04E0244BE1
:10CAA8009C420CBF0F9B109B2268A879170448BFB3
:10CAB8005B00B3FBF6F206FB1233B3EB560F2368A9
:10CAC80028BF01321E0441BF4FF6F073C2F3420182
:10CAD800134041EA03026B7992B213F0020FA2816C
:10CAE80000F0010114BF4FF400320022DC0748BFF8
:10CAF80042F480322B6D11B159680A4302E059683B
:10CB080021EA02025A609A6801074CBF42F0080203
:10CB180022F008029A601A6842F001021A6015B001
:10CB2800F0BD00BF0038014000440040004800400C
:10CB3800004C00402DE9F0471E46A14B8CB09842AE
:10CB4800894690469DF8507040F085809D4B9E4ADE
:10CB58001A609E4A5A6102F580729A614FF4807297
:10CB6800DA601A619A4A1A63143A5A63A2F548427B
:10CB7800203ADA6404329A64C3F808801865954B41
:10CB88009A6942F480429A615A6942F001025A61F4
:10CB980002238DF80830032317F0010A8DF80930B5
:10CBA8004FF000038DF80A3014BF022301233A071F
:10CBB8008DF80B3019D54FF090444FF4007501955E
:10CBC8008AF001038DF80A30636A23F0F003636288
:10CBD800636A43F070036362204601A9F9F7EAFE2D
:10CBE800BAF1000F27D1A56125E0B30710D50CA92C
:10CBF8004FF4007341F82C3D4FF09040436A23F006
:10CC0800F0034362436A43F070034362F9F7D2FECC
:10CC1800F50710D50CA94FF4806341F82C3D4FF06F
:10CC28009040436A23F470634362436A43F4E063C9
:10CC38004362F9F7BFFE0E238DF80030002201236E
:10CC480068468DF801308DF802208DF803305D4C70
:10CC580003F068F973E0604B984240F005815F4B40
:10CC6800594A1A604FF48072DA601A615C4A5A6154
:10CC780002F580729A61574AC3F808801865D3692B
:10CC880043F40033D36102238DF80830032317F0EF
:10CC9800010A8DF809304FF000038DF80A3014BFEF
:10CCA800022301233C078DF80B3017D54D4C202566
:10CCB80001958AF001038DF80A30236A23F4700382
:10CCC8002362236A43F4E0032362204601A9F9F7AB
:10CCD80071FEBAF1000F23D1A56121E0B0070ED58E
:10CCE8000CA9202341F82C3D3E48036A23F4700325
:10CCF8000362036A43F4E0030362F9F75BFEF1079A
:10CD08000ED50CA9402341F82C3D3648036A23F080
:10CD180070630362036A43F0E0630362F9F74AFE53
:10CD280026238DF800300022012368468DF8013053
:10CD38008DF802208DF8033003F0F4F8274CC4F87E
:10CD48002C900025012384F844302562E561A56212
:10CD580065626671C4F80880A7712046FFF756FE21
:10CD6800F20748D5236B002B3ED001A8F9F7CAFB80
:10CD7800E36C01934FF480530A9380230693E3688E
:10CD8800ADF8103020230993206B636902930B954B
:10CD98000595079508950395F9F7DFFB01A9206B21
:10CDA800F9F7BDFB236B216D1A6842F001021A6086
:10CDB8008A6842F040028A605B689BB223641AE08A
:10CDC800003801405026002058640108B82000208F
:10CDD800580002400010024000440040FC2500209A
:10CDE800B8220020000C0048236D20221A621A681D
:10CDF80042F020021A60B3072FD5636B43B301A832
:10CE0800F9F780FBA36C01934FF480530A938023B6
:10CE180006932369ADF8103000251023606B039347
:10CE28000B950595079508950995F9F796FB606B9D
:10CE380001A9F9F774FB636B1A6842F002021A60E1
:10CE4800226D5D605D60936843F08003936004E049
:10CE5800226D136843F080031360226D136843F05A
:10CE680001031360204600E000200CB0BDE8F08705
:10CE78003D4B1B78012B30B514BF00240324B1B9F6
:10CE8800036A23F0010303628169036A21F0F30155
:10CE980023F00A0341F0010142F001021A4341EA7A
:10CEA800041181610262836923F00C031BE00429E9
:10CEB8001DD1016A4FF6EF730B4003628169056A61
:10CEC800120121F473414FF65F7342F0100241F4EE
:10CED80080712B4092B2134341EA043181610362AD
:10CEE800836923F4406383618369836130BD0829C2
:10CEF800016A1AD14FF6FF630B400362C169036AE6
:10CF08009BB289B223F4206343F4807321F0F301C8
:10CF180043EA022241F0010192B241EA0411C161DF
:10CF28000262C2694FF6F37319E04EF6FF730B40C5
:10CF38000362C369056A40F6FF41194045F6FF736D
:10CF48002B4043F4805343EA023241F4807192B299
:10CF580041EA0431C1610262C2694FF2FF331340F2
:10CF6800C361C369C36130BDAC01002038B510F896
:10CF78000E2C50F8043C044652B9012200F80E2C3D
:10CF880020F80C1C997A18680222BDE838406FE72F
:10CF980030F80C2C20F80A1C891A89B220F8081CD1
:10CFA800074A10F80F0C002522F8101004F80E5C40
:10CFB8001868997A2A46FFF75BFF04F8065C38BDC3
:10CFC800BC2A0020044B53F820301BB107289CBF13
:10CFD8001B681960704700BFD802002038B50024CC
:10CFE8000B4D6059254402F0E5F9696811B109480B
:10CFF800FDF7AFFFA96811B10748FDF7AAFF074879
:10D00800103402F0D7F9B4F5E07FE9D138BD00BF9C
:10D0180078640108C97F0108CF7F01085189010898
:10D0280070B50546284607F0E8FC064658B91A4B7D
:10D038001A485A791A4B03EB8203BDE87040D3F8BB
:10D04800BC11FDF786BF28461649324607F0DEFCBC
:10D0580060B91548154C02F0ADF954F8041F19B120
:10D068001348FDF776FFF8E7124805E00024124B55
:10D0780053F8241021B91148BDE8704002F09AB95C
:10D088002846324607F0C2FC01340028EFD1024B93
:10D098000B4D5C71C6E700BFEC100020D57F01087E
:10D0A80078640108E17F0108E67F01083466010819
:10D0B800F97F01085189010838660108E27E0108F4
:10D0C800D77B0108F0B585B0044607F096FC082820
:10D0D80026D1621EE01D1F4912F8013F0968194454
:10D0E800497801F00301022908BF203B82421370EE
:10D0F800F1D1254604F1080715F8016B16483146A9
:10D1080007F06DFC20B12846314607F068FC10B1E5
:10D11800FBF7DAFB1CE0BD42EED12046F8F7E6FF4C
:10D128000E4802F047F900230D4A1A4404A992F860
:10D1380088210A440849595C02F80C1C0133082B61
:10D14800F2D1002307488DF80C3001A9FDF701FF43
:10D1580005B0F0BD10010020167D0108FD7F010813
:10D16800EC100020F5870108234B244C1D6820682B
:10D1780080B5FCF7BBF82846FCF7B8F82068417979
:10D188008B0704D4036841F002015B6998471C4B84
:10D198004FF488521A854FF488421A852068FCF7A4
:10D1A8003AFCA0B1164E4FF48853B361134B18687C
:10D1B800FCF72EFC0746FEF7BDFE08B101F086FB22
:10D1C80028463946FCF72AFC4FF48853338528460D
:10D1D800FCF721FC0028E1D0094ED4F800804FF478
:10D1E8008847B7612846FCF713FC01464046FCF720
:10D1F80015FC3785D2E700BF8C270020B824002013
:10D20800001000482DE9F047054607F0F6FB314EBF
:10D218000446D6F8088090B92F4802F0CBF82F4B77
:10D2280053F8241049B10123A34013EA080F02D090
:10D238002B48FDF78EFE0134F1E72A4822E0284604
:10D248002949224607F0E2FB58B92848284C02F041
:10D25800B1F854F8041F0029EFD02148FDF779FEF2
:10D26800F7E72B782D2B03BF013504F1FF344FF07E
:10D27800010A4FF0000A4FF00009184B53F82970C3
:10D2880027B91C48BDE8F04702F094B8284639464B
:10D29800224607F0BBFBC8B9012000FA09F0830554
:10D2A80001D51548EEE7BAF1000F03D0FDF76AFF84
:10D2B800124803E040EA0800B060114802F07AF82A
:10D2C80039461048BDE8F047FDF743BE09F10109AA
:10D2D800D3E700BFEC10002003800108A066010816
:10D2E800F97F010851890108E17F01080D800108D3
:10D2F8009C660108E27E0108198001082780010860
:10D3080030800108F487010810B5084802F052F887
:10D31800074B00241C715C63064B1C70FCF70EFD68
:10D3280002F0FAF9044B1C6010BD00BF38800108F8
:10D33800B8240020F92B00208C27002070B5064661
:10D3480000240B4BE518AA8816420AD0E158094870
:10D35800FDF7FFFD2846002101F0B9FF064802F05D
:10D3680029F8143440F644439C42EAD170BD00BF0A
:10D37800286A01086480010851890108F0B5047819
:10D388008BB005460CB1002436E04B4B19680E23D0
:10D3980003FB041101F58C70B1F91D51B1F9192184
:10D3A800B1F91B31009591F82051019591F821515F
:10D3B800029590F90700039001F590713F4891F9A3
:10D3C8000210049121460134FDF7C3FD082CDCD17D
:10D3D80070E02D2B14D1072C1BDC284607F064FBCA
:10D3E8000AAB661C03EB440424F8100C15F8013F43
:10D3F800303B092BFAD934462B78002BE9D104E0CD
:10D40800A3F13002092A09D8E5E7082CBDF818204D
:10D4180009D00BB0BDE8F040FBF756BA202BF8D185
:10D4280001352646E7E7072AF3D8BDF81A00224B4C
:10D43800A0F2EE2189B240F2DC55A9421B68E8D877
:10D44800BDF81C10A1F2EE24A4B2AC42E1D8BDF89C
:10D458001E6004B237B2A742DBDB0DB2AF42D8DCA4
:10D46800A542D6DBBDF8247007F16404A4B2C82C29
:10D47800CFD8BDF826E00FFA8EF4112CC9DCBDF820
:10D488002050B42DC5D8BDF82240B42CC1D812B252
:10D498004FF00E0C0CFB0233A3F81901A3F81B1173
:10D4A800A3F81D6183F8205183F8214183F81F7187
:10D4B80083F822E10BB0F0BD501000206E80010807
:10D4C800F0B504468FB0204607F097FAC5B225BBE1
:10D4D800AF48B04C01F06EFF94F8D21009B9AE48CD
:10D4E80054E049B294F8D02094F8D130009194F8DF
:10D4F800D310019194F9D410029194F9D5100391A5
:10D5080094F8D6100491A54829460135FDF721FD68
:10D51800102D04F10704DFD1E1E72046A0490522D8
:10D5280007F074FA0546B8B929469E48702207F0F4
:10D5380020FA9D4B196828460E2303FB001301307F
:10D548000022082883F8232183F8242183F8252141
:10D5580083F82621F0D119E120469449042207F0E6
:10D5680055FA05462046002D4AD1202107F037FA02
:10D57800002800F00B81461C304607F03EFA2C4686
:10D5880007468B4B53F824502DB98A480FB0BDE895
:10D59800F040FDF7DEBC30462946FAB207F036FA0D
:10D5A80001340028EDD17B4A02F1700116460023B0
:10D5B80082F8D63082F8D23082F8D13082F8D03072
:10D5C80007328A42F3D17C4901EBC40191F88022E9
:10D5D800934210DAD1F88472C3EBC302B0183A440C
:10D5E80000F1D0011768C0F8D070908888809279CF
:10D5F8008A710133E7E729467048FDF7AAFC96E0EF
:10D608006F49072207F002FA05462046002D4AD145
:10D61800202107F0E4F9064607F0EFF9C4B274BB1D
:10D628006848FDF796FC214667480134FDF791FCF0
:10D638000E2CF8D15848FDF78CFC0024634821468D
:10D64800FDF787FC0025584A614811680E2202FB45
:10D6580004120123D2F823215E49AB4013425E4BEA
:10D6680005F1010508BF1946FDF773FC0E2DEAD137
:10D6780049480134FDF76DFC082CDFD186E03046BF
:10D68800564907F015FA2C46002852D0022C55D0DE
:10D6980007F00AFA06AB514943F82400002007F0C6
:10D6A80007FA0134F0E74D4907F002FA002460B1A7
:10D6B800082C3ED007F0F8F906AB484943F8240097
:10D6C800002007F0F5F90134F1E7082C31D1069B69
:10D6D8000F2B2ED8DDF81CE0BEF1070F29D8089FC4
:10D6E8000D2F26D8099E06F16402C82A21D80A9D62
:10D6F800FF2D1ED80B9864281BD80C99642918D8BC
:10D70800884216DA0D9C032C13D8224AC3EBC303B4
:10D71800134483F8D0E083F8D17083F8D26083F89B
:10D72800D35083F8D40083F8D51083F8D6402C4C16
:10D73800C9E60FB0BDE8F040FBF7C6B8069B072B5B
:10D7480020D807990D291DD80278722A0DD06E2A83
:10D7580018D1154A12680E2000FB032301228A40C3
:10D76800D3F8231121EA020209E00F4A12680E20B9
:10D7780000FB032301228A40D3F823110A43C3F88C
:10D78800232101E0FBF7A0F80D4C9CE60FB0F0BD9B
:10D7980096800108EC10002051890108C180010819
:10D7A800B27E0108BC11002050100020DD7E010867
:10D7B80038660108E27E010878640108F17E0108F4
:10D7C8008E800108D37F0108DD8001080D880108DB
:10D7D800E2800108AA8B0108648C0108E680010830
:10D7E800D77B01082DE9F743047805468CB9324DFB
:10D7F80095F89F12B5F89C2295F89E322F48009113
:10D8080021460134FDF7A5FB102C05F10405EFD1E5
:10D818004EE007F049F90F28044636DC2846202157
:10D8280007F0DDF8264EE4B2D6F83880451CA4008F
:10D838000027284607F038F95FFA87F9B9F1010F90
:10D8480083B208D0B9F1020F0BD0B3F5B47F24D25C
:10D85800B26B13530AE0FF2B1FD8B36B23449870A5
:10D8680004E0FF2B19D8B36B2344D87028462C2129
:10D8780007F0B5F8054608B1013502E0B9F1020F25
:10D888000BD10137032FD4D112E00E4800210F220B
:10D8980003B0BDE8F043FAF794BF08EB0400002199
:10D8A800042207F066F803B0BDE8F043FBF70CB8B4
:10D8B80003B0BDE8F08300BFEC100020E880010849
:10D8C800B8240020707E01082DE9F0412DED048B6D
:10D8D800B1498AB0044607F055F8B04900282046F7
:10D8E8000CBF0126072607F04DF8AD490028204651
:10D8F80008BF022607F046F8002808BF0426F107EB
:10D9080040F1F080A748A84C01F054FD002001F038
:10D9180057FBA64801F04EFDA54801F04BFD627982
:10D92800A44BA54803EB82032546D3F8BC11FDF7A9
:10D9380010FBA248FDF70DFB4FF00008274695EDB8
:10D94800048AB5EE408AF1EE10FA04D19C48FDF73E
:10D9580000FB002570E09B48D5ED059A95ED069AE9
:10D96800D5ED078A4146FDF7F4FAB5EEC08AF1EE27
:10D9780010FA02D5202001F015FDB0EE480A06A8DD
:10D98800FDF77CF901469048FDF7E3FAF5EEC09AF9
:10D99800F1EE10FA02D5202001F004FDB0EE690A7C
:10D9A80006A8FDF76BF901468748FDF7D2FAB5EEF0
:10D9B800C09AF1EE10FA02D5202001F0F3FCB0EE87
:10D9C800490A06A8FDF75AF901467F48FDF7C1FA4A
:10D9D800F5EEC08AF1EE10FA02D5202001F0E2FC43
:10D9E800B0EE680A06A8FDF749F908F101080146F2
:10D9F8007648FDF7AEFAB8F10C0F05F110059ED187
:10DA0800A4E749B294F8D02094F8D130009194F862
:10DA1800D310019194F9D410029194F9D51003917F
:10DA280094F8D61004916A4829460135FDF791FA11
:10DA3800102D04F1070403D094F8D2100029E0D186
:10DA48006448654C01F0B6FCD7F8088054F8041F08
:10DA580019B16248FDF77DFAF8E70D46604B53F8B7
:10DA6800254054B10123AB4013EA080F03D05D48A9
:10DA78002146FDF76EFA0135F0E75B4801F09AFCA4
:10DA880021467B180AAA93F888311344574A8A5CBE
:10DA980003F8102C01310829F3D1002306A95448B2
:10DAA8008DF82030FDF755FA524801F083FC5248B2
:10DAB800FBF740FA514801F07DFC4F48FAF70AFF9E
:10DAC8004F4801F077FC4C48FFF78CFE4D48FDF7B6
:10DAD80040FA4020FFF732FC4B4801F06BFC464807
:10DAE800FBF7CEFAB20739D5484801F063FC48483D
:10DAF80001F060FC404801F0A3FA464801F05AFCE6
:10DB08003D48FAF76BFE444801F054FC3A48FBF7ED
:10DB180063F94248FDF71DFA3748FAF7E7FF40482E
:10DB280001F048FC3448FFF729FC00270E257D4307
:10DB380000243C4AD26B2A440123D2F80A20A3408D
:10DB480013421ED101340E2CF3D10137082FEDD129
:10DB58002C48FDF7FEF98020FFF7F0FB730716D578
:10DB6800314801F027FC314801F024FC224801F03B
:10DB780041FA2448FDF7EDF94FF48070FFF7DEFB1A
:10DB880005E0394622462A48FDF7E3F9DAE70AB004
:10DB9800BDEC048BBDE8F081FC80010837850108E5
:10DBA8000381010809810108EC1000201781010890
:10DBB800298101087864010835810108408101083C
:10DBC8004D8101085A810108D27F0108F5870108B3
:10DBD80072810108628101089C660108918101082F
:10DBE800A06601089F810108AC810108167D010823
:10DBF800B8810108C1810108D77B0108D0810108DB
:10DC0800DC81010851890108EA810108F7810108CE
:10DC18000A8201081882010822820108318201085B
:10DC28003F820108B82400204B8201085C82010869
:10DC38006E820108054B98420CBF054A054A1388B5
:10DC480001339BB213800020704700BF005400408E
:10DC58001010002012100020084A13689B050BD5ED
:10DC6800074B00211970074908684FF6FE730340F7
:10DC78000B604FF400735360704700BF0000024010
:10DC8800F42B0020300002402DE9F047664D2B6848
:10DC980066490A78581C02F0FF068E460AB1034608
:10DCA800F6E72B60687BAB6895F80C80AA7B374653
:10DCB80039B2202900F09B80DFF880C10CEB81038A
:10DCC8003CF82110DC789B78C3F1FF039BB2002B52
:10DCD80065D0C3F1FF0363434FF03C0C1B12B1FB4B
:10DCE800FCF9B9F1050F5DD8DFE809F0030B1A2933
:10DCF8003A4AE01ADAB24143B1FBFCF01044C0B230
:10DD080051E0B1FBFCF00CFB101189B2DAB2C1F1A1
:10DD18003C01E31A4B432046B3FBFCFC94442CE043
:10DD2800B1FBFCF00CFB10115FFA83F8E21A89B220
:10DD38004A43B2FBFCF24244D2B2204632E0B1FB85
:10DD4800FCF90CFB191189B25FFA83F8E01AC1F1EA
:10DD58003C014843B0FBFCF04044C0B2224621E0FD
:10DD6800B1FBFCF80CFB1811D8B289B2E31A01FB1D
:10DD780003F2B2FBFCFC224684445FFA8CF412E006
:10DD8800B1FBFCF80CFB181189B2D8B2C1F13C0107
:10DD9800E31A4B43B3FBFCF20244D2B203E022463F
:10DDA800204600E044464FEA042C4CEA004C4CEA7A
:10DDB800020C172306F117014FF0010808FA03F8BF
:10DDC800C91A18EA0C0F89B2DFF8748014BF4FF033
:10DDD80011094FF0090913F1FF3308F80190E9D24E
:10DDE80018360137B6B2BFB2114BA04660E7AA7326
:10DDF800AB60104AE98001238EF800300E4985F89F
:10DE08000C8040F22A336873AE80536000234B6263
:10DE18000B889BB243F001030B80136843F00103A6
:10DE28001360BDE8F08700BFF8240020F42B002021
:10DE3800042500203000024000440140B20D0020BB
:10DE48002103002073B506460D46002401232A88C5
:10DE5800A34013421AD0AA78009302F003038DF866
:10DE68000430EB78022B03D0032B0CBF03230123D0
:10DE78008DF805303046C2F301136946C2F38102BA
:10DE88008DF806308DF80720F8F794FD0134102C32
:10DE9800DCD102B070BD2DE9F04F734EF57B07461B
:10DEA8000C4687B011469A4600686B1C914622467C
:10DEB8004FF0020BF37300F041FB3B897868ADF833
:10DEC800043001A98DF806B08DF807B0FFF7BAFF46
:10DED8000023ADF80A30ADF81230ADF816307023D3
:10DEE8000193BA7A3C68CDF80CA0012306F110081A
:10DEF8002D01ADF808304FF48073A844ADF810B088
:10DF0800ADF814300C2A7ED8DFE802F0077D7D7D5D
:10DF18000F7D7D7D387D7D7D5E00204601A9F8F767
:10DF280095FBA36943F0080326E0236A4F4823F0D2
:10DF380010032362236A6168A26922F0807222F4C6
:10DF4800E642844242F4E04206D000F50060844292
:10DF580002D043F0300307E023F0E00321F44061EE
:10DF680043F0300341F480616160A261C4F838A0D5
:10DF78002362A36943F40063A36144E0236A3B4836
:10DF880023F480732362226A6168E369844223F080
:10DF9800730343F0700306D000F50060844202D09A
:10DFA80042F4407207E022F4606221F4405142F4E6
:10DFB800407241F480516160E361C4F83CA0226280
:10DFC800E36943F008031DE0236A284823F48053DB
:10DFD8002362226A6168E369844223F4E64343F4D6
:10DFE800E04342F4405203D000F50060844201D17E
:10DFF80041F480416160E361C4F840A02262E369B2
:10E0080043F40063E3613A7B3B681AB15A6C42F40B
:10E0180000425A641A8892B242F001021A80BA7A0F
:10E028000C2A18D8DFE802F0071717170B1717176D
:10E038000F1717171300721903F134010AE0721948
:10E0480003F1380106E0721903F13C0102E072198C
:10E0580003F14001116135444046A5F818906B6101
:10E0680007B0BDE8F08F00BFF8240020002C014065
:10E07800F8B53A4E3A4C4000C7B24FF420453068E4
:10E08800C4F8D050D0F818E01EF4004F05D0AE46C2
:10E09800013DBEF1000FF5D116E0D0F804E0314D96
:10E0A8000EEA050545F490353D4345604FF420459B
:10E0B800C4F8D050D0F818E01EF0020F2DD1AE46AB
:10E0C800013DBEF1000FF5D1C4F8D0501FE029463C
:10E0D800013D0029F8D081694906F8D5C4F8D05027
:10E0E80020494568294041F0007141F4105141EA46
:10E0F8000241394341604FF42041A2B1306885693B
:10E108006D071ED411F1FF31F9D2C4F8D010FFF712
:10E1180091FD003018BF0120F8BD4FF42045816201
:10E12800C4F8D050D7E73068C4F8D0100B468269DD
:10E1380092060CD41A46013B002AF8D1C4F8D03014
:10E14800E5E7416A03F8011B013AD2B2D3E7C4F804
:10E15800D0302023C3610120F8BD00BF0C1000207F
:10E16800F8240020009800FC400070B5C5B2324881
:10E17800324B00684FF42044C3F8D0408669360417
:10E1880004D52646013C002EF8D113E046682C4CF5
:10E19800344044F0807444F490342C4344604FF489
:10E1A8002044C3F8D0408669B60729D42646013CE6
:10E1B800002EF8D1C3F8D0401CE02146013C0029CC
:10E1C800F8D081690E06F8D544681D49214041F010
:10E1D800007141F48031294341604FF42041C3F874
:10E1E800D0108469A40711D40C460139002CF8D149
:10E1F800C3F8D010FFF71EFD003018BF012070BD16
:10E208004FF420448162C3F8D040DAE782624FF4C9
:10E218002042C3F8D0208169890606D41146013A04
:10E228000029F8D1C3F8D020E4E7C3F8D020202390
:10E23800C361012070BD00BF0C100020F82400202D
:10E24800009800FC026D036B70B50446D5699BB954
:10E25800A90611D5C36A1BB1908C80B298470BE010
:10E26800E169928C40694E1CD2B2E6614254E16980
:10E27800E268914228BFE361616BA1B92A0612D511
:10E28800636AA26A9A42236D09D0501CA669A062EB
:10E29800B25C1A852369984205D3A16203E01A6823
:10E2A80022F080021A602B0742BF236D08221A62EF
:10E2B80070BD026BC168034610B5406942B11A6C63
:10E2C8008C1A013A005D08BF0A46C0B21A6410BD34
:10E2D8001A6A805C01328A4228BF0022C0B21A62E0
:10E2E80010BD436B13B190F844007047836A406ACD
:10E2F8001B1A584258417047036B13B15B68016C95
:10E3080001E0C369016A8B423CBFC2689B18581A76
:10E31800C0B27047836A8169426B1944D160416A0F
:10E3280099429DBF0169CB1A5360CB1A96BF00234F
:10E33800536083624FF0000380F84430136888BF4D
:10E34800816243F0010313607047436A8269D154C4
:10E35800436A02690133934228BF00234362436B37
:10E368001BB11B68DB0705D4D4E7026D136843F0C3
:10E37800800313607047274A73B55369264C43F4EA
:10E388000013536103236946082501268DF80530DB
:10E39800204600238DF806308DF8073000958DF85B
:10E3A8000460F8F707FB1D4AA561138823F04003B2
:10E3B8001B041B0C1380138823F038031B041B0C4D
:10E3C8002B43138013889BB243F04003138024200F
:10E3D800258501F07FFD802001F07CFDA56164208A
:10E3E800FBF700F92585202001F074FDAF2001F02E
:10E3F80071FD3046A561FBF7F5F82585232001F06E
:10E4080069FD602001F066FDA5616420FBF7F5F861
:10E4180002B070BD001002400010004800300140FA
:10E428002DE9F0410369C76805460E461F40002FD5
:10E4380035D0B7FA87F24FF00043D340DB432B6166
:10E448001F40A2F11B03042BF1D8DFE803F0221FC1
:10E458001C190300746A24B1013C0023A4B273623E
:10E4680001E0EC6AA4B2D6F82080B8F1000FDED043
:10E47800D8F80030404621469847D8F80480F4E799
:10E488003068696B07E07068A96B04E0B068E96BF5
:10E4980001E0F068296C036889B29847C7E7BDE8CE
:10E4A800F0814171FEF7B2BA8160FEF7AFBA014858
:10E4B8000149B5E700480140E41D00200148024930
:10E4C800AEE700BF00340140941D00200148024916
:10E4D800A6E700BF00340140941D0020014802490E
:10E4E8009EE700BF000800406C1D0020014802495B
:10E4F80096E700BF00040040441D00204FF0804014
:10E5080000498DE71C1D002010B5054C0548214623
:10E51800FFF786FF04F1C8010348BDE810407FE714
:10E52800F41C0020002C014000440140014802492D
:10E5380076E700BF002C0140F41C0020224B10B5E8
:10E54800224C5A43224BB3FBF2F203880139013AB9
:10E55800A04289B292B29BB20ED004F50064A042E8
:10E568000AD0B0F1804F07D0A4F59834A04203D068
:10E5780004F58064A04202D123F070039BB2154CCD
:10E58800A04206D004F58064A0421CBF23F4407367
:10E598009BB203800D4BC162984202850FD003F5F0
:10E5A800006398420BD003F54063984207D003F507
:10E5B8008063984203D003F58063984201D1002319
:10E5C80003860123436110BD40420F00002C014027
:10E5D80000A24A0400100040134B800A984220D041
:10E5E8000AD84A3B984212D00133984211D0B0F56C
:10E5F800801F14D1012070470C4B98420BD0013377
:10E6080098420AD0053B984209D10420704702205D
:10E618007047032070470520704706207047FE208A
:10E6280070470020704700BF4B00100051001000D9
:10E63800F8B50468064620460F461546FFF7CCFF96
:10E6480006284BD8B27A910847B902238B40D4F8F0
:10E658000CE0DB439BB203EA0E03E3600A23204A83
:10E6680003FB001342F82370043342F82350154685
:10E678003FB1B17AE268890802238B409BB2134309
:10E68800E360282202FB00522032EFF31286502367
:10E6980083F3128803B203EB8303DB0003F10C015D
:10E6A8001C3329442B4451F8047F17B117600A68BA
:10E6B80004329942F7D100231360F3B283F311882F
:10E6C800282303FB0050036A1BB1E36843F00103EE
:10E6D80003E0E2684FF6FE731340E360F8BD00BF45
:10E6E800F41C00200048ADE5FC2500200048A9E501
:10E6F800502600200D4B0E484FF400525A600D4A28
:10E7080011684FF6FE730B401360D0F8882011682B
:10E718004FF6FE730B401360826FC36F9A4201D0AD
:10E728005430F7E5012380F8983070470000024024
:10E73800FC2500204400024010B54B88DC0641BF90
:10E748002F4B14791B6853F8244044BF2D4B43F8D2
:10E7580020404B889B0641BF294B54791B6853F8CE
:10E76800244044BF274B43F820404B881C070ED554
:10E77800254B0C781B78B3EB141FA1BF204BD47822
:10E788001B6853F82440A4BF1E4B43F820404B8815
:10E798009B070ED51D4B0C781B78B3EB141FDFBFFE
:10E7A800174B54781B6853F82440DCBF154B43F8CB
:10E7B80020404B88DC070FD5154C0B78247803F0E4
:10E7C8000F03A342DFBF0E4B14781B6853F8244095
:10E7D800DCBF0C4B43F820404B885B070FD50B7808
:10E7E8000C49097803F00F038B42A1BF044B9278C0
:10E7F8001B6853F82220A4BF024B43F8202010BD09
:10E80800F0240020B20D0020DF1E0020DD1E0020B5
:10E81800DC1E0020DE1E0020254A2648264900234B
:10E82800F0B5156803700B701C461A462E197688C9
:10E838004EB92F5D3FB9037000230A704B700778FB
:10E848001C461A460CE0360548BF013204F10404A0
:10E8580003F1010348BFD2B2802CDBB2E6D1EAE76C
:10E86800E0B2B8420CD215F8240006099E4200F026
:10E878000F00A8BF731C9042A8BF421C0134EFE7E9
:10E888008A704B70C2F3470102F001020A444C1E21
:10E898000A490B480A70C3F3470203F00103134403
:10E8A80004700849501E084A08701370F0BD00BF74
:10E8B8000C1C0020D41E0020A4260020DE1E0020F0
:10E8C800DC1E0020DF1E0020DD1E00202DE9F04F99
:10E8D800C24BDA682DED028B1A61C14A1168D96002
:10E8E800C0490B6843F020030B60BF4B197801291E
:10E8F80090460CBF002201221A70BC4B1A7891076F
:10E9080089B040F13D83BA490978042940F2388337
:10E91800B849097801F0040101F0FF0011B922F0AB
:10E9280001021A701B78DB0702D408B1FDF730FF2B
:10E93800B149CA78531C052293FBF2F202EB82021A
:10E948009A1AAE4BCA701B78039392000023AC4C02
:10E95800DFF8CCC2DFF8D8925CF8231091FBF9F508
:10E9680004F1080004F1100640F82350A54844F8C3
:10E97800231000FB051142F2107091FBF0F080B2F9
:10E9880026F813004FF0140E04F1140604F13C0AA3
:10E998000EFB036E5AF823605EF802704EF8021000
:10E9A800F61B314444344AF82310052691FBF6F14E
:10E9B80009FB051144F82310039C012C4FEA830B33
:10E9C800E24605D10238B0F5797F98BF4BF80C10B4
:10E9D8000BB90123BBE7884CD8F80030226D9FEDB6
:10E9E8008A7A8A4E8A4D9B1A07EE903AF8EE677A31
:10E9F800D8F800302365C7EE877A7C4B1B78B7EED2
:10EA0800008AF4EEC87AF1EE10FA58BFF0EE487AB0
:10EA180013F00103C4ED157A12D005AA00927D4BBC
:10EA280006AA01920CCB9AE80300FDF7AFFD64211A
:10EA3800059A069BB2FBF1F293FBF1F3328000E0FA
:10EA480033802B8094F858306B48002B3BD0D0EDA6
:10EA5800157AC26DDAF80030C8EE276A9B1A026E82
:10EA6800022507EE103AB8EEC77ADAF8043027EE36
:10EA7800267A9B1AFDEEC77AB0F9662017EE901A2F
:10EA880007EE903A644BB8EEE77AD3ED007A67EE7A
:10EA9800277A67EEA67AFDEEE77A17EE903A02FA41
:10EAA80083F3B0F9642093FBF5F302FA81F29BB289
:10EAB80092FBF5F292B2A0F86A30A0F86820A0F8AC
:10EAC8006630A0F86420012384F85830534BDAF8F4
:10EAD80004101B88DAF80000474D514E216603F0F8
:10EAE8003003E065002B00F04B8205F174030093BE
:10EAF80005F178030193EA6E2B6FFDF747FD726805
:10EB08002B6F9B1A07EE903A434B326893ED007ACD
:10EB1800EB6EF8EEE77A9B1AEB67384B67EE877A6D
:10EB28001B78FDEEE77A012BC5ED207A03D0022B86
:10EB380000F0DF8024E2D5ED287A3A4BD5ED215A52
:10EB480095ED255A95ED156A95ED264AD5ED274A96
:10EB580035491D68B1EE677ABDEEC77AFDEEE77AF2
:10EB680017EE10EA17EE90CA0020304A91ED007AAD
:10EB780052F8207007EE907AF8EEE77AA2F11403C3
:10EB880067EEA57A33F81060FDEEE77A283217EEC3
:10EB9800903A9B1B9BB222F810301BB207EE903ABA
:10EBA800F8EEE77A3B4467EE857A4400FDEEE77AB3
:10EBB800CDED037A07EE903AF8EEE77ABDF80C80CF
:10EBC80067EE847AA7EE867AFDEEC77A17EE902A6A
:10EBD800724531DB6245A8BF62462EE0A4060020DC
:10EBE800E8270020D018002076100020D418002034
:10EBF800DA180020F52B0020A42600203C0F002066
:10EC0800A8260020806967FF00007A444E1900207A
:10EC18005019002078100020F800002098190020D2
:10EC2800DC180020400F0020700F00202027002053
:10EC380080969800DB0FC940724607EE902AF8EEDE
:10EC4800E77A5FED046AC1ED007AFDEEE77A3136C6
:10EC580017EE903A43449AB2AB78D1ED027A07EEB8
:10EC6800103AB8EE477A4B684F6027EE267AFB1ABF
:10EC780088EE077AB6B2622E06EE903AF8EEE66AA9
:10EC880037EE067AC6EE866A86EE077A76EEE76A89
:10EC9800E7EE267AC1ED047AC1ED027A0FD964EE67
:10ECA800A77ABA4EFDEEE77A17EE903AB3F5FA6F07
:10ECB800A8BF4FF4FA63B342B8BF334600E000235D
:10ECC80013441BB240F6B8329342A8BF1346B04A69
:10ECD8009342B8BF1346AF4AA352AF4A142303FB6B
:10ECE800002351F8142B1A60002840F049810120B4
:10ECF8003BE7AA4BD5F874801F68D4F878903E8912
:10ED0800DFEDA78A4FEA58039E4228BF1E46B5F892
:10ED1800A8301AB29642C3BFD5ED157A9FEDA17AF5
:10ED280067EE877AB6B2C1BFFDEEE77A17EE906A52
:10ED3800F618B6B2C8BFA5F8A860D4F8AC50C5EBB1
:10ED480009052846FDF766FC0028D8BF404241F275
:10ED580093129042CCBF0020012088B307EE905A4E
:10ED6800B8EEE70A20EE280AFCF784F907EE908A45
:10ED7800F8EE677A40F6B83320EE270AFDEEC07A3F
:10ED8800CDED037ABDF80C20A4F8B02012B29A4257
:10ED9800A8BF1A467E4B9A42ACBF09EB02034B440C
:10EDA80048F6A042934203DDA3F50C43A03B04E0E0
:10EDB800002BBCBF03F50C43A033C4F8B43001E00A
:10EDC800C4F8B490D4F8B450C5F50C53283307EE02
:10EDD800903AF8EEE77A67EEA88AB0EE680AFCF790
:10EDE800A9F98DED070AB0EE680AFCF743F9D4EDEE
:10EDF800317AD4ED2E4AD4ED155A94ED2F4A94ED7C
:10EE0800305A65498DED060AB1EE677ABDEEC77ACC
:10EE1800FDEEE77A0DF1180E17EE10AA17EE90BA6C
:10EE28000020614AFEEC016A32F91030DFF88C915B
:10EE380007EE903A07EE106AF8EEE77AB8EEC77A6E
:10EE48003C32D6EE877A4FEA400CFDEEE77ACDEDFC
:10EE5800037ABDF90C30B3F57A7FA8BF4FF47A7303
:10EE68004B45B8BF4B461FFA83F922F810900FFAAA
:10EE780089F207EE902AF8EEE77A27EEA47ABDEE3B
:10EE8800C77A8DED037A27EE847AD1ED007ABDF842
:10EE98000C90E7EE257AFDEEE77A17EE902A5245B8
:10EEA80003DB5A45A8BF5A4600E0524607EE902AAF
:10EEB800F8EEE77A9FED3D6AC1ED007ABA7891EDF8
:10EEC800027A06EE902AF8EE666A4A684B6066EEA9
:10EED800866A9A1AC8EE266A143106EE102AB8EE27
:10EEE800C66A76EEA56A86EE256AC5EEA66A36EE8D
:10EEF800476AA6EE867A01ED017A01ED037A25EEDE
:10EF0800077ABDEEC77A17EE103ABDEEE77A4B44A2
:10EF180017EE102A13441BB240F6B8329342A8BF2A
:10EF280013461B4A9342B8BF13461A4A2CF80230BC
:10EF38001F4A142303FB0023C3ED007A08B90120FC
:10EF48006FE73B7923B1642395FBF3F5194B1D80DB
:10EF58003B8898450DD9D4F8AC30A06FC01AFDF79E
:10EF680059FB80EAE072A2EBE07242F210739A4217
:10EF780006DD114B01221A700E4BB4F8C8201A8016
:10EF880009B0BDEC028BBDE8F08F00BF30F8FFFF81
:10EF980048F4FFFFC40F0020980F0020400F002006
:10EFA800D30237390000C8420C270020DB0FC940C4
:10EFB800700F0020380F00203C0F002018FCFFFFC6
:10EFC80007B5064B0093064B01930649064A074BC3
:10EFD8000748FBF7BEFF03B05DF804FBEC780108B7
:10EFE800C17801088C8701089D870108E07801082D
:10EFF8006987010808B5037833B90C4B0C481978B0
:10F00800BDE80840FBF7A5BF05F04EFD02280CD867
:10F01800064B1870074B0C2202FB0030064B0630DB
:10F028001860FCF77BF90548E5E708BD7027002064
:10F03800A48701088C18002070100020D77B0108D5
:10F0480008B503783BB90B4B0B4893F8A417BDE8F8
:10F058000840FBF77EBF05F027FD022808D8054BBE
:10F0680083F8A407FCF7C0F8FCF77CF90348E8E745
:10F0780008BD00BFEC100020A8870108D77B010855
:10F0880038B5037803BB214B1B6801330F2B07D816
:10F098001F490C2202FB03121C4695682DBB00E099
:10F0A8001C4601340F2C01DD002400E005D8184966
:10F0B8000C2202FB04129568BDB99C42F1D1154897
:10F0C800BDE83840FBF745BF05F0EEFC0F280446C5
:10F0D80005D80F4A0C2303FB00239D682DB9214650
:10F0E8000D48BDE83840FBF734BF084B1C60FAF701
:10F0F800E1FB21462A460948FBF72BFF0C235C431A
:10F10800034B185DBDE83840FAF7ECBBFC00002063
:10F1180088680108B5870108CB870108E3870108DB
:10F1280073B5037813B9F9F7CFFB3DE01F4901AA7E
:10F1380005F01BFD002401462646254699B134B149
:10F14800012C08D1084605F0AFFC064603E0084646
:10F1580005F0AAFC05461549002001AA05F005FDA1
:10F1680001340146EAE70B2D02D911480C220BE0C5
:10F17800022C10D1A6F57A73B3F57A7F07D90D481A
:10F188004FF47A714FF4FA62F9F71BFB0CE00A4B63
:10F1980003EB45035E80084B084803EB450329460B
:10F1A800B3F90220FBF7D5FE02B070BDE680010876
:10F1B800707E01085984010870270020FA87010829
:10F1C80038B50D4C23688342054606D1FAF799F8FD
:10F1D800204600214C2205F0CCFBE36CAB4209D160
:10F1E8002846FAF78EF8054800214C22BDE8384039
:10F1F80005F0BFBB38BD00BFAC190020F8190020CE
:10F20800034B1A68D379591C1344D171187A704783
:10F218007819002010B5FFF7F3FF84B2FFF7F0FF6D
:10F2280004EB002080B210BD10B5FFF7F3FF0446D1
:10F23800FFF7F0FF04EB004010BD064B10B5044685
:10F2480021461868FAF7EAFB034B1B689879604077
:10F25800987110BD7C19002078190020014B1B689B
:10F268009879EAE77819002038B5044624200D4635
:10F27800FFF7E3FF4D20FFF7E0FF002C084C14BF19
:10F2880021203E20FFF7D9FF2368002228469A71E3
:10F29800FFF7D3FF236893F84900BDE83840CCE76F
:10F2A8007819002001460020DEE710B50446C0B2F8
:10F2B800FFF7C3FF200ABDE81040BEE710B50446BB
:10F2C80080B2FFF7F2FF200CBDE81040EDE737B53C
:10F2D80082888368044610060D4641BF2B4991F881
:10F2E800A4174FF4CC7000FB0133D10544BF284963
:10F2F800097802F03F0244BF01EB410103EB8103AF
:10F30800042A12D006D8012A0DD0022A32D193F944
:10F31800001030E0102A0AD0202A0AD0082A29D161
:10F32800B3F9001027E0197825E0198823E0196857
:10F3380021E093ED000A6846FBF7A0FC014615485A
:10F34800FBF707FE05B3D4ED037A6846B8EEE70A83
:10F35800FBF794FC01461048FBF7FBFD94ED040A0B
:10F368006846B8EEC00AFBF789FC01460A48FBF775
:10F37800F0FD09E000210948FBF7EBFD25B108483D
:10F38800E1682269FBF7E5FD03B030BDEC10002011
:10F3980070270020D27F0108CB7F01080D88010863
:10F3A80009880108024B0146D869FAF737BB00BF44
:10F3B8007027002010B5441E14F8011F21B1034B1B
:10F3C800D869FAF72BFBF7E710BD00BF70270020BC
:10F3D80010B503781BB90A48BDE81040EAE705F004
:10F3E80063FB0446062899BF2146064806480621BD
:10F3F800FBF7AFFD601E40B2BDE81040F9F7EABE6A
:10F40800108801085788010883880108F7B52B4937
:10F418002B4B08782B4D1C682B4B05EB80001A886A
:10F428002A4BD0F8C0101B78294800914FF47A7104
:10F43800B4FBF1F1FBF78DFD26484821FBF789FD68
:10F44800254B1F680026F3B205EB8302D2F8D010D3
:10F45800E9B101249C403C4217D0220715D01F4A2D
:10F46800D25C0B2000FB0323164A1D4802EB8303E2
:10F47800D3F8F020FBF76DFD022C06D1194B93F859
:10F48800281011B11848FBF764FD0136DBE717486F
:10F49800FFF790FF164B17481A68174B9A420CBF94
:10F4A800164B174B1A88174B198892B24FF4FA6308
:10F4B80003B0BDE8F040FBF74CBD00BF20190020A9
:10F4C800E827002088680108C018002000010020F3
:10F4D800AE880108F1880108D01800200801002032
:10F4E800018901087027002009890108518901084C
:10F4F8000C1000200D890108005400401010002055
:10F5080012100020081000202DE9F0410024804648
:10F5180025460F4EA7594146384605F0ADFA58B171
:10F5280039460C48FBF715FD30190021FFF7CFFECF
:10F538000948FFF73FFF0135143440F644439C4225
:10F54800E7D11DB90548BDE8F04133E7BDE8F081D2
:10F55800286A01086880010851890108E27E0108CB
:10F568002DE9F04F2DED028B83B0054605F045FAE5
:10F57800064620B1012818D12B782A2B15D15C48D2
:10F58800FFF718FF00245B4D5B486159FBF7E1FC6E
:10F5980028193146FFF79BFE5848FFF70BFF143434
:10F5A80040F644439C42EED19CE028463D2105F0BC
:10F5B80016FA002800F08F800346994613F8012DAB
:10F5C800202AFAD0441C204605F06EFA80462046D0
:10F5D800FBF7CAFAC5EB0909B0EE408A0026DFF846
:10F5E80034A1142202FB06F40AF5D07B54F80B7000
:10F5F800384605F002FA03461A462846394601936A
:10F6080005F004FA019B00285BD15FFA89F29A425F
:10F6180057D10AEB0402D2ED6B7AF8EEE77A0BEBDE
:10F628000405B4EEE78AF1EE10FA48DBD2ED6C7A05
:10F63800F8EEE77AB4EEE78AF1EE10FA3FD8B2F8BE
:10F64800A431D2F8A82113F0200F08BF08EE108AC1
:10F658001C0641BF2A4991F8A4174FF4CC7404FB47
:10F668000122D90544BF2749097803F03F0344BF65
:10F6780001EB410102EB8102042B18EE100A0BD0BA
:10F6880004D8013B012B0ED810700CE0102B05D0CC
:10F69800202B06D0082B06D1108004E082ED008ACA
:10F6A80001E082ED008A39461748FBF752FC2846EC
:10F6B800002103B0BDEC028BBDE8F04F07E613480C
:10F6C80003E001369D2E8AD1114803B0BDEC028BB0
:10F6D800BDE8F04F6EE6284603B0BDEC028BBDE8EE
:10F6E800F04F11E703B0BDEC028BBDE8F08F00BF0F
:10F6F8003F890108286A01086880010851890108C2
:10F70800EC10002070270020548901085F89010847
:10F71800E27E01088868010808B50748FFF74AFE35
:10F72800064BD869F9F7E2FDFAF7E4FAFBF732FD80
:10F73800034B044ADA6008BD7F890108702700205E
:10F7480000ED00E00400FA0508B50548FFF732FEB1
:10F7580000F036F8FBF748FDBDE80840DCE700BFDD
:10F768008B89010808B50448FFF724FEFBF73CFD28
:10F77800BDE80840D0E700BFA18901080E4B1A7800
:10F788006C2A16D15A88B2F5FA6F12D11A79BE2AA4
:10F798000FD193F8CD27EF2A4FF000000BD113F8C3
:10F7A800012B5040054A9342F9D1B0FA80F0400944
:10F7B800704700207047704700F80308D0FF03081F
:10F7C8002DE9F04F2DED028BEC4D00214FF4FA623C
:10F7D80085B0284605F0CDF8E94B05F537721A6073
:10F7E800E84A00231370E84A05F2A67111606C22FA
:10F7F8002A7003226A714FF48072AA604FF416725D
:10F80800A5F86421FA22A5F866214FF4FA7220219E
:10F81800A5F86C21012285F85E2185F8681185F824
:10F8280069216E2185F86A2185F87C2185F8842173
:10F83800052285F87A1185F81B220A2140F2DC524C
:10F8480085F87B11A5F896212B2140F24C4285F8CA
:10F858007D11A5F89821212140F26C7285F87E115E
:10F86800A5F89A21232140F2753285F87F11A5F871
:10F878009C214FF4C87140F64302A5F89E21A5F8D3
:10F8880080112A462C46032BCCBF0121002103F10D
:10F89800010382F8A01114BF1E217521122B82F8D2
:10F8A800A11102F10202EED14FF4FA63A4F8C631B5
:10F8B800A4F8CA31A4F8CE31A4F8D23140F27E407F
:10F8C800052340F27E5684F8E031A4F84001C823AD
:10F8D80040F23A70A4F8486140F2EA5601274FF422
:10F8E8007A794FF0320BA4F8E431A4F842014FF4CE
:10F8F800C87340F2DC50A4F84A61DFF884A2A4F887
:10F90800E83140F2B4561E211922A4F84601A4F8A1
:10F918004C61A4F8C491A4F8C891A4F8CC91A4F8B7
:10F92800D09184F8E27184F8E37184F8E671A4F860
:10F938004491A4F84EB184F89311029184F8E1211E
:10F9480001920390A4F8503184F8DF7184F8EC71C7
:10F95800A4F852B184F8EF71F6F782FBDAF80030B8
:10F968000299019ADFED897A9FED898A002626732C
:10F97800D97219735521D9700F215971DA71222161
:10F98800212299715A740E2153221974DA7635217D
:10F998005A224FF0780C4FF028084FF02D0E997628
:10F9A8001A720A21642283F80AC0DFF800C283F8B9
:10F9B8000DE0997402911A7783F814E01E7083F8A9
:10F9C800018083F8158083F8028083F81680DE753D
:10F9D80083F804B09E731E76DE735E7683F8098022
:10F9E8009F77C3F838C0C3F83CC0DFF8C4C1C3F878
:10F9F80028C0DFF8C0C1C3F834C04FF4FA7EDFF87E
:10FA0800B8C1A3F84EE0C3ED0B7AC3ED0C7AC3F886
:10FA180048C04FF0140EB7EE087AF1EE047A039856
:10FA280083F850E04FF04B0C83F84CC083ED087A14
:10FA380083ED097A83ED108AC3ED117A4FF0460CF5
:10FA4800A4F8B007042084F8A62784F8A7C784F888
:10FA5800AEE784F8A8B784F8A96784F8AD6784F896
:10FA6800AA6784F8AB6784F8AC6783F85C00152054
:10FA78000192A3F85860A3F85A60A3F85660C3ED42
:10FA8800187A83F8648083F8658083F868004148B1
:10FA9800D866414818674148586783F878704048E5
:10FAA800F6F724FBDAF80030029983F81161C822CE
:10FAB8004FF4487083F8126183F8138183F8147146
:10FAC80083F81861A3F8160184F8D721019A84F8FD
:10FAD800D611A4F8D89184F8DA61A4F8DC21194683
:10FAE8000E2202FB06326FF0170082F8190103207C
:10FAF80082F81A016FF02F0082F81B01072082F8A4
:10FB08001C016FF0230082F81D01052082F81E01F8
:10FB180001365A2081F8200181F821016422FF2052
:10FB2800082E81F81F2181F8220101F10E01D7D199
:10FB3800002183F88911C821A3F88A11142183F8B8
:10FB48008C11A3F890211E214FF4967283F88D1121
:10FB5800A3F892210121282283F88E11A3F8942179
:10FB6800104B18EE102A45F8102F9D42F9D10E4877
:10FB78000021402204F0FDFE20E000BFEC10002030
:10FB8800501000207027002070100020CDCCCC3EF3
:10FB9800000000009A99193FF6287C3F3D0A773FFC
:10FBA8007C930108AC110020881300208FC2F53C1B
:10FBB800000060406666663F000040400023274D15
:10FBC800274C59591A1904330868C2F89C02382B73
:10FBD800F5D104F507700021802204F0CAFE05F172
:10FBE8003801702204F5077004F0B8FEFEF714FE21
:10FBF800DAF8006000230125314604F274404FF41E
:10FC0800CC7284F8CC3784F8CA5784F8CB5704F000
:10FC1800A5FE04F20C6031464FF4CC7204F09EFE4F
:10FC2800104B1B681A68C4F8B2275A68C4F8B6277C
:10FC38009A68C4F8BA271A68C4F8BE275A68C4F87C
:10FC4800C2279A68C4F8C627022384F8C85484F8DF
:10FC5800603605B0BDEC028BBDE8F08FCC760108AC
:10FC6800EC100020701000201549D1F8883043F4BA
:10FC78007003C1F88830134B1A6842F001021A6009
:10FC88005868114A02405A601A6822F0847222F4B5
:10FC980080321A601A6822F480221A605A6822F4A4
:10FCA800FE025A60DA6A22F00F02DA62186B074A1B
:10FCB80002401A6300229A604FF000638B6070471D
:10FCC80000ED00E0001002400CC07FF8CCFC00FF03
:10FCD80038B5094B93F8CC5765B9084C2068F9F743
:10FCE80010FB074B25601B78022B03D1BDE8384079
:10FCF800F6F775B938BD00BFEC10002008280020C1
:10FD080005280020044B93F8CC371BB9034B18681F
:10FD1800F9F778BE00207047EC1000200828002072
:10FD280038B505460446204614F8011B21B1034B9B
:10FD38001868F9F773FEF6E7401B38BD082800205D
:10FD48000FB407B504AB064953F8042B0193002000
:10FD5800FBF712F803B05DF804EB04B0704700BF7E
:10FD6800D7FE0008024B01461868F9F757BE00BFD6
:10FD780008280020F8B5011F06460023083051F86E
:10FD8800042F02F120043F2C3AD802F108040F2C6A
:10FD980006D80232032A04D9002B08BF012300E049
:10FDA80002238142EBD1012B30680ED0022B1AD0EE
:10FDB800736803F003039B0000F0030043EA00109C
:10FDC800B36803F00303184317E000F00F0040F096
:10FDD8004000FFF7C7FFB068736800F00F0040EA03
:10FDE8000310C0B209E000F03F0040F08000FFF7C8
:10FDF800B9FF3079FFF7B6FF307ABDE8F840B1E7D0
:10FE080006F10C0734463A46002552F8043D03F142
:10FE18008001FF294FEA850510D903F50041B1F5A6
:10FE2800803F02D245F0010508E003F50003B3F175
:10FE3800807F34BF45F0020545F00305B242E4D1A6
:10FE480065F03F00C0B2FFF78DFF05F00303022BFA
:10FE5800207807D0032B0CD0012B13D1FFF782FF9A
:10FE680060780FE0FFF77EFF6078FFF77BFFA078F0
:10FE780008E0FFF777FF6078FFF774FFA078FFF7D7
:10FE880071FFE0780434FFF76DFFBC424FEAA50527
:10FE9800DBD1F8BD10B50446C0B2FFF763FFC4F369
:10FEA8000720BDE810405DE710B504467F2C06D951
:10FEB80064F07F00C0B2FFF755FFE409F6E7E0B24F
:10FEC800BDE810404EE7430083EAE070ECE70846DF
:10FED80048E700BF40F2E9330F4A1289920704D479
:10FEE800013B9BB2002BF7D10BE00C4A40F2E933FF
:10FEF800107009490989C9070AD4013B9BB2002B34
:10FF0800F7D1074A138801339BB21380FF2070474B
:10FF18001078C0B2704700BF003001400C3001407B
:10FF2800B42700200C4B0D49DA684378D243C2F35A
:10FF38000222C2F10402934002781B010A44DBB298
:10FF480082F8003303780122580903F01F0302FAEC
:10FF580003F341F82030704700ED00E000E100E0D5
:10FF680073B50546002100680122FEF7E7FA2A6802
:10FF780013889BB243F001031380EB7A8DF80430A9
:10FF88000124002601A88DF805408DF806608DF83B
:10FF98000740FFF7C7FFEB7A1B2B0BD1192301A8EA
:10FFA8008DF804308DF805408DF806608DF807400F
:10FFB800FFF7B8FF02B070BDF0B5BE4CA3782DEDC9
:10FFC800028B013B012B85B000F26F81E5788542F9
:10FFD80040F06B812379022B00F06781B64B5B5DA3
:10FFE8006371A3796D00F2EE048A1BB16319B3F94A
:08FFF800083009E06319D4EDA3
:020000040801F1
:10000000037AB3F90830F1EE677AC4ED037A5B4204
:1000100008EE103A2369A94EB8EEC88A1A0388EE92
:10002000288A35D5D6ED037AFDEEE77A28EE280A40
:1000300017EE903AD6ED057A8DF80A30FDEEE77AA4
:1000400017EE903A8DF80B3004F0ECFEFCEEC07A1F
:1000500096ED060A17EE903A20EE280AADF8083021
:1000600004F0E0FEFCEEC07A96ED070A17EE903A37
:1000700020EE280AADF80C3004F0D4FEFCEEC07A75
:100080000C2017EE903A02A9ADF80E30F7F772FF88
:10009000D4ED077A894BF5EE407AF1EE10FA60D193
:1000A000D3ED067AB4EEE78AF1EE10FA04DDDA68F1
:1000B00083ED068A5A61E8E0F5EEC07AF1EE10FAB7
:1000C00040F3E38093F8202042B1022A00F2DD8061
:1000D0005A6B83ED078AFA329A63D6E0D3ED037A3E
:1000E00038EE678AF7EE007AB4EEE78AF1EE10FA9E
:1000F000ACBF01210021D3ED0A7A69B19FED717A7D
:1001000027EE877ADFED707AB4EEE77AF1EE10FA37
:1001100058BFF0EE477A03E09FED6C7A67EE877A7E
:10012000C3ED0A7A2369654A1B0311D58DF80810BF
:100130005379116B0B440B205A788DF80920DA7A29
:100140008DF80A205B7D8DF80B3002A9F7F712FFBE
:100150000123226B84F82030637913440022DA7281
:1001600091E0B4EEE78AF1EE10FA48BF83ED078A1A
:10017000A16B636B94ED067AD4ED076A591AC943F3
:10018000C90F77EE667A59B9B7EE006AF4EEC67A0F
:10019000F1EE10FA79DDB4EEE68AF1EE10FA74DDD4
:1001A000D4ED056A454BB4EEE67AF1EE10FACCBF19
:1001B0000126002666B1D3ED097A9FED427A67EEFB
:1001C000877A9FED427AC3ED097AD3ED0B7A0AE084
:1001D000B0EE007AF4EEC77AF1EE10FA08DDD3ED56
:1001E0000B7A9FED387A67EE877AC3ED0B7A07E0DA
:1001F000D3ED097A9FED357A67EE877AC3ED097AF8
:10020000D4ED097A206B627967EEA87A1044FCEE8F
:10021000E77ACDED017A9DF804304370D4ED0B7A86
:100220002769FCEEE77A3F03CDED017A9DF80420C3
:1002300042750ED546EA41018DF808108DF8093057
:10024000C37A8DF80A300B2002A98DF80B20F7F73E
:1002500091FE94F82020194B022A11D1D3ED0A7A8D
:100260009FED1B7A196B67EE877A002283F82020B6
:10027000FCEEE77A5A7917EE903A0A44D37202E01C
:10028000022283F82020FCF7F3FAA2790B4B0AB183
:10029000104A00E0104ADA602544D4ED037AB5F93B
:1002A000083000EE103AB8EEC00A80EE280A37EEA9
:1002B000C00A05B0BDEC028BF0BD00BFB427002022
:1002C000A4770108EC51783F6F12833A0AD7833F35
:1002D00000007A440000A0410000A0C12B4BF0B503
:1002E0002B4D1E6805F110002F78F3192C46597814
:1002F00001F00401013501F0FF0219B18542F3D18B
:100300000020F0BD224D631B022B0ADD1AB102EB67
:1003100082025200D2B215F8013B303B1A44D2B2ED
:10032000F1E70021AC420AD919B101EB8101490082
:10033000C9B215F8013B303B1944C9B2F2E72E2F80
:1003400016D10134042000232578771903EB8303A9
:100350007F785B007F079BB244BF303D5B1900F1A3
:10036000FF3044BF01349BB210F0FF00ECD100E03D
:10037000002308484143642000FB03130620B3FB1D
:10038000F0F3054800FB0230F0BD00BF1001002073
:10039000F027002040420F008096980030B50023DF
:1003A0001A4610498C1894F83C40BCB12E2C06D14A
:1003B000013298B18C180444002584F83C50114453
:1003C0000A2491F83C106343A1F13004092C9CBF2E
:1003D000303B5B180E2A03D80132E2E7184630BDE5
:1003E000002030BDB42700200EB40FB5074901909E
:1003F00006AB01A8064A0393FAF7C2FC019B002250
:100400001A7004B05DF804EB03B07047B1AA00089D
:10041000847E01082DE9F04FAA490B7813F0010FF3
:1004200087B003F0040200F07381002A40F07D8160
:10043000A548076817F0806740F07781980700F1BA
:10044000678143F004030B70A04B1A88A04B1A80FD
:10045000A04B1A6812F4002F984600F014819E4BAE
:1004600080201F70F5F7BEFE08B1FEF7ADFE9B4C75
:100470002678012E40F00781994D95F8CA2722B1C0
:1004800095F8CB370BB19A4203D3012385F8CA37CD
:100490000FE01846114630B191FBF0FE00FB1E1E26
:1004A00001467046F7E792FBF1F285F8CA2793FB05
:1004B000F1F385F8CB3795F8CC371BB1884B002288
:1004C00083F8CC27874B95F8CCA71B6841F66902C7
:1004D00003EBC303934284BF40F2E242B3FBF2F367
:1004E000814A8CBFDBB204231370BAF1000F1FD115
:1004F0008020F8F779FF8146D0B18021F8F750FFCE
:1005000099F80620794B607053F8223099F9000071
:10051000DFF8C891B3F5613F0CBF0222002202212F
:100520008DE8060080215246F9F775F8606008B939
:100530000023A7E0514609F10800142204F01DFA37
:1005400009F12803C9F81C3009F19803C9F82030D3
:1005500009F58473C9F82430654BD8F800201B884E
:10056000A9F8783195F89231624895F88491059010
:10057000002B614B1B68C3F3C00E6B79A3F1190B01
:1005800002F4006CC2F3400AC2F3C03218BF012269
:10059000DBF1000141EB0B01012B14BF0B460123E2
:1005A00095F8CAB7049395F8CB3705689B45534B2C
:1005B0001B7803932CBF4FF0000B4FF0010B711E03
:1005C000C9B24B1E132B39D8DFE803F00C0C0C0C0E
:1005D0000C0C0C0C0AA93BAB273B33121212353B17
:1005E000049B9FE0039B8B42B4BF0023012324E0C4
:1005F0002B78022B0BD105EB810353ED027AF5EE3C
:10060000407AF1EE10FA14BF0123002315E06B18B5
:100610005B79003318BF01230FE0BCF1000F04D059
:1006200009F1FF304342434100E0634603F0010318
:1006300078E0134676E05B4674E013B101238B400B
:100640001F43142E02D80136F6B2B8E7059BC4F852
:100650007C71186819217930F8F756FF0023C4F827
:100660008431A4F88831A4F88A31C4F89431244B39
:10067000D4F890211B68C4F8983184F88001C4F83C
:100680008C21022323701E4B154A1B6892F8E0212F
:100690004FF47A7101FB02331A4A1360D8F8003024
:1006A0001A0609D5184B1B789B0705D5174B1B78E5
:1006B000042B01D9062000E0052007B0BDE8F04F6B
:1006C000F9F714B9F52B002014100020E0100020D9
:1006D0003A0F0020C42700204D1A002004280020D3
:1006E000EC100020601B00200C010020105E0108AF
:1006F000C01A002050100020D0180020F01C00204C
:10070000E8270020EC0E0020D4180020DA18002082
:100710005AB9012007B0BDE8F04FF9F70DB973469B
:1007200000E05346002B89D18DE707B0BDE8F08F7C
:1007300010B5154A1378590725D523F00403137013
:10074000124B1B681B0319D5114C2378A3F1080227
:10075000012A0BD8FF200021F7F70CFC0D4B1B687A
:10076000C4F89831FFF7D2FA0A2306E0012B05D925
:100770000A2B03D0FFF7B0FA012323700420BDE851
:100780001040F9F7B3B810BDF52B0020C4270020A6
:1007900004280020E827002003788B4286BF024B04
:1007A00033F8110000207047A429002070B5002202
:1007B0001346234914180C44247E83EA0423082496
:1007C00013F4004F4FEA430318BF83F4815304F13D
:1007D000FF3418BF83F0010314F0FF049BB2EFD184
:1007E0000132192AE5D100F1190200F11A050A4473
:1007F0000D44167E2A7E02EB062292B29A421ED148
:100800000F4B93F83950E2B2AA4215D2431C03EBC6
:100810004203DBB2CA1801330B44127E1B7E03EB8A
:1008200002239BB24FF4AF6253431B1303F548738B
:1008300021F814300134E6E7012381F83A3070BD25
:10084000A429002003788B420BD9074B1A78074B59
:1008500089001944C86B02B1400800F5777080B276
:1008600070470020704700BF4C1A0020A4290020C8
:1008700007299DBF034B03EB8101B1F86C000020F9
:10088000704700BFA4290020034B03EB4101B1F8DE
:100890008C00C008704700BFA42900200A4BDFED80
:1008A0000B7A03EB810191ED2B7AB8EE477AF6EEE5
:1008B000046AE7EE267A82B0FCEEE77ACDED017AA3
:1008C000BDF8040002B07047A429002000005C4479
:1008D000024B03EB4101B1F8F4007047A42900205A
:1008E000024B03EB4101B1F818017047A429002025
:1008F000024B03EB4101B1F818017047A429002015
:100900000020704770B5334C0546F8F753FED4F815
:100910003031C4F83001C31AB3F5FA5FC4F834318A
:1009200082BF002384F8383184F8393194F83831A3
:100930002BB9A12D02BF274A012182F8391194F861
:100940003911244A29B1D118EDB201330D7682F85C
:10095000383194F8385194F83A31AB4239D11D4BC3
:1009600093F83B31052B02D0062B03D02CE000205E
:10097000FFF71CFF637E1E2B26D100200246C1B26A
:100980006B1E994219DA21440B7E0821DBB283EAFF
:100990000206F60744BF83F01803C3F3460301F1D0
:1009A000FF3154BF5B0843F0800311F0FF01C2F335
:1009B0004702ECD101301A46E1E723441B7E9A42FC
:1009C00002D10320FFF7F2FE002384F8393184F8C6
:1009D000383170BDA429002010B50446F8F7EAFDAF
:1009E0000F4BD3F83C21C3F83C01821A41F2883105
:1009F0008A42C3F8402184BF002283F8442193F83F
:100A00004421074913440F2AE4B218BF013283F886
:100A1000454112BF81F84421012381F8553110BDB1
:100A2000A429002010B50446F8F7C4FD0F4BD3F8F5
:100A30005821C3F85801821A41F288318A42C3F81A
:100A40005C2184BF002283F8602193F8602107496C
:100A50001344142A18BF013283F8614112BF81F890
:100A60006021012381F8763110BD00BFA429002048
:100A700038B50446F8F79EFD274A2749D2F8783161
:100A8000C2F87801C31AB3F57A6F84BF002382F8E5
:100A90007C3192F87C3133B9A82C3BD181F87D317F
:100AA000A1F87E3106E0022B02D181F8804101E0FD
:100AB000242B02D8D11881F8814192F88011164D6B
:100AC00001330231DBB249008B4282F87C3118DA03
:100AD000B5F87E31E0B283EA0020082310F4004F1D
:100AE0004FEA400018BF80F4815003F1FF3318BF74
:100AF00080F0010013F0FF0380B2EFD1A2F87E0175
:100B000038BD01318B4201BF002385F87C310123C0
:100B100085F87D3138BD00BFA429002010B50446FA
:100B2000F8F748FD104AD2F8A83140F6AC51C31A84
:100B30008B42C4BF002382F8AC3192F8AC31D1189B
:100B400081F8AD4123B90F2C0DD10749C1F8A80197
:100B50000133DBB2192B044982F8AC310CBF0123FD
:100B6000002381F8C63110BDA4290020094B1A6862
:100B7000137844F6FB7103EB431300FB0313507827
:100B8000C0EB0030B3FBF0F39078B3FBF0F080B231
:100B9000704700BFBC180020124B10B5D3F8C82115
:100BA00002EB40010C7E14B1022C11D00BE00228A4
:100BB00005D9032807D10C4B1B68DB0401D5D0896C
:100BC00010BD908A10BD03EB4003B3F8F40010BDD4
:100BD000487E00EB800000EB800000F2EE2080B247
:100BE00010BD00BFA4290020C427002008B5F8F7D5
:100BF000E1FC074B022283F8D021064AC3F8CC015E
:100C00001268C3F8DC21012283F8F52108BD00BF7A
:100C1000A4290020E827002008B5F8F7CBFC084BF2
:100C2000022283F8D021D3F8DC2100F5B71000F5BB
:100C3000587002F2DC52C3F8CC01C3F8DC2108BDC5
:100C4000A4290020044B1B6842F201021A420CBF87
:100C500001200020704700BFC4270020114B93F8EB
:100C6000F821012A10B51C460ED008D3022A0FD154
:100C70000D4A938A9BB283F48853938208E00A4B0F
:100C80004FF488521A8503E0074B4FF488529A615B
:100C9000F8F790FC00F5F42000F59070C4F8FC0122
:100CA00010BD00BFA429002000100048034B1A7893
:100CB000202A04BF00221A70704700BFF82B0020C2
:100CC000014B04221A607047DC2B0020034B9B7AF7
:100CD00013B1034B05221A60704700BF8C1C002023
:100CE000DC2B00200D4B0E491A680E4B92B21344B8
:100CF0005B000D4A1B68C3F3090310B5136013684A
:100D00009BB201335B1000229A4206D0074851F88B
:100D1000044B20F812400132F6E710BD505C004051
:100D2000206200401E300020E41E0020E91E00204A
:100D3000014B00221A607047E01E00202DE9F843A5
:100D4000664B674E1B68DFF8B881664A00254FF096
:100D5000C0099D7283F80990DD723560D8F80030C3
:100D600023F4EC4323F0700343F400739BB2C8F800
:100D70000030D8F8003023F4E04323F040039BB266
:100D800048F2800483F010032343C8F8003033682E
:100D900012FA83F35B0040271A681F6033689BB226
:100DA00003F1005303F540535B0028461A68802284
:100DB0001A60D8F8003023F4F8731B051B0D234389
:100DC000C8F80030484B93F82C10F5F7D3FAD8F850
:100DD0000030464A464923F4804323F070039BB217
:100DE00083F440532343C8F80030136823F4EC43E2
:100DF00023F070039BB21360336811FA83F35B0036
:100E000003201968C3F8009013683A4923F4E043BB
:100E100023F040039BB283F0200323431360136845
:100E200023F4804323F0700323439BB21360536881
:100E300023F4EC4323F0700343F4C0639BB253608C
:100E4000336811FA83F35B0019684FF480711960FD
:100E5000536823F4804323F0700323439BB2536011
:100E6000536823F4E04323F040039BB283F0200354
:100E700023435360D8F80C301F4A23F4EC4323F08B
:100E800070039BB2C8F80C30336812FA83F35B002E
:100E900039461A684FF488721A60F5F76BFAD8F879
:100EA0000C3023F4804323F070039BB283F440534F
:100EB0002343C8F80C30D8F80C3023F4E04323F077
:100EC00040031C43A4B2C8F80C402846F5F7C6F905
:100ED0000A4B01221A60BDE8F88300BFA419002064
:100EE000505C0040043000200C000020045C0040F6
:100EF00008300020103000201C300020DC2B0020A7
:100F0000005C0040134A144B50681B68181810B559
:100F1000146808D011490822F9F767FD20461049E6
:100F20000422F9F762FD0F4B1A68002393720E4AF0
:100F3000012111600D4913604FF4E0500B60106007
:100F40000B480B604FF4364101801160094A136071
:100F500010BD00BFB0F7FF1FACF7FF1FDE00002081
:100F6000EE000020A4190020405C0040445C0040DA
:100F7000A42B0020DC2B0020024B4FF480221A60AF
:100F8000704700BF14040140022803D0431E58429A
:100F900058417047064B1B681B7823B1054B1868F6
:100FA000C0F3C0407047044B1878C0F3800070470E
:100FB0004C06002014100020F52B002010B50A4C20
:100FC0005E280146206805D15D21F8F72BFD2068D9
:100FD0003E2105E05D2903D1F8F724FD20683D217D
:100FE000BDE81040F8F71EBDA82B002030B5002842
:100FF000104C114AB8BF40423C2590FBF2F304FB71
:10100000030068430D4D90FBF2F22D682D7B25B94E
:1010100003EB830303EB830301E0C3EB031302EB56
:1010200083030B8004FB02024FF47A7392FBF3F20A
:101030004A8030BD806967FF80969800C418002000
:1010400010B50446C0B2FFF7B9FFC4F30720BDE8EE
:101050001040B3E7024B5E211868F8F7E3BC00BF0D
:10106000A82B002038B5064C05465E212068F8F70D
:10107000D9FC20682946BDE83840F8F7D3BC00BF4A
:10108000A82B0020674B73B51878674DFFF77CFFDE
:101090002B788342044620D0C8B1644B1B68E3B16F
:1010A00093F9000002230093614B1B685B780033C7
:1010B00018BF0123019304214FF416530022F8F7BF
:1010C000AAFA5C4B186040B101232B7005E0594E21
:1010D0003068F8F71AF934602C70574B574D187870
:1010E000FFF752FF2B788342044618D088B1544B47
:1010F0001B68A3B10022012493F9000000944FF46F
:10110000964301920821F8F786FA4E4B186028B9E9
:1011100005E04C4E3068F8F7F8F834602C704A4B14
:101120004A4D1878FFF730FF2B78834204462E464D
:1011300042D0002837D0464B1A68002A3CD0D379D9
:1011400092F90000434C002B08BF022302220092B8
:10115000002254F8233001921021F8F75CFA3E4B3C
:101160000546186040B33D4C94F84A30022B0BD032
:1011700094F89620022A01D14C3405E023B1002ACC
:1011800004F14C0418BF0024354B1C6044B12046C8
:1011900000214C2203F0F1FB0223256084F84A3041
:1011A0000123337008E02C4E3068FEF70DF83068EC
:1011B000F8F7ABF834602C702A4B2B4D1878FFF7FA
:1011C000E3FE2B788342044629D000B3274B1B68EB
:1011D0002BB3274A93F9000012685278002A0CBFFB
:1011E000082209220323009301924FF46143202136
:1011F0000022F8F710FA1F4B186080B11E4A012335
:1012000013702B701D4B1A681D4B1A6007E0194EA6
:101210003068F8F77AF8184B34601C702C7002B004
:1012200070BD00BF54060020D010002050060020E2
:10123000C4180020A82B002055060020E418002028
:101240006819002058190020600600206E1900203F
:101250005C060020105E010870190020AC19002007
:10126000741900206C0600208419002068060020F4
:1012700064060020881900208C190020E82700202F
:1012800090190020064B1B7803F0040303F0FF00C5
:101290001BB1044B1888C0F3C01000F00100704768
:1012A000F52B0020981900202DE9F04F2DED088B2B
:1012B00083B00AEE102A0093D14B01931A8812F0E2
:1012C000020F0546F7EE009A4CD0149BCD48DC89FE
:1012D000B0F900301B1B03F2F31640F2E6329642DF
:1012E00003D8002BB8BF5B4201E04FF4FA73B0F9AA
:1012F0000220121B02F2F31440F2E630844203D8BB
:10130000002AB8BF524201E04FF4FA7295F84C003F
:1013100058B39342B8BF1346C3F5FA7307EE903A39
:101320009FEDB97AF8EEE77A6423C7EE877A93FBEC
:10133000F0F307EE103A77EEE97AB8EEC77AB0EE3E
:10134000699AA7EE879AF7EE006AB5EEC09AF1EEB9
:1013500010FA0AD4B4EE669AF1EE10FAC8BFB0EEF5
:10136000669A04E0B0EE699A01E09FEDA89AA84E53
:10137000CF1C2C464FF00008B8F1020F17F801BF40
:10138000DFF8DC924FEA480AF2EE04AA0ED1B9F96E
:1013900004109FEDA07A0BF10A0B01FB0BF307EE93
:1013A000903AF8EEE77AC7EE877A68E0F8EE4A7A84
:1013B0009FED956A39F91830C7EE867A06EE903AB5
:1013C000954B33F9183007EE103A1AEE103AF8EE52
:1013D000E66AB8EEC77A5B42A6EEA77A07EE903AC5
:1013E000F8EEE77AB4EEE77AF1EE10FA08D4F8EE08
:1013F000CA7AB4EEE77AF1EE10FAD8BFF0EE477A87
:10140000864B33F90A3008EE103A009BB8EEC88AD2
:1014100033F9183077EEC87A08EE103AB8EEC88A79
:1014200037EE888A88EE2A8AFFF72CFF40B17C4B82
:1014300013F80800B0EE480AFEF7C2FDB0EE408A8D
:10144000019B1988CA0704D5D5ED117A68EE277A71
:1014500015E039F90A309FED6F7A0BF1140B03FB9D
:101460000BF307EE903AF8EEE77A8B07C7EE877A30
:1014700042BF95ED127A28EE078AE8EE097A694BA9
:10148000DFF8E0B133F90A3094ED08BA9FED668ACF
:10149000DFF8D49107EE103A644BB8EEC77AD3ED7B
:1014A000046A18F80B30E7EE667AB8F1020FF0EE36
:1014B00048BAF0EE678A67EE8B7A0BEE103AB8EE18
:1014C000CBBA27EE8BBA8BEE08BA09D1B0EE4B0A35
:1014D0005748D9ED000A1E21F9F720FBB0EE40BABB
:1014E000D9ED000A94ED0B7A68EEA07A67EE877A60
:1014F00096ED007AA7EEAA7ADFED4E7AB4EEE77A9F
:10150000F1EE10FAF0EE47AA09D4DFED4B7AB4EE13
:10151000677AF1EE10FAC8BFF0EE67AA01E0F0EECC
:1015200067AA89EEA08A45494FEA8809494491EDA6
:10153000000AC6ED00AAC1ED008A38EEC00A95F88F
:10154000501020EE080A21B13D4800EBC800F9F721
:10155000E5FAD4ED0E7A1BF8083060EE277A00EE3B
:10156000103AB8EEC00A27EE800ADFED367A80EE38
:101570002B8AB4EEE78AF1EE10FA09D4DFED327A65
:10158000B4EE678AF1EE10FAC8BFB0EE678A01E0E8
:10159000B0EE678A3BEE2A0A08F1010830EE080A2D
:1015A00003F0FAFB2949B0F57A7FA8BF4FF47A70AF
:1015B0008842B8BF0846BDEECBBA25491BEE103AAB
:1015C00021F80A00FDEEEAAA2249BDEEC88A49F8D0
:1015D000013021491AEE903A49F801301F4918EEBE
:1015E000103AB8F1030F49F8013004F1040406F190
:1015F00004067FF4C1AE03B0BDEC088BBDE8F08FEC
:1016000098190020982A00200000FA4300000000EA
:10161000E01B002000004842EE2B0020BC270020E9
:10162000345E0108341000200000C842AC2B0020BA
:10163000541B002000007AC300007A43C02B002016
:101640007C1B0020000096C30000964318FCFFFF9F
:10165000941B00209C1B0020A81B0020B41B002012
:10166000E4100020501B00205C1B0020044B0022D3
:101670001A605A60034B00221A605A60704700BF1C
:10168000C01B0020EC1B002010B50B4C0123E370A5
:101690004FF48060022384F82030F9F767FD074A91
:1016A000074B126A1B685178642212FB0133636195
:1016B00023880133238010BD782B0020AC2B002021
:1016C000E827002008B5044B1B7803F00503052B21
:1016D00001D1F8F713FBFEE7D02B0020D0400B1C04
:1016E0001141203A03D49C461341184363465242A9
:1016F00093401843704700BF81F0004102E000BFF3
:1017000083F0004330B54FEA41044FEA430594EAC1
:10171000050F08BF90EA020F1FBF54EA000C55EAFC
:10172000020C7FEA645C7FEA655C00F0E2804FEACD
:101730005454D4EB5555B8BF6D420CDD2C4480EAAF
:10174000020281EA030382EA000083EA010180EADF
:10175000020281EA0303362D88BF30BD11F0004F2D
:101760004FEA01314FF4801C4CEA113102D0404263
:1017700061EB410113F0004F4FEA03334CEA13339E
:1017800002D0524263EB430394EA050F00F0A780B6
:10179000A4F10104D5F1200E0DDB02FA0EFC22FAB1
:1017A00005F2801841F1000103FA0EF2801843FAA5
:1017B00005F359410EE0A5F120050EF1200E012A96
:1017C00003FA0EFC28BF4CF0020C43FA05F3C018D4
:1017D00051EBE37101F0004507D54FF0000EDCF14D
:1017E000000C7EEB00006EEB0101B1F5801F1BD3F6
:1017F000B1F5001F0CD349085FEA30004FEA3C0CFA
:1018000004F101044FEA445212F5800F80F09A80EF
:10181000BCF1004F08BF5FEA500C50F1000041EBF3
:10182000045141EA050130BD5FEA4C0C404141EBF7
:10183000010111F4801FA4F10104E9D191F0000F1E
:1018400004BF01460020B1FA81F308BF2033A3F1A1
:101850000B03B3F120020CDA0C3208DD02F1140C98
:10186000C2F10C0201FA0CF021FA02F10CE002F1D3
:101870001402D8BFC2F1200C01FA02F120FA0CFCCC
:10188000DCBF41EA0C019040E41AA2BF01EB045115
:10189000294330BD6FEA04041F3C1CDA0C340EDC13
:1018A00004F11404C4F1200220FA04F001FA02F356
:1018B00040EA030021FA04F345EA030130BDC4F114
:1018C0000C04C4F1200220FA02F001FA04F340EA09
:1018D0000300294630BD21FA04F0294630BD94F0BA
:1018E000000F83F4801306BF81F480110134013DA1
:1018F0004EE77FEA645C18BF7FEA655C29D094EA12
:10190000050F08BF90EA020F05D054EA000C04BF8F
:101910001946104630BD91EA030F1EBF002100207A
:1019200030BD5FEA545C05D14000494128BF41F019
:10193000004130BD14F580043CBF01F5801130BD7D
:1019400001F0004545F0FE4141F470014FF0000008
:1019500030BD7FEA645C1ABF194610467FEA655CB9
:101960001CBF0B46024650EA013406BF52EA03355B
:1019700091EA030F41F4002130BD00BF90F0000F49
:1019800004BF0021704730B54FF4806404F1320485
:101990004FF000054FF0000150E700BF90F0000F3E
:1019A00004BF0021704730B54FF4806404F1320465
:1019B00010F0004548BF40424FF000013EE700BF35
:1019C00042004FEAE2014FEA31014FEA02701FBFC5
:1019D00012F07F4393F07F4F81F06051704792F097
:1019E000000F14BF93F07F4F704730B54FF4607411
:1019F00001F0004521F0004120E700BF50EA01025C
:101A000008BF704730B54FF000050AE050EA010208
:101A100008BF704730B511F0004502D5404261EB78
:101A200041014FF4806404F132045FEA915C3FF4B9
:101A3000DCAE4FF003025FEADC0C18BF03325FEA52
:101A4000DC0C18BF033202EBDC02C2F1200300FA07
:101A500003FC20FA02F001FA03FE40EA0E0021FA2C
:101A600002F11444C1E600BF4FEA4102B2F1E04383
:101A700024BFB3F5001CDCF1FE5C0DD901F0004C75
:101A80004FEAC0024CEA5070B2F1004F40EB8300C5
:101A900008BF20F00100704711F0804F21D113F1F1
:101AA0003872BCBF01F00040704741F480114FEA2A
:101AB0005252C2F11802C2F1200C10FA0CF320FAB3
:101AC00002F018BF40F001004FEAC1234FEAD323D0
:101AD00003FA0CFC40EA0C0023FA02F34FEA43033A
:101AE000CCE77FEA625307D150EA01331EBF4FF0C3
:101AF000FE4040F44000704701F0004040F0FE40DE
:101B000040F40000704700BF7BB972B90029BEBF26
:101B100000204FF0004106E008BF00281CBF6FF016
:101B200000414FF0FF3000F073B882B0EC462DE971
:101B3000005000F03DF8DDF804E002B00CBC704746
:101B400007EE900AF5EEC07AF1EE10FA01D400F03B
:101B500009B808B580F0004000F004F8404261EB9D
:101B6000410108BDD0B5FFF72BFF00220E4B064602
:101B70000F4600F04FF800F05FFA0446FFF7FEFE54
:101B800000220A4B00F046F802460B463046394622
:101B9000FFF7B6FD00F050FA2346002242EA0002A9
:101BA00010461946D0BD00BF0000F03D0000F041D6
:101BB0002DE9F041069C154606460F46984600F072
:101BC0005BFA05FB01F300FB0838A5FB0023B21A02
:101BD000434467EB0303C4E90023BDE8F08100BF81
:101BE0002DE9F041069C904606460F461D4600F042
:101BF00091FB00FB05F5A0FB082308FB0155B21A79
